:020000040004F6
:10600000A0670020D9D7050033EE040033EE04006A
:1060100033EE040033EE040033EE04000000000011
:1060200000000000000000000000000033EE04004B
:1060300033EE04000000000033EE040033EE0400F1
:106040001C00000054464C33140020001C001800B3
:10605000140010000C0000000800040014000000F0
:106060001C00000080000000D8000000245F000039
:10607000345F000090650000030000000100000094
:10608000040000008AA0FFFF0C0000001C000000BC
:10609000380000000F00000073657276696E675F5C
:1060A00064656661756C7400010000000400000006
:1060B0009CFFFFFF0C000000040000000700000030
:1060C00064656E73655F320001000000040000002B
:1060D000DAA1FFFF0400000007000000696E707580
:1060E000745F310002000000340000000400000072
:1060F000DCFFFFFF0F0000000400000013000000A1
:10610000434F4E56455253494F4E5F4D45544144BF
:106110004154410008000C00080004000800000081
:106120000E00000004000000130000006D696E5FA7
:1061300072756E74696D655F76657273696F6E00F6
:1061400010000000485E0000405E0000B05D0000EE
:10615000905D0000005D0000E85C0000D8110000C8
:10616000C8010000B8000000B0000000A800000056
:10617000A0000000980000009000000070000000E7
:10618000040000008EA2FFFF040000005C0000007D
:106190000C00000008000E000800040008000000C9
:1061A000140000002C00000000000A000C00080091
:1061B000000007000A0000000000000104000000C9
:1061C0000000000000000A0010000C00080004009D
:1061D0000A000000020000000200000004000000AD
:1061E00006000000322E31332E300000F6A2FFFFF1
:1061F0000400000010000000312E31342E30000069
:1062000000000000000000003C9CFFFF409CFFFFDE
:10621000449CFFFF489CFFFF4C9CFFFF26A3FFFF11
:1062200004000000000100002A142B3CDDC800BE61
:106230007F127CBCA9DE03BC5DD571BCAE56CDBC63
:106240001ADD52BCD318263D66CE84BC480441BC3E
:10625000F77B80BE87391EBE6FAF1ABC7769233DBE
:106260004478B53D95AFCA3DF2FDF1BB7E96703DD9
:10627000CD27173E8B17A9BCAB7F36BD2030FDB9AB
:106280007A16D03C02103EBDE61579BD8BCC4ABED5
:1062900029571CBE634C823CAC5B653CA96C253D18
:1062A00059515E3C1569C5BBD08551BC8EF93CBEC9
:1062B0006415543C6ECC2D3C1874993CA3C8CD3C5D
:1062C00043CCFF3B1D83F1BCE7F0A53A7F44DD3BA7
:1062D000429BC23EAB483C3EC9D80C3CB48D74BD19
:1062E000908BA4BDF87D7EBD126D7F3DC24F92BDE7
:1062F0003E4E11BEF121DABBA18F6C3DB3F0C5BBA0
:106300006A56A6BC1541303D8FD5883DAE186F3E0C
:106310009232343EA0F77DBCB2B465BC9F8420BDF0
:10632000377F52BC41E18DBD32A4FFFF0400000065
:10633000001000006D50AC3E9364083F6AE0813C61
:10634000CAA00DBEBA2E15BEA29FDFBE201FEFBD94
:10635000CB43E13DFE46A83E5A8D63BEC8053ABE1A
:1063600059AA8A3BCAD4C73DE11B79BEAACBC03E1D
:106370002531863E3F81E3BE129BA2BEF184C13E21
:10638000D475B3BE7BA2773E7F52F7BDF1F588BDD1
:10639000D06F7DBE9EE496BC298C5D3E5621B9BE71
:1063A000A5763EBE12B0AEBEB5C58C3BE0BFF13D9A
:1063B000C855AFBEAB372FBD78293A3E9FFA833C14
:1063C000AE1810BE8E45D1BD3A8A03BE3AA2783DC2
:1063D000C08E41BEC5C478BE7CF20DBE3B800ABEF5
:1063E000F7286EBD656D103ECC9D7DBE924D0EBEF4
:1063F0009BD0B6BD19C56ABD781C8CBECDDC4E3EA7
:106400007059443D6C7E9BBE634D87BE4C7D15BE6E
:10641000AAFCBFBDC0D130BE25F105BE29B25ABD10
:106420004B0D96BE9B2A86BE20E54A3D69949CBED4
:1064300002213ABE7309ED3E8762683DC8813A3E4B
:106440003C600BBE12ABB53E775A5C3E84568EBDA7
:10645000C31E95BED27870BE145AC7BDD985A33E5F
:10646000B9A92FBE17FD09BEB315DABD984B1E3C66
:10647000EC289DBDF9DB3CBDF1C3193E53B0833E12
:10648000AD6ED2BDF9AB843ED3882DBEB9CC573E9C
:10649000022F243FECC63BBD5A429FBEDD3FCCBD20
:1064A000D3876C3EA0A82E3E83FE1E3C9008BF3EC4
:1064B0003A24833E2EA576BFB31B5F3EED16F23D18
:1064C000F05DC6BBF4FD72BE4A1CF9B8C6A4DC3D43
:1064D0005AE215BE4F20BABDDB393BBE994E093E8C
:1064E0003DD703BFAC47D9BEAF530CBF9C984DBD41
:1064F000E32F8D3C1C49563E451641BD91A40BBE71
:1065000025E2A03E29637A3E03F38ABE590EE83C99
:10651000D242C9BEE5503DBE01FBF23D3291923DF3
:106520008ADD29BF983A39BED0D4BDBCEAAB653EFE
:10653000B413C43EFB0C74BDD74C88BE084D86BD59
:1065400083F816BEB2E863BD41F23ABDF48AB03BAF
:1065500076AA0DBEC2EC49BEEE50FDBCC941FFBCDF
:1065600037D950BCA188BD3D09B55FBD0E47F5BD0B
:10657000498FBFBCF83121BDCB2C0A3E112830BE5B
:106580007992963DF8A2853CB91C17BDC21858BC3B
:10659000EDC7073DBB5A6CBC7CF58E3C70E0E33D1B
:1065A000CEB1453E57F412BE18C2ECBD284C0F3D8B
:1065B0003FE2BABD790B79BD3B35633EE6BDE4BD34
:1065C000A5050ABE8D6A3D3EA711E63E7D62543D9B
:1065D000A7591BBE5CF2833E7347E6BDC95C613EB2
:1065E00014F8943DF7AEF8BEC7BC11BF912484BD2A
:1065F0003017BDBD4B189CBDDC71923EAB9DC43EB7
:106600000A5AD23E10689B3E2AFB36BD7F7255BEA9
:1066100003D612BE819E1C3E9C63933E823145BED2
:10662000DDCB35BE724D91BED9FE463E88E10B3FB3
:106630007FBAA43EB91BB43E95BFD73D37D008BE44
:10664000643321BE6CBBF33EA2EF11BEE1AD41BE8F
:10665000127766BE54F0CD3D2DAC88BDA6CA58BE9B
:1066600040951ABE31595BBDC614BD3D57CE6C3E38
:106670001E5770BDC163C2BDEB8DDC3E9DF46A3E0A
:10668000C0C91ABED6F34D3DA71EC53C28FC04BEAA
:10669000B400C23E104EF73D52D889BEA7F043BEAB
:1066A0002CA5143E849B363E2B416DBDE1438B3EB1
:1066B000363CFA3EA3EC87BD8E4FFC3D1E34353E82
:1066C00084D743BE11366DBEF724A6BE31D6ED3E4B
:1066D0005634CD3EF1AD143F1F61CA3D9B076D3E60
:1066E00024C89F3E4B95483EDF6749BE86500EBD8D
:1066F0000141A53EE57477BF0375583E005D2BBE92
:106700008DDADF3EA0A6EFBDA47B1ABF4566A13E91
:10671000A0E7A0BED19C10BEEA4E21BF2694AA3E9F
:10672000C4E2963CEEB62DBEC3B595BD2AA893BE75
:10673000F05E17BE220E8BBE464ABABB13179ABE36
:10674000049A39BE5F453ABE6550573EDB4D2F3D3A
:106750006C3139BE60BA61BE5DEC4FBE09E55EBE0C
:106760002F138FBC610349BEF328463E048310BE3D
:10677000B79EDE3DD9DE323EE51A023E725C07BFAF
:10678000F7F16FBECAF6803D26D95A3EC87E0F3E4D
:106790005FC78EBE8B0B16BE6AC2EDBD85111ABCDB
:1067A0008AB076BC8496BABCD1F156BEE6DACDBDCD
:1067B00031E31E3E5655213EAF28883EB5AF71BE2F
:1067C00055FE30BEDE114A3ECBA6783ED5837DBD58
:1067D000514EEF3BAD710C3E045E94BE8D59A63D0B
:1067E0003C3D28BE6BBBE43D7215983E6663DEBD42
:1067F000AE2EF63D1CA2EFBE0241193C2B813E3F5E
:10680000609760BE40FE283F227B76BEECD112BE70
:106810005810143F72149A3D5C33183E41439EBE9B
:106820007940B33ED39BD5BC8EAADF3D8EFF7F3D22
:106830005A23AF3E61DAD1BEF98181BC66527BBE7C
:1068400078F97FBEDE338DBEBAE3183DFD8797BD74
:1068500036FED8BD72DC87BE156A153E26AD723E87
:10686000DE9431BE2631E03D285EDFBB52D4D13DFF
:10687000A1E954BE42FE82BEFF46D6BE09E045BE37
:10688000F7B71C3E9F9897BEA03CB8BE0E7F733DE5
:106890008D007FBEFA0DF3BD3D2ED63E4E67C8BEBD
:1068A000B174603C072DF8BE3C5230BF0C48E6BEC8
:1068B000A57CD6BD8AF51BBE8198963DBE277E3E3F
:1068C00086F898BE03152DBE8084463D905FE03D5E
:1068D000B53925BDB8E30F3E5C1347BE158D1A3E92
:1068E0007295D6BDF21AC3BD0EBD0B3EECDD28BEBF
:1068F0001E62B3BEEBE1EFBED6E2E6BD88E7B83E6E
:10690000509D553EFCBC303E590FEBBEB58E1E3E31
:106910004E996CBE9D1C92BE29CE1FBF799EA4BE0F
:106920003D9CE93BA1046B3E0500B5BD53F46FBE31
:10693000395D2CBE1F909D3E24F4773EBB9CEE3DFE
:106940004C2494BEF213863E6A06C13E29257DBDC5
:1069500055C1FE3C2B22913DD22AC93E314D253EE8
:10696000C01E8C3D89DE29BD9083DCBD43E48A3E98
:106970009FFF91BE0B9449BBDA7C0F3E08AEC33E2D
:106980003542F83EE73F583D03701E3ED3B149BE45
:106990005EEF143FBB087D3CB5C02B3E26D866BEDB
:1069A000B99E533D6992033D9831A53E12E3893E5D
:1069B0000EF5D53E820234BD86EC223E359EB0BD3A
:1069C000B5E6F0BEC858CF3D423937BE791AB3BEDE
:1069D000A37BD43D13C538BE1832DABC7C65C9BD73
:1069E0007BD1853D7942E33D9EF1A03CF63760BE08
:1069F00024B510BE7F6AF5BE4F2D0ABFCF7DEB3E9A
:106A0000233225BED03CB7BEF0A1B43EF41CF93D04
:106A10008DF7183EC009AEBED402F53CAA6B3D3DD1
:106A2000E761B53C2229C2BE6AD38C3EB1B75A3E5B
:106A3000D6E92B3E2173033E330423BF9291A2BCBF
:106A40001C8C8ABEAAD88FBE5E8B1CBE37EDEABDF9
:106A5000A15ADDBE3A8FF4BC8EDE273E776175BD4C
:106A60004813993E7CD66A3E378A623E4F8C18BEE8
:106A700036092A3ED6DF09BE600F92BE2E7E90BE3A
:106A8000AD06EBBED46CC7BE6417883EAF251D3F74
:106A90007E27EEBCDAB2433E7C6CE13D026A7A3E70
:106AA0005FAD5FBDF1C5FD3D27A5E73BC4902A3E24
:106AB0002D0A7BBE600E81BE1913E2BD2E638CBE13
:106AC000BB461DBE8DCCBEBD8B36C4BCC31C4BBEED
:106AD0005D1F0EBEA370AEBD6AF1273D44BB613B96
:106AE0000A6217BD1D3F81BEC3D338BE85EF6EBE9F
:106AF00010701ABD00F610BF10D82D3D2339E6BD29
:106B000058001B3E7F98E9BC2DF96A3EFDA984BE62
:106B100076B801BECBBB51BEE705963D03D43ABE65
:106B200053F1D2BDF8B386BD1C8EEF3D110B0FBDE6
:106B30008ADC223D5952403D9D343FBE3FFFA13E7D
:106B4000A2EE85BEF7A54B3D0BA6B73E8B9213BBBD
:106B5000CE81803C2CD0CEBE6FFE08BD667DA5BE2A
:106B60005465EE3E5D11313E31B7BFBD4DB07A3E4A
:106B7000A69F2CBE6531473E7D1ACF3D9A5D35BE3E
:106B800020A897BE1862A73E4146D9B94D9306BECC
:106B9000CCB3F23E6B4F83BEC235D8BEB59CF23D3E
:106BA0009656513D20DFA13E2C60CBBDE305933EC0
:106BB0004911513EAC93EDBC062874BE1D85E03DE5
:106BC000199A1EBE8FDEC2BD4BC2133D477DD43D18
:106BD00014824FBD9A3A503EFC90743CDB33673EC2
:106BE000607C9F3E7B5BA8BE7DA13FBE10B447BDCD
:106BF0009E6E533DE8C0E4BD8B6C8F3E9C26323EBA
:106C00002A8919BDC5E6843E17A517BEED42023D8F
:106C1000445C8C3E52F446BE737375BE8F27063EAD
:106C2000BE9767BD56587FBE36040BBE28F7DE3DC3
:106C3000792E053EFEC73BBE4277BA3C58BDAA3D01
:106C4000879EB5BEF8EAE1BC8590ACBDBEEA73BED6
:106C50002EA6D0BC027BB13ED38628BE01990FBEC2
:106C60008A2EB73E0F1BD43D69A5B4BD5C6281BEC0
:106C7000840B1D3EE9D02EBF515850BE1E9A9D3C3C
:106C8000BD5D8F3E1FB08A3E237E88BE920C043FBE
:106C90001A4C00BEE21525BEE6F972BC63CC0BBEF1
:106CA000FACD683D705E84BE9F9056BE77288F3DBA
:106CB0004E819A3DCB6E89BE50FD02BD73DA9ABDFE
:106CC0000EBF0FBE3B648FBE0508B4BE89BAF3BCCD
:106CD000F593833E7E20EDBB8901B2BD0F6EEABC09
:106CE00042488D3E16844B3E4D8419BE7CB48D3A8D
:106CF0000338883DADA0A7BE91F0EBBDE869EEBDBD
:106D0000C7356A3DDDC302BFB3EE243E8C68433E07
:106D1000BDD396BE2CD7973AF76E13BE13485B3E91
:106D2000288C1CBE584369BEB8A52CBD0734CCBC0A
:106D3000F86CAABEDC471E3EB297D93ECB108B3E04
:106D400018887EBEB7229F3E636FD73D5CDFACBE26
:106D500073E7CCBE275656BD9656EDBDFD044CBE1E
:106D6000F3C7F6BD1DC9003F60146C3D9A58F0BDD5
:106D7000B0A5EF3C93AA933E411A143EBCAD19BE98
:106D8000F5D82A3E0F21093F3C624D3C264B58BEA8
:106D90004B13773DA260A5BED86414BF49DF423EC5
:106DA0003D8E8D3EECDABEBC39BA6C3EA2BFD13D01
:106DB0008BD9E4BD5A1D9D3D77895DBD1252A7BE9A
:106DC0000D8F27BEABE102BC06C864BE2826B5BD48
:106DD000C8B38FBE0C2090BE80AF4CBE620072BEA6
:106DE000D72D18BEE4ECE2BE26CA3D3D84801FBE0E
:106DF0001CAAD8BEB70041BE49B72D3E4D07E8BE1C
:106E00000DF3B7BD7AFE9CBC9F06BF3D547376BEA2
:106E10009B344D3E2F2B88BE065FB23DBE1474BE20
:106E2000E18208BD28630C3E2A5307BD8597A2BDA9
:106E30002FB85D3ECE827EBE7D47BCBD6F7D053DD9
:106E4000A6C306BE37FF04BEF55AF3BD4AE85DBED1
:106E5000CE27D93D05611E3E5A6192BE22F435BE51
:106E6000819FAD3E1E128B3E4501DC3DBCE1383EAC
:106E7000983EAEBE2EB587BEC1DAB53DADA3BEBE4F
:106E80008588CABE038005BF577D223D028BD03E58
:106E90003345C9BE76588A3D6412E1BC77285A3E14
:106EA0006DB52F3EB912763DBF6F8F3EC068A73ECD
:106EB00065F862BD0C21DC3BF72E6D3EFEAE2B3E2D
:106EC000F3061EBFC8A1B5BE37E4F13D349715BF28
:106ED000B60B303EBAAF06BD8636703E161E493E32
:106EE00035C718BF7C52A13E31CBE2BEDB1A873DCD
:106EF000280D4ABE69F2623E3152ED3DB6E5503E84
:106F0000345A123F7886883ED7BA63BECC74FEBD31
:106F1000FE6098BEED762F3E20AB583D7A3C5E3E3B
:106F20006F611CBE13BA05BE20FAAE3E7F26F33D4C
:106F3000CE578F3D75C3053E48B5EB3D29C7CBBD48
:106F400054580BBE74F4273E18C041BD198979BE50
:106F500058F160BEB24441BA64A86ABC3454BE3E23
:106F600071707BBC46BD193EA990FF3DE721563E9E
:106F70009A72DFBD64FC46BDD48A83BE314F09BE20
:106F80008712313E4B81853BB2F5CD3B940D0DBE52
:106F9000DC57153FC2FBD73DD429D33C14E54D3E09
:106FA00089ACA33D9815AFBE567B7CBD1D5E61BE0E
:106FB000B4447D3E8E70623E3514923EBA71F3BD8C
:106FC0006F3F93BE2834BD3D1BD757BE63A1B7BEEC
:106FD00072E605BE4B7CFEBE2AEAB7BDD286C73E2E
:106FE00058FCAB3D023993BD5EFC1EBF8B37713D33
:106FF0007644FEBB31CE02BFBCAE8D3D68F0D53EBF
:107000001C5FC53E02DD2F3E7C92383ECCEA66BD59
:1070100003E4443E7C2DD5BC76E9B7BD56D8063E88
:107020003BE381BE071E053ED0CB303E52A6BF3D9E
:1070300002316A3E8E79A03ECAB38ABEC45AD3BE1C
:10704000F4E17EBE6343AC3ED72CC4BEA8D5333E2C
:10705000FE68CDBC766FC4BD44C9C2BD2B669FBE61
:107060006B4ED83E9DC1613D82C8843C16A908BDC7
:10707000E1110BBEE291EEBD22D038BEA23485BE36
:107080006C04F4BEB63FF43EC1F96FBD0FEA24BEF6
:107090004887023DFE1692BB1CD517BCB34DB4BD4C
:1070A0008B1E0F3F9BB3D1BE0B0837BD6111E9BDED
:1070B0001AF9F63DC356CFBE5C397FBE9D2F4ABE3E
:1070C000069E5A3B14351FBEB5B1B73D09B90A3EFD
:1070D00070DB113D094670BE8130023E6FC435BE83
:1070E0003454923E20AEF23D3D16853D8EC221BF06
:1070F0005BBE193E2F5D70BEA0BABCBE1E5E3BBE1D
:10710000CB429F3C69BE6FBEC68C493EA1F29A3EFF
:1071100096AF0DBE301B233EB5B5333E2357963E8A
:1071200072BAA8BE1588D23D632F01BE18ACE6BE68
:10713000DFACC5BD8E0230BEFD9C0CBD514AE0BD2A
:10714000F9B7F33CEF4B14BE569027BE40023A3ECF
:10715000C464253E6182A63CE9AF8CBC55C12BBE00
:107160002091C83D4E8630BD5EFD62BCEACAAD3C92
:1071700050C2153E77C2BA3C89C32DBDAF193FBE80
:107180006FD5D3BDB9EEB7BD27154B3E2F74073C65
:1071900011C5C8BE2438323BBF8EA8BDA825693EA4
:1071A000FAFE68BEA37A953D2E9FE13D4FC32DBEEA
:1071B000DEAE69BE83BA283E49D8AFBB4EB91D3E8C
:1071C00048B8ACBE783E3DBFEFE16A3D298E713EC6
:1071D000B604B2BE6366FD3E88A8F03D5F028D3DF9
:1071E0007AACA23EDCCE1A3EFE57C13E4A1889BE9A
:1071F00098262F3EC95F673CFB2F1ABECB2289BE63
:1072000005CE2FBEB01039BE8232903E1A7AA23E11
:10721000C383ADBEBBA2963EFDC7533E872548BA89
:1072200083B982BE8F3DF63D409B6CBED84050BEB8
:1072300069EB85BE426129BE9AA3B5BE873A2ABBD7
:107240002B22223B989400BFB8035EBE2E523A3EDA
:10725000A1396F3E8A2A27BE4C36363D49D4953E29
:1072600003D88C3E4ACE853E3E3CBD3DD817E43D1A
:107270004EB044BE7D8602BEF58B8FBED8F086BD73
:10728000A76EDBBE7F121DBF70AD5D3E2B02453E7B
:107290008A8522BF17BBEBBC8FE0B3BE456A24BE14
:1072A0005EC483BECD0FF8BD0997363E7F67A73E0B
:1072B000A6941BBD00E70BBE602375BD3F38B0BE72
:1072C00085B4D1BD76C03F3DCD387BBC4CDAE93CBE
:1072D000F118A43D314381BE11858ABEDD30103DD9
:1072E0002C7DD8BCD2EF0E3EB10C9FBE93F724BDCF
:1072F000625757BE99D6A6BE2A09ADBE7D58053E37
:107300004F1D683E278968BD60D49FBCD090A93DC1
:10731000E4E62DBE254650BE03481ABE1E8434BE88
:10732000E39C363D8F9BB0BEF5F887BE6EBB023E38
:10733000CAF7203E3EB4FFFF04000000004B0000EF
:107340001B6B4BBE606890BE431CEDBD8AC6933E6E
:107350008EE5793DD5477A3F64949BBE14EAC6BD5D
:10736000668014BD0063873CCC1B03BD6EC2263F04
:10737000F803B9BE3CC4183D51654FBDEBCBA6BD6B
:107380001B7DDA3C2716A13E8B2302BF237610BD5E
:1073900083F86C3D0029333EFFCE5BBE63550D3F45
:1073A000A3F7C6BE7A82503E961DF23D5E296C3E22
:1073B00024E275BE41D52E3F40DB60BE23BDF7BD44
:1073C0000CC5803DD5D9103E8CCA0CBF81421D3FF3
:1073D0001CC3AABE3DB927BEDC09053D840C2EBEE8
:1073E0000DAB27BFC08D153F22C9A0BE064E3CBDC8
:1073F0006E1E05BC0F4F403E9B2631BFFC2FE03E6A
:1074000028C46CBD48BD30BD0119C43DE2B4753E11
:1074100063801FBFE3700FBEE91849BEBF11813AF8
:107420008E3ED03DB27AB03E8E1501BFE10462BB04
:107430003581FDBC5DC4CBBD751CCA3D1132B83E63
:107440005BC7EFBE02DFF6BC188E343CC7DD49BD1A
:10745000F708D53D2CEBB63E0343F2BE7551C53E51
:107460004763C13C707596BDB30A3C3E71E8053E6A
:10747000738DD5BE7408A63E5071203E5996423E8B
:10748000C3FD2E3EBD5F933ED466B2BE0648A03E0D
:107490006201083E72FDE23D1B42E9BBC43AF13D88
:1074A000DFE30EBFB238493E83696B3E5579143E27
:1074B00024CE30BD737D42BE679A1FBF1608543D6F
:1074C00030A7873E05E91C3EA50C1CBE464264BEA3
:1074D00091CA3BBF5D3A823E247D9D3E7F88663ED9
:1074E00084BE25BE6F4419BE4C68EFBE92D5AF3E38
:1074F0002894B23E58EC88BC7EDA463D38993DBEB1
:10750000F868E1BEFFF4783E00DE533E8108E23BBE
:10751000EE5F78BE1674443DEC2A52BEE141443E13
:10752000694B963E59054F3D29D00EBE51FCD93EC0
:10753000336D38BEA93FF53D4EDD9F3EE721763DD8
:1075400074161CBEB264223F5254A8BEAA08B23EB2
:1075500002994E3E6EAF2D3EB06833BEC47D993F5A
:10756000FE9E70BEAE08FA3ED4244B3E34884B3E9D
:107570008B1200BE5206903F2C947D3E00EC3E3FA5
:10758000E9509A3EEC1E193F43F87ABD773DDE3F45
:10759000AA879FBD274C0740CE6F2ABE9D4AB4BC28
:1075A000D8B7C23E97FD8A3E9383A93C9EE6763FBC
:1075B00003C684BE6FC5CABC0400853E0C5AD6BC47
:1075C000323D943E04B0513F9F2CA4BE20125BBDBF
:1075D0002C63823E66393B3B7032B73EFEA33F3F91
:1075E00089CCFABE87F652BD1E54AB3EA37AACBE20
:1075F000D0F0DC3ED03D493FEF0A01BFAAF9F5BC0F
:107600005AC3A83EB241C5BE1718F73E799C113F38
:10761000AB560ABF0C2D10BE9C22823EB49FA6BE64
:1076200075700B3F7F8CD23E987C29BF7B7AF4BD6E
:107630003EA7123EC593C3BE3DACDE3E6390683E9E
:107640007044FBBEEE666EBDFC57283E67AFA2BE1F
:1076500054B2A73E9B3E7F3E6E18FEBE4872E7BD09
:10766000575B173E033BAD3D8EDEE43ECFF6913EC9
:107670007825BEBE91D680BED22A18BE3F87053E71
:10768000E94D423ED12FFFBD2BA6B9BDA7BDA3BC7E
:107690000F7F83BE20B5413E284C903D8C2B80BE91
:1076A00070F7C6BBDE833ABEEFD89D3D6984AC3C23
:1076B00011AEDABC858D8EBEBA50DB3EA93ECCBD84
:1076C0009C04D3BE17B725BE899684BD4B47633D46
:1076D000B352C03ED5B5953E2DAA093DA03CEFBCA6
:1076E0004CC390BED95D4A3EBB01343E3F6A3A3E30
:1076F0007430473A3A272EBE7CDF7EBE20BAEE3D7C
:107700001733C63D66298A3E3939043DCE3EF1BD68
:107710000D59C8BE03A7DE3D308C893E8471453EBD
:107720009807593EE6096FBEB8E8B2BE927F42BEE6
:10773000498D5EBC895DB73E7B6E333E72C486BEAA
:107740001F1BCEBEF780B3BE4B10C4BE50A3043F78
:10775000F581863EBEC81EBE1579E2BDC10764BE76
:1077600044E202BEDAC74A3E09CD9C3C1F7DCE3CB6
:10777000DDD819BEFDAF72BD4331423EC1E0473E88
:107780000A57A23EF069F3BB62F47CBD9DB7C53BCE
:107790008484773ECDF8443E15961F3AC6E80ABE6B
:1077A00008D5A2BE06AC583DCF64FB3E02428D3EDA
:1077B00072633F3E706AB2BD8ED8CABDC5352CBE5D
:1077C000E335993EF7549B3ED2AE34BD9DDD8DBE70
:1077D00012418BBD59F58BBE60DFB33E6893063F07
:1077E0003DF1453E6F78B3BEE99E9CBE1982E23DF5
:1077F0006AD2FCBEE36CAD3E5C6DC9BE3ADDF1BE43
:1078000068EF5CBED57A403FD42C06BEEFD7993ED8
:10781000D8DD1CBEF7A07FBE4343A8BE21201D3F7C
:10782000A19E29BEDD46B83E6F4E77BE2B11D7BE56
:10783000906E8FBE28BC043F3469B9BEAB8E133E38
:1078400009BF8CBE073D95BD53CD43BE0B7F233F83
:10785000C2DE15BE4D78EE3DD45C33BE23B6BEBE4F
:107860003F8BB3BEB7FCA03EB11F06BE356B733E67
:10787000357350BE582E07BE3A16E1BD70BC7D3D33
:10788000661122BECADE223E0AC2D0BDD82272BE16
:10789000F1C2373D3422443E81EB47BE3447C73DF9
:1078A000C96301BE433E14BECF6679BE7671D53D35
:1078B000F8FCACBE5887A93D11D082BD56B2C8BEF7
:1078C00019488EBE6EA0093E0B9D7EBE84614F3D61
:1078D000DB42CFBD032AB0BE030B79BD2FBC4C3EAB
:1078E000975EECBD49678D3DA22816BE20938DBEE4
:1078F0002D80C9BEA140B73E502B10BE1079E83D87
:10790000195659BEDDC507BF7D2B94BE0159E83E0F
:10791000D8544BBEE41E87BD2979B8BD16A854BE05
:10792000F51ADCBED0777E3E7702933B45DAA03D68
:10793000EC51ECBDD9D9FBBEFE64A0BE0C1A3D3E95
:107940000A91C13DD833C9BD56A9ABBD95EEADBEB8
:107950005DB1FDBE7A22BC3ED38CB23DF3C7243D5F
:1079600056A105BEDF0A41BEA851CABE5D6DBE3E2E
:10797000478A9A3D88EB3DBE2AD3A7BCF1E78EBD6E
:10798000369700BFCD2333BC4B24863DC53E863D94
:1079900068A33B3DC01909BD255053BEF51C4A3EA6
:1079A000F8BD8C3D2ED2BA3D6EFF29BD6F9F8F3C36
:1079B000E96089BEBA38013E00F9F23DF1755E3DDD
:1079C0002429283A07B93A3DF8478ABD412EAAB979
:1079D000AAE5833EC7DECE3B0E0E223C065CAF3DE1
:1079E000C6B5E7BDF3CC43BD125E493E166A663D9F
:1079F0002291E33D36C2BFBECD5D7CBE183D283D21
:107A00007E25793E38E537BCA874633DF8915FBFA9
:107A1000AC7FEFBCC827213E13B56D3CC4ABE2BDC3
:107A2000BE12E53C845BC7BF217602BCFF8C773E6B
:107A3000F174FF3D99CD17BF0188ED3D1DF626C0BD
:107A4000AED9AEBE36DA993E08518BBB0BA473BFDC
:107A5000CA23B73EE67F2EBE0D269F3D4109B13DAC
:107A6000DC96BCBD886344BF5BA52C3E0803BE3DCD
:107A700037B07B3D7C30A0BE372501BE0AFF45BF35
:107A80002B7B5B3D5E92753EEBA5043ED2A7C2BB4D
:107A90009A36C6BD924034BF379A91BBFEA6B23E1D
:107AA0006390A73C2BFC90BC4138F5BC03B427BFC6
:107AB000102010BEBAD87E3D5E24DC3DD3F6193EC0
:107AC00077D40FBE277801BF0EF09BBD74DD403E1A
:107AD000584ACE3DCBB21BBDEE9FACBDE326EEBEF9
:107AE000C2644EBEEC69853E1E4C87BB107C6B3E6B
:107AF000E1B43DBD9EDADDBE842D2CBEDD000C3F21
:107B0000090DFEBDAD74C23DB7BE77BEA39515BFCE
:107B10006E4148BEDF50453F694CD8BCF7AC7D3E56
:107B20008A5F8FBE59CF04BFD0E591BEA591683F53
:107B3000880328BE564E213DE4C5A0BD55E7A3BE2F
:107B40003C3904BE73504B3F3A2AD1BDD633863EF2
:107B500041CB44BE96C7E2BE441030BE0821303F40
:107B6000F396FFBDBBACD23D05E7B4BEFBB2D0BEC1
:107B7000710147BEF57B4E3F1E79023E426177BDE3
:107B800091A254BE3FDABFBEE744A7BE30A83B3F38
:107B900010C91CBD6089593E532634BE7A5BD4BEE1
:107BA000F42EB8BE4387503F93AEEDBD6CF73CBE9C
:107BB000A52D95BDCACAC9BE5D16B7BEFDED283F4D
:107BC0009D5467BE683C91BE4306E1BD5EB6CEBE25
:107BD0008898E7BE7D4F343F899AC1BD91E141BE8F
:107BE0000FFDA1BED872BFBEF1F937BEB4CAD73EF1
:107BF000146824BDCD97A0BE58B9983B647AE0BE06
:107C0000846AFEBD729D923E0F1B983D495B803D8C
:107C100098EFD0BDF08FCFBEAB5711BE9CB31A3FCB
:107C200063B116BD82998C3EE11736BE7952E6BE2D
:107C30005ED182BC55A3D83E0F15083D9073A23E7D
:107C4000E59B2CBD967670BE638FC13C402DF33E04
:107C500031EB32BD6944193ED433033E19F093BE73
:107C6000B9CED23CB156013F57511E3E453F693D0A
:107C7000BFAD733D712B02BF30E09DBD08B5483FDD
:107C800029862A3D26A49D3D668B043DEC4AA4BE70
:107C90002E91153E92EEA93FF05FD7BDFE0FE43D59
:107CA00057E1883A5C7D16BE4D504E3EDCAC103E2E
:107CB000348FA4BD1B8024BE5AFDBE3DC1E309BE66
:107CC00049D0CF3C3A7EE83B54E1D1BE86AF59BFA4
:107CD0007CEA823E8C7917BB87B9F5BBAFD708BE6B
:107CE00032D53CBE9B5D05BFB208C13D3D1EFABD0D
:107CF000EB8C273D29CCBABDDCE175BC95DD11BF0D
:107D0000373D7B3E4FFE5E3D2F3F81BE58A1CF3DAC
:107D1000880513BE366C19BF5CCA1C3E188F4C3EDA
:107D2000896574BDDCAC44BCBAD4E93D853EF6BE81
:107D300009E5B53CD69BBD3D71F817BEEE344DBE8E
:107D4000BD90EFBD5821CCBE02BABB3D39BCC73D8A
:107D500098BC2CBE3ABDD2BE82985CBE163294BD91
:107D600020A1143E9F692F3D127545BE71D2F2BE0F
:107D70001A2EE13DC606B5BD8DEB003EC4A3A9BDDC
:107D800047951DBE7FAFF7BE57ACCD3D3EF58DBECE
:107D900048C4DF3D2A026DBE9EA38ABD763EC7BEA3
:107DA000C0137DBE76412C3E9F0D013E9FA62E3D09
:107DB000D683BF3D8F41D3BE9C99C5BE270E853D5E
:107DC0005A94DCBDBD291D3EA2CCB83E2401563DCF
:107DD000F68B75BEA1F695BE11CE44BEF7EB573EAD
:107DE00026B69A3DFA155A3DEE18143E24A4FDBE5F
:107DF000B3B484BEA8A55D3E82E1DE3BB29D843E65
:107E00001904593E122AB6BD402D91BE4C10553A68
:107E1000FCA692BE41C4B43E16E8893D26EA9EBD4A
:107E200037D621BE820DEA3D853561BDA2F48E3E76
:107E30009112E2BD5C3019BFC0548DBE5A52BB3D99
:107E4000D98C64BE6DA2813DEF3B9ABE98F479BE99
:107E50006E9E92BE725FB83DDAD170BE79CFF33EAE
:107E6000238E08BEFA2DA43C477699BEF2641F3ECD
:107E700045A988BD14DBE53E00E3EEBD538F133EFC
:107E80004CB4D2BE61A9113E1B37383EC13CB33E53
:107E900020AE6BBE0545383EEF1F24BE051C543E88
:107EA000D6B78B3E037B403FCED441BEB966833EFE
:107EB000AADC8D3DDDD5473E3E39993EBB9E1E3F37
:107EC0003295BFBD1BAFEBBDCC1D853E8D8EC23D37
:107ED0001FB5903E2117903FAF145C3E44BF3DBE9E
:107EE0001A4FA0BBF1C4253EEA1B133FEBABB93FD1
:107EF0004844083ED7F1FB3E3D4BF5BD9CD90A3EB8
:107F0000FFCD12BE70EDF2BDF2DC19BFC6F749BD60
:107F100022E54ABC6E4A503D4F55A7BCB12633BE40
:107F2000ABF885BEA4ED413EAF1590BA3B00533C83
:107F3000C72518BE582CA2BD7E776EBE8E13833D1A
:107F4000F24D6F3D6E14BEBC44C985BC0CD5C8BE95
:107F500097A3DB3D2C59AA3DACC6AEBC1866B5BD97
:107F6000040818BE0BC803BD2C9A81BE371112BE7F
:107F70007A2AF73CC8D7993DBD2C31BEF5EC5F3E5F
:107F800036A88D3DA539153EBE02083E9A6B4ABD06
:107F9000321C0FBE93D9913E0CC7803D3BDF823E21
:107FA00051E6073E6F31C73D3A6A9FBD2176AB3E31
:107FB000A20F9CBD4E90333EDD64133ED27D8D3DBD
:107FC000D0EAB6BD1052BE3E60E5DEBDB65AADBDCC
:107FD0005D8A483E169F96BD0D61FD3AE237253E0B
:107FE000E9038E3D305130BE86E0773EB39E413D81
:107FF000EBAE663D7016BB3EC98D123EF8C79BBE08
:10800000DFA85CBDD2F0AEBDFFE3803BF734283E75
:10801000B7F8BA3E06277BBD263259BD089DE03D24
:108020009607673DCCEF7B3E3E2DAC3E171FD9BD7A
:10803000730C4BBD7FF122BE71EBF7BD4CA7603EC8
:108040002CB2683EF2676ABEBD3B503D53B8EDBCF2
:108050004601C4BD884BCA3EA4388EBD12DBA93B85
:1080600076C4BEBD21DFDCBD34384B3DD681343E05
:108070002934333ED3FF603EC6E273BD771C18BD82
:10808000EB8D6B3D6A2D21BD39668D3DC59B6C3EE8
:1080900076CE173D55780CBD3336973D26F8133D07
:1080A0008F150E3E20E0993EFF09C4BD4A16063BDF
:1080B0001CA1D23D385315BFAAB8A03E03D6A43D9B
:1080C0001D9D6F3DDF73F83DAE3DF63D1618F7BEC2
:1080D000D2AA113E46F92FBEE3BA09BE67B01E3DD3
:1080E0008F304E3D1501D5BE4B8510BEEA878ABE46
:1080F0009AE99A3D685A81BD79257E3D3F5E68BF09
:108100007E6C42BEAB36CABEABF850BD367770BC93
:1081100002B119BC4453A6BFCBB492BEDB3F0BBD2A
:10812000CE38B0BD4941A9BCF6CCCB3C62D9E2BF48
:10813000270FBFBEA7C6E7BD52C761BD09DD053E1B
:10814000A16ADE3CA28041C0430AF3BEEDDC2EBF33
:1081500091F5EEBE9659A33D3595583E083A873EB7
:1081600041096D3D798DE33ED78170BE11E7763DC3
:10817000A5D8773E70B1573EF051AA3C15B19E3E4E
:1081800053BD28BF6CDD513E92FB2D3E8AFD803DE4
:108190003ADC093E03815D3EE5BD29BFB4EB833E79
:1081A0008C04B33E07A1A2BDBE3D273EF7F5823E3B
:1081B000F3D7BBBE8D35FB3DDF5B613E0CADA13D12
:1081C0005562E3BDFC12813EE0B7D6BE29982C3E35
:1081D00030B6433E5B99D5BC4A2CCA3CFA6937BDE0
:1081E000742EDEBEA54A283EC50F763E3664D7BD46
:1081F000311B8EBE51537BBC733903BFD727153E4D
:108200002E6E79BD08620CBE8F60C5BE99CD17BEBB
:10821000308ABFBEF708573E338AE83D9C162ABE17
:108220001D0501BF0FC0C7BE72EC01BF65D7813EFF
:1082300073A84E3EE02CA2BEF7CC0CBF99353BBED6
:108240006C8E93BED4C0CC3DA013E63D4DD743BE4B
:108250007F4AF7BEFAECB4BEB7E586BE262D2FBD29
:1082600043AA3C3EF42814BE692A38BFC14775BEF4
:10827000ABA0DCBE3D2D42BDA23E433EC4C21ABFF0
:10828000809142BF5DFEC7BEC4CA03BDA872C93D8E
:1082900059DF183E733309BF1D5E3BBF699280BE34
:1082A000407A78BE63BFA63D3927853D9D143CBF0B
:1082B000DD5C3BBFD151E3BEAADC56BEB764613D75
:1082C00010A6163E72F00FBF7E5406BFE262B2BE29
:1082D000FFC792BECA3FBCBC0DF9453ECD0CD5BE12
:1082E00030571CBF8CFB16BE58BBF53DDE33C73D77
:1082F0005BF5A73E810D1CBF12FB08BF76492FBE60
:10830000672096BBF7EE883DFA18733EA98961BED7
:1083100045C159BFE62EECBD6729E3BD20BA9DBD1E
:10832000CD12BB3ED89359BEC4AA4EBF16DED6BEF0
:108330008620043D72D2AA3D31F96B3ED81342BE6D
:10834000F4B51DBFCF2BD3BE0D20B43CEDF26B3D79
:10835000F928A73E7A34C0BD740C31BFBC93EEBE81
:108360002FFEE33DA87812BEF0F8223E78E293BEDD
:108370007BEC2CBF65A6D9BE993489BC4574E8BD99
:10838000C73C193E1CFCBCBDD10073BFC31D57BF09
:10839000EA0D9ABD7F3366BE9F63933D9CF0A9BEF4
:1083A000929D41BF82A2AEBFDCFEDF3C6AAB233FA1
:1083B000EC7D143FF6535FBF7933613FB3F9693EFB
:1083C000D92D123EB6E8183F63F4C03E044010BFFA
:1083D000B6A7853FBA357A3DCAC07A3A1D931A3F8F
:1083E0003A77EE3D2BD84ABE0CC0193F477C8DBD75
:1083F0009F963A3E02C2323EE69D973C9CEF09BEF4
:1084000034A61B3F369B01BD958056BC1416283BF5
:10841000A4BEC33D28725DBEF8BD803E637CF1BD45
:108420005D9D813E534FA6BD5BA6563E34B778BDD9
:10843000080FC83EB8A663BDAA78253EC59132BED6
:108440005981293D3249633E4948963EC1EE8BBE73
:10845000ED508E3B4F3790BE6656973D69714B3E4F
:10846000754E783E59E7823D9D1DE4BD963365BE4D
:1084700072BDFDBD21AA853E28792E3E4F14713E66
:10848000EF578CBE8A0D63BE5BEA4EBE653CC33EB1
:10849000F111473EB211FD3C8ADB43BE546D54BE20
:1084A000F16216BE2225323E8F8BB93D7816903E82
:1084B00050A2F2BE2FA359BE04147DBEE5E5CE3E08
:1084C000B5C4683E8EFA893E91510EBF114B4DBE28
:1084D000CF1C72BE50600B3FF77F533E39A6E63E7D
:1084E000B09D2DBF0EAD9ABDCBA134BEE7E0CE3E10
:1084F0008AFDA13B274D153FFA66B1BE574B90BD93
:1085000067F094BE14C5E03E733E883DA96D313FCF
:10851000255306BFD33C7C3E246F5DBEC9C5DA3E01
:10852000924B7ABEAFF7013E283DD7BE61251D3E76
:10853000874606BEB51DB53E6B0F9CBD9FCBC33CA9
:108540008DA8E3BE92FC943E7EE550BE1C7A023FAD
:108550009291373EF7ED42BE8116FBBE7B36993EC7
:1085600087C8A1BE910DFA3D434E4C3E4B88E5BEF7
:108570003E967CBEDF5B163F4620A6BE3B888EBB88
:108580004BD99D3E69AC29BD450418BEE12AC83EC1
:10859000847D633C253D513EB303F93EA0DF40BEE0
:1085A000DF2291BD333FCF3EB694BF3D11257D3EC6
:1085B000CB7F713D84C911BEE754C6BE1BEBF93DAC
:1085C00008D2833EA83C17BE7C9C00BD7B02BEBE89
:1085D000776394BE677639BE094020BE2F53C2BD73
:1085E000BC530BBE209297BE7AC6E7BE9A3C61BED2
:1085F00081DD24BEEB2285BE6747CBBE9F87CDBE03
:1086000014C5EDBEECD8A3BD7108733CD9C2903F30
:10861000540BE6BED88F89BE003E30BE0DE8043E46
:1086200077F644BEB3CAA53FBABB9EBE6301313ED6
:1086300082457C3BE9AE093EA43326BE1AEF313FAA
:108640004B3CD6BE70279A3D65CB0CBFB007853E2C
:10865000DA5E87BD6C452C3FE944DBBE8EC65D3ECD
:10866000603003BE04384F3E6BCA6C3D9613EE3E3D
:10867000D9DC2DBECC00C0BCE77E473D835BE43D2A
:10868000B4E7B63DEBE89C3E4D0729BD8223DC3CB8
:10869000A55A2F3E488B893E5C319C3EEB0C763EC2
:1086A00078EC413C1815D53E3F32B53D8865BF3E5C
:1086B00088831E3FFD91543ECCEB243D00EAC53E2D
:1086C000F001D3BDFAB3C13DC559203FDC2EA83E11
:1086D000E1F1F83D8446923E947D7A3EBDDE8C3ECB
:1086E00037F1443F8F9A753E78E9B7BD9A6A643E88
:1086F000C297AA3DEB20A63E1AAC063F380174BDD6
:10870000E02A4EBE409F8F3D3D57193D32517D3D81
:108710001AC9DB3E3B3E56BE684822BE0E9C3BBAA1
:10872000B66624BDC451D63D4F1DD53E71A3A8BE2B
:108730001C0C54BCF2CF9EBEC1EE98BE653BD93C2A
:10874000EFB53C3E2830C7BE8F4109BE3837BCBEAE
:1087500088F911BEFF86103EF28B503E7A4505BF68
:10876000CCC77ABE9110F8BB07F50EBE4DFE7B3E1E
:108770003A282F3EF35ED6BE872625BD44D9763EE5
:10878000DD69D5BD3E70833C1A422B3DFF4FC3BE11
:10879000F1F260BDA2FEA53E5F3EDFBD859FBBBD81
:1087A000BC90E9BDE80919BED92921BE9E2E973E8D
:1087B0001B50E9BEAB3F13BECA73A3BD912380BE5D
:1087C000E42F243E585D1D3EE21A91BD17248EBE53
:1087D0000B7DFFBD5E2B81BD0BD4D6BC4D25BF3DAF
:1087E0000D5479BEA1C580BE33653A3EF89347BEAD
:1087F00030142CBE066C3EBE75DA1DBE44E447BE86
:10880000860F133EE64C7DBEC985F1BED176F9BE1A
:10881000C63C96BC2ECC44BE1FA9B73DC94D143EE4
:10882000EAA843BE42136CBF96ED243E11119ABCD8
:10883000D6F51FBDCA7C223DFCA8F7BE3BE7FABEB9
:108840008ADB5D3E4D5219BE62EACD3C8AF8CA3DD4
:108850002B42A8BE421B5FBFAA83F53CA7032A3B5D
:108860006D03183F7E3A0F3F8643A23E046A4BBE1B
:1088700070D926BDCEB2A9BDA5D1D23E8672A43E86
:10888000878A833B2037B93D84385EBEF6F406BE46
:10889000A56F803E0BEB373EB663E33D398277BE72
:1088A000370D19BF2EA583BDCD7A443D1E14A8BE39
:1088B000BDE09F3DB3BEA0BE45BC03BFCBCC73BDE6
:1088C000F729ACBD69E1CCBEFAB24D3EC70EDCBEA5
:1088D000182A17BE39A8D93DA783A5BD5CA297BEAB
:1088E000EDD4A83E35008CBE523BB7BDF8E59FBD28
:1088F000AC43CDBD91483FBE6AB3A23DE48787BE7D
:108900004EA6A6BCD5401C3CB057383EBE2858BE2B
:10891000FC4F813E51F84B3D9EA09BBEC79769BD61
:1089200090B3103EF9DD88BE660B6C3EB019ABBE4D
:108930001DF5C4BEAF3827BE2911CA3DCD0ECBBE32
:10894000BD470F3EAA57F8BDA8B9C0BEBB357B3D99
:10895000D500063E570804BF22C0AA3E237FA6BE0C
:1089600020491EBF5EEEE43CC703193EDF5CFABE41
:108970005977A83E685982BE35D5B1BE75EFBCBCEB
:10898000E488883D6732CEBEDA30953E28ECABBE37
:108990004AED36BE1143A53DBD26483C52EC2EBEE5
:1089A000F06D7E3E3E5FDABE5B7F60BDD73996BC20
:1089B000D5360E3E6D13E7BE6EB3013E1CE3F0BE2E
:1089C000FC6BAE3BBFFC15BE5817E03C4A13AFBE74
:1089D000D032313D626E76BE3A91093E4DDC0F3E9B
:1089E000E1E3843D75180BBF5E62B2BDBD18A4BE45
:1089F000AFC23B3DB3B3B7BDD7AC873E8ED18ABEC5
:108A00004FC76CBD4EEDC8BE08822B3DF7C7903DE9
:108A100086233F3B9981C4BE916580BE5D54EB3D8A
:108A20003C8B903DF0B6C13D1922663E9ABE19BFFF
:108A300021BB80BEAD51D03C43FE963EDBBBCC3D5E
:108A40009E63313E54B807BF302C16BF2078363EA7
:108A5000AE73EFBD8C6B0CBE3ED73B3E9FD451BF77
:108A60001A5655BFF16A65BDE49346BE393822BE39
:108A7000A6FA33BB0EA249BF28471DBFA11613BEDD
:108A800049468BBDABBD5EBEA997C23E29132FBF21
:108A9000FCFB1BBF860CD9BE1531EEBD446B4DBD32
:108AA00043256E3D197BDF3D579D2DBF12801EBFB4
:108AB000F942A0BBD9E204BD10DF9E3E4A802FBD23
:108AC00014B49EBE90B84B3D65A27F3EAC02DB3D28
:108AD0008D81353EC9D9A0BD3FB87ABE445F1F3EE7
:108AE000AF22323E7C0E483E52AAC43EBE76DD3CEA
:108AF000BA0939BEF7FCE6BC7553A73E44CDB33C7A
:108B00006CDC953EDB1725BD61BC36BE035F3B3E8A
:108B1000FA765B3E067DFEBCF722BC3E990588BE18
:108B2000881483BEA4D18D3DF941043E9025B73D04
:108B30000E32753E14C49EBB3A8547BE318B823ED1
:108B40006EA9A93E11A6F5BDF42272BDFE65A9BEAF
:108B50006D31F6BD544D0E3ED173BB3E1DE2983CC7
:108B6000816FCABDCCC7A7BE75A32E3E407C98BD01
:108B70005201C03E2D0129BD2791383DC36775BD07
:108B8000130BF63D994061BECA45043EA497D23C02
:108B90004926153D58CC74BEAB368A3C14A733BE6B
:108BA00020A482BE6F4389BD485333BECA6A13BE38
:108BB00020F9B73D79F486BE2ECBE0BE8ECE22BD25
:108BC0001642E03D3A5A5DBE15355B3ED129DBBE0B
:108BD0005C5186BEDCB8293D8B62AE3E634CD4BD91
:108BE000B071363E9B398DBE9FCCB53DF36A0EBD4C
:108BF000A8CF0D3ECF0090BDBC77D63EA2B6EDBE4D
:108C000099F460BE86645B3EE60D143D66B8123D85
:108C1000D96CD73EC53321BE80508FBEDC67BB3DCB
:108C20008A40C13D8845153BA432103E700EC6BD3A
:108C3000F3DA99BE1CDC393EF6DB41BED36746BE93
:108C400008C5C33E6E43C7BB63DBBCBE707F743DCB
:108C50005E4611BD60B8ABBD8A3E853E31958E3D06
:108C600096BF64BED47A793E1CD093BDBE6E443E9E
:108C7000C47AF1BD42285FBE96900EBEB2B674BDF6
:108C80006B4FE6BDCB6080BDA73F2D3E1CEA85BD86
:108C90006EEF31BDB4BD043FFC5BEDBDA3AD843EC2
:108CA000C05F9E3E332A9A3E40B63DBE1E99AB3E03
:108CB000F1F51EBEE95BAF3ED446C8BD9588A23E25
:108CC0009FFC103D367EF33E9A719BBE9DB2143FD1
:108CD000CCD72CBDEC4ECB3E5908E73D69E5233F90
:108CE0006A898BBE11EA0A3FBD6ED43DB92BF63EB0
:108CF0002820013D941DE13E70B35EBE78B1DB3E9D
:108D000087438838693DA13E0232C33E81CC053F8E
:108D10004F5B17BE64632CBE10AA8B3DCBA4E2BE92
:108D20009A40C53ED806053FF1BD273E4E7506BDAB
:108D300013F890BD0FDE10BF0B3FC13E4ABADD3EB7
:108D40002A25703EE8A7C2BD7008513E4F0CFBBEFD
:108D5000FBA56A3E9C11E33E3D33423DF9AFB5BEF3
:108D60009E57A43EA58409BF6846AF3E94C69E3E6A
:108D700094B8813DCBCCA9BEB3125B3EBE7088BE19
:108D80002359613E91FFE43EA2DA3C3E2C49DFBE0E
:108D9000EAA27E3EAFA197BE585A383EE1A18D3E71
:108DA000FFF0AC3EF0C43EBF0FDDB53EC796D2BD6E
:108DB0002D35063E4225D13E9AC90F3D313D47BF74
:108DC000420FFF3E185FC5BD34ECE0BC63A91F3FF6
:108DD000B8CBF93D3EFA31BF0073783E7B095CBEEB
:108DE000A21BCF3E96F7C23EC23EE03DABC6C7BE19
:108DF000E2A4323EB54AB6BDD44F003E90DBDD3D25
:108E0000D62C3A3EAB54CBBE7B01193E02D23ABEC1
:108E100037A4EC3A5AFEC3B9E756DF3DB34B00BF67
:108E2000A93E253EFE709E3D0B625DBD2241953DF3
:108E30004B3A1CBED82ABFBE7E64AEBC461532BEBD
:108E4000DBCA8CBE07A04ABD8E42673C3F445DBE74
:108E50008AC0CDBD901A42BD9C5A013E0A2C10BE5C
:108E60007D2001BEE92C40BEA8D0843E6380F9BDC0
:108E7000A013493E54A78EBD24DDF0BD39F1CE3D8F
:108E8000BE73313E3499813D72D2913E5F8040BEC7
:108E900021C611BEF011273E6E02A23E58EB103FD4
:108EA0001A7A3F3CA8DD87BDB07636BEC53FD83EB6
:108EB0003987973E914F083F6AC4E3BC4DAE5EBE12
:108EC000758116BD6C22893E244E913EFEAE983EC1
:108ED0009B6A3A3E4C3B2BBE771A18BE50BE653E8D
:108EE00043FBB13E4C967B3E4E82973D6E96B8BD9D
:108EF0007449573E67EA0D3F746FAD3E8D3D913E1C
:108F000022EBBF3DB26858BE00F6E9BC5741CE3EE9
:108F10004507803EB0608B3E236B223C5CD922BE6D
:108F200027F9F8BD180FA83EC80D913E0253893E9F
:108F30006901C8BDAAB36DBE16FCCCBDC6692BBE07
:108F4000B3D6933E125BC83ECB6D29BE3947B0BE47
:108F50001EFCBBBBA6B3B4BD60551C3EC340323F34
:108F6000E572C5BD5596803E3481213E197B463E53
:108F7000C7DF0ABFC36A53BF0B887B3D8DE99A3CAC
:108F8000FC168ABBC1AAFA3C163E16BF420C0CBFA7
:108F90009A6F4B3E3F3638BDC89621BE33A869BD97
:108FA0007C0D0FBF52A195BE33872C3E7282093EC5
:108FB000CA1C44BE52C284BECBAA07BF945B06BF84
:108FC0002B23DBBD8A27BB3D9C89503D36FA67BC0D
:108FD00075C104BF728162BE72E9EC3D02EE7E3D56
:108FE000216123BDE3927FBE5710EEBE3EFD08BF58
:108FF0007535413E764B14BDB0E7483CF1AD3A3D86
:1090000059BDFABE708C1CBF8594D8BCA140B63B3C
:10901000FBCE683D011034BEC26B5BBE68A8E8BEE3
:10902000EE22C6BD4E12733D371A6BBEBF4824BE3A
:1090300024A1BBBEE9B7B8BEB7167CBD4B809A3D34
:1090400098B5F73DCF0C9ABBB61B04BFA3BA52BD6F
:10905000D23D873CDA6C0EBE344EE73D57C54ABD63
:10906000AF999FBEF66F3BBEBB31913D4A166A3D3C
:109070001395703ED6722E3EA8E314BF2C919DBD71
:10908000A3C362BD9C2E16BEABCEF63DDB70B4BB57
:10909000C7DAE1BECACD6DBE20E2E3BD652C183E45
:1090A000517BB4BD7149DBBD00F6EFBE2C2D01BE76
:1090B000F53D9D3D93E23ABEBBFF4FBE394F47BEE3
:1090C00031EFCABD429D0ABE2E79493E1516DA3DE2
:1090D0009D0C3BBD6865E5BDFC1FECBD329922BE11
:1090E000BCF7923E7701D03C018F343E5371803CF7
:1090F000035685BDF00021BC2E39B63E58538A3B3D
:109100007D8F383E57DD1D3EDB08A8BDCF5061BDC9
:10911000FDD4C93EC220303E11D1773E91C9593DA0
:10912000DA161EBC16138F3C892D493E1C6ADE3CA4
:10913000F72C983D9728FBBD8FE690BE7042ADBDE1
:10914000BD30B03EA7F8EFBCD00041B9579343BB48
:10915000446EA3BE1EBE15BE13C6A83E491C12BE59
:10916000D858FA3DAC73383E5A34E83D99860EBE65
:10917000901FB33E9509783D52FF93BCB25038BC66
:10918000BD2C72BD9DA54BBE023BB53EA1CF5CBDC3
:10919000F6963ABD4C5C01BD24083DBD4E07FEBEAF
:1091A000EEC8073EF8A31E3D885FC13DA3754BBCCA
:1091B000DBD391BDEB5D29BF579160BEA1C7F13DE7
:1091C000341DDD3EE3BF52BEA77BD23E3CEE573E90
:1091D0005491A1BD6247863E7B80F83D307247BE08
:1091E0003EB1613E98E09C3E547FFDBC4203793D18
:1091F0006B20583A150BDDBC1025333E0EAA163EE7
:10920000FC8107BE7D9D8C3DBA110A3E84A90FBE2C
:109210009DE792BC251CFCBC48134A3D25AD8ABD88
:109220000E3CC53D3D96D1BD30526EBE6C03DB3C5D
:10923000984249BED281BABC08888F3E8309333D2B
:10924000117CFFBD01969D3D227795BDDC846B3D71
:1092500034AB4D3ED3652DBEA118623E1287FEBDD4
:10926000C5AF8E3DACBAED3DAA32863E6BE753BD2D
:1092700099236B3C2014ACBE388A25BCE637A8BDC8
:10928000630BFDBCFEA8093E8A06163E426995BEE8
:109290007BB262BDC43199BCBC1C88BDB9F73FBE6E
:1092A000B0BCCA3BCF04D93DDE9C283E167E80BEB2
:1092B000CC87203E36A6D7BD830926BEC42987BDEC
:1092C0005052133EE9ED8BBCE18E963E9A79ADBCCF
:1092D000B2CAD5BD33C298BE3106BD3DDACFFEBCA1
:1092E00002EE593E73DA01BDC7D540BDCB778EBEC5
:1092F000BF9C01BD50F9653D9932523E293D513D1B
:10930000533C0D3E25B5BB3C40B821BD4F6040BE2F
:109310006270673DB1FE723ECBE9193B0FF132BE80
:10932000A04776BC3D9A16BEDAEE66BDD015F23D7A
:10933000062EA83D69710A3E37AA41BE0B058DBEB7
:10934000791FEE3D3C22563E2DA2A83D8B108C3E4F
:10935000A274FA3DFB7D86BE4B60103CD0A6903DCA
:1093600022AF33BE3924DF3E2979833D85740EBD9B
:10937000B93A0C3ED58D463E552E053ED8F71B3EDC
:109380002C4AE33D179F6CBED192A13ECB6E53BEDB
:109390001C9B4D3E8CA9EE3EA228B83D237921BEF0
:1093A000217B243E6901053E6D06B43E8FE5C43E37
:1093B00051F588BC9B8DFFBD14DA533E7158813D39
:1093C000F0D4B53DB921A83D54C9C23D43C377BDD2
:1093D00061422D3EB7F63EBE87A8B23E5CF0D63E57
:1093E00018F9A6BCE542AFBDBCB54E3E85EBE83EE4
:1093F0007DF6813C3077213F45020C3D96B329BE76
:1094000029519F3E62E37C3F03DA193EC185983FB4
:10941000436066BD968688BE4A2D3ABFBFE749BF06
:1094200064172BBE8A2B28BFE72E94BED990A0BE0E
:109430003D69C8BEEBB8DCBE0636E03B565544BFBE
:10944000440F073E807AB2BEA98B90BE4A9902BFF4
:109450009B7B91BCF37FA0BE2A48C83D491501BE45
:109460007B5C05BED78BE5BE09B86B3DA42929BE40
:10947000743ED8BDA4F68BBE7FA656BE8A8702BFB7
:109480006FA7AF3DC840A1BD8D85C03DB6D4C9BD55
:10949000528AE7BD9FCB75BEDA6C893E256D44BE0E
:1094A0009B9425BDE3BF69BE87B8DD3C825B503B22
:1094B00089D9703E5F9754BED4D66ABD3E9C34BEF7
:1094C000E650CDBC32E52E3D830E7D3E2041553E1B
:1094D0004232A83DC9C8583CEFB184BD7FEADBBB2E
:1094E000E2305B3E0E1A433EC576DE3C6FC653BD8E
:1094F000043ECE3D77FBB33D994971BDDB23913DE1
:109500000E7E383DEF3B333E2BF9C23EE292A23E47
:10951000B4F5D13D7A72A3BEDF9E7F3DE0B51C3E1F
:1095200082EEF23E0C97E43EBEB705BCD872CFBEC9
:1095300098B0303DE248953E76F77A3E5FCDE13E09
:1095400006132F3ECF8BD8BE3146E63D7835463EDA
:109550004B70F23E065A0E3F5543293EC4533ABE65
:10956000EA639E3ECC0C063E7E24953E0B99053F59
:10957000600BDD3E08AEBBBBF212AC3EE289513E51
:1095800064124A3E1C78393DE8E2133F5DA3C4BD36
:10959000D6D4243EED526E3E9ADC1A3EC757943D17
:1095A000AC96F83E74FBEABEFF4E743ED463753C45
:1095B0007E87313EB8A3223E96F2993E78DB53BEB9
:1095C000E1EF81BDE9A23E3EE668653EDB9009BE63
:1095D000BEF3F13E4208A6BEE3D52BBD7638D7BC1C
:1095E000BF11573EB3031B3E40EFC63ED0C90FBE6E
:1095F0004BA9063D6582933E41E0213E307A38BE5C
:109600001BCF053E87E991BB7B0C72BE01EAF1BD21
:109610008F9C1C3E8AAD86BE17F49A3D58A431BE7D
:109620000F3625BECAEA953DB1278C3E73443FBE36
:10963000E42FE23D0088F1BE3B8005BEBF305D3EB9
:10964000E9F1273CFBAA13BF0912A53D813F32BEB9
:109650008F1953BE2856913DB581A83D35047DBF75
:10966000C12C26BDC52C283E20593FBE03B943BEA0
:1096700093FA3FBE4AFE773F9BD7CC3EE4AF5C3FB8
:1096800036C7343C3F2FC7BD399510BDC4AC703FC1
:10969000AB7F0C3EC156813FFF063CBED7F535BEC1
:1096A00019D450BE2B6B4C3FE374513EDBEA433F71
:1096B000F010BBBEF55D05BEE9DAC5BEDFD7413FA0
:1096C0005D670F3E0A73323FFA0F7DBE0BC0203D2F
:1096D000BAD3B9BEAD7B523F6D7E8E3EC9B3B13EAB
:1096E0006858CDBCD0D00C3E3A1264BE2D3C1C3F15
:1096F0002ECAB43E8EBA1F3F82726ABE49F84F3EF0
:10970000671312BE9333533FE90B773E60D0DE3EC2
:1097100026C394BE8780003E3D0F82BE9FC8153F82
:1097200030C1113E4F18B03D685354BEEC6D2B3E16
:10973000EF91223AC2D4363F55901B3ED2A31EBCB5
:10974000ED19A7BD80C24FBD17AF73BC1D2E133FCF
:109750006802593EBD0B26BC2D1A52BE13BA573EA5
:10976000700AB7BE158A183F6DB3123EB8FA0E3CA8
:109770002E9226BEA568433E5C6C413C2394223F5A
:10978000C03DBD3BBCDE38BD34C190BED98AB33EBE
:10979000543A68BEF8280D3F88B218BEC57E18BE80
:1097A000723FC4BD7CBF953E452710BE8657083F1B
:1097B000E83DFFBD3FF639BEDFE699BCCCD5BE3EE5
:1097C0006C8D2BBE32BDF63EE2268F3C35134BBE70
:1097D0007AD999BE2B00F73D8CB73DBEA82E583ED6
:1097E000FD89D0BD59DA04BE81044C3D47E9AC3E49
:1097F000850BC3BD37ED983E08F3B2BC316091BE16
:109800008F98763D16F66C3E92C56EBE479EC7BCDD
:10981000C750BC3D78682BBF7AAC063E1681C53D6B
:109820002BBEF0BD65FE37BDDEC6BA3E9EBE35BF5F
:1098300055EE38BEE7064C3E8EBC38BEC5675DBEF1
:10984000998C883EA6CAF8BEB2103FBDA2C3223E84
:10985000A1C568BDC861A3BE73F8943DCE7E12BE9B
:10986000FCA4D03D87F6EA3D30EE1FBE312871BE24
:109870001AE70ABD22BAEDBD4A41A0BD58AB4E3D24
:10988000D4D879BE02C378BD9899E13DBC748DBE31
:10989000AA5ADC3D8C85423D7A47B5BD055BD43E76
:1098A0001A0CFFBD48FE3C3E555BF8BD618569BEA4
:1098B0000223A4BD81B4033F08094B3E697BD43C1D
:1098C000039D953EDFFF0E3E6051F4BE5F983CBEA7
:1098D000A41631BEF7EA933D7B294C3E278C503EBF
:1098E000F9286BBE86EFD0BEAE9475BEAA193DBDF9
:1098F00003988A3E8730593D44767EBE5AA92BBED6
:109900009EE65ABDEC00B5BC9749A53EDDAB783E5E
:10991000B35F44BE4DB673BEE833763E3A17463D5C
:1099200091D5FC3DC210BD3D2D32E7BDD8FD04BF31
:1099300022C8A3BCB97ABBBDF68D3A3E6BF9ACBC6C
:109940002A279EBDEF8DECBECAEA02BE87B65B3BFE
:109950004816E43C7F1901BE845936BE66471EBFD7
:10996000F3EECEBB9B86E1BD70D8373EE68E153E4A
:10997000846536BED76C8CBF5D4C423D071774BE04
:109980006107A13D134B5BBE663F00BFCEDF7EBFCC
:10999000AC0CD0BDF18868BE3EB9543EC276F73DEE
:1099A000C47BDFBEAE9663BFC5BC88BE7104943C69
:1099B00031C6413E11720FBDA955A4BEEABC72BFAB
:1099C00054F875BE3C283C3DCD74233E8E2C033E9E
:1099D000DDE3FEBD384462BFDADDAFBD55BA9B3C66
:1099E0008424DC3CB460133D3E1B80BE0B3059BF69
:1099F00097C5CD3DA3CE113E1E4396BD92DFDD3D02
:109A000088F32DBDE3F123BFFAE73ABD389EFE3D52
:109A1000B9C9843D9A98A2BA853F65BEB369B9BEFB
:109A20008AE2E0BDB1A71E3E2009163C7E85A8BC97
:109A300076F838BE7DB789BE44FCA13D43D9EDBC64
:109A40000712EFBD51AA863DD69697BEC5C53ABE50
:109A5000E40183BDFE0C593D7D2D28BCF7700ABE84
:109A600009FE9FBD2E5759BE1C612C3E84E0C53AAD
:109A70007BB88E3ECC128C3D6466213E2BC3323EB9
:109A8000652E2C3EA7864B3D2D22EE3E26DB943DD7
:109A900057608F3EB920663E56EA743D1E7289BDFE
:109AA000D6D1953EB371AEBC7716DC3ED8D3093E15
:109AB0002988CFBC12B582BEB6052A3E02009DBDE4
:109AC000C343F63E83F0C73DA17D503DEB83D9BD36
:109AD000DBC7013DDF5FF33CA7C21E3FDFC2403E54
:109AE000E94C973E238DB9BE98FB27BD336163BD1A
:109AF00034AC363FABDD8CBE3C9C263F61111DBFB4
:109B00004F24333D506012BEB5705A3F133539BFF4
:109B1000B6C2173F88A898BF8FAF01BEB646873D33
:109B20003FEE413DBAC6943F1AE32B3E5B11773FAF
:109B3000BA94153EBCA40FBD1E000A3E82D6133F48
:109B400028FC6A3EA3DE253F6FA600BEC8F3E63CB4
:109B5000AEADDF3CD2FEE63E0D186A3E6A57F73ED8
:109B60000C7A03BE509EA4BCBE4D4DBD6D24C73EB5
:109B70004BC7A13D3E45313FFAEE213DBF82CD3C72
:109B8000A2AC5A3E9BE9903E69956FBD3AE5E13E35
:109B9000A3E027BDCFA0EA3B9128363E35EDB8BD06
:109BA000035B2CBD99FDB73EDA99DEBDC7D91F3ED8
:109BB000A3808F3E9A5251BEA9A1EA3B1F48C03EE6
:109BC000E3FBBABEE1B003BE3D2F363E7B23AABE07
:109BD000A3B9883E5674C93EC84ED7BEB2561B3E86
:109BE000EBC0293E17F170BE61A5863D00D95D3EF0
:109BF000A4581EBFC175CE3D1D2F3E3D679233BD9B
:109C0000D45357BD185BCD3E66F50BBF8943373D36
:109C100050406F3E8765C1BE628E85BD416B263E5A
:109C20005CE828BFDCEBAFBDDC5F493CCE4176BED3
:109C300019614DBEE660583E961D0FBF11EA4EBD3C
:109C4000C41945BD3575B3BEEB9332BE44CFD03D8C
:109C50002BD60EBFB9700DBD2FA5B5BD6E53CDBEB1
:109C600045C8AEBE399F3F3DF584F2BE48B703BE3E
:109C7000EC48E2BD1E3715BFB9B2C2BE5217A23DB5
:109C80000E0869BEDAA8613AE0E90DBECC66ADBE49
:109C900066E3A4BEC19B703E6D67FDBD0D2510BC83
:109CA000080F4C3DF9B792BE3665A1BE2998DE3E3D
:109CB0003437B8BCC4F50ABE8AB7EB3D2F9109BE54
:109CC000512AD2BEAB5DE93E6072CF3E83048A3D2D
:109CD00068DF4DBEFF1804BF7D4CF6BEDD35203E6B
:109CE0004697013E36F8043EC2DF7A3E012460BE4C
:109CF0008D77E6BED8369A3DE525EB3EBE29143E6B
:109D0000AD7AA33DBEC1E6BE562706BF5E92FEBD3C
:109D1000CF3D883E06FFDE3E4903143DF7BC0DBE35
:109D2000878DA7BEF24FA7BEAAA4773EB960153EA5
:109D300080C7B6BD35C066BEDD2FA1BEF7A41DBE6F
:109D40005FB4763DD684DE3C13A9903D365089BE83
:109D50008BDBC4BD99DDA03E99223E3E3E610E3EA6
:109D60001E0CFF3E3A6512BFE874CEBE6A8EC53E39
:109D7000A32457BEB4D65C3E9B4729BE4687CBBEC4
:109D80004D3A11BE6CF072BFD45D64BEC9EA1C3E90
:109D9000B5E5233E61D8233D91A042BDFF7837BF92
:109DA000975813BE77FA8E3C3AE8AB3DD8A7E33C10
:109DB000AE88963E740EE3BE09984F3D617D653EC8
:109DC000A4D3F3BCC5619D3D20F539BD9DB6223EAF
:109DD0008EAEC9BC0E4A033ED9462E3E3C01B63D6E
:109DE0008FF5A5BBB35E0C3ECA478ABDEE94863E96
:109DF000FC96083E2C2AE43EC8E189BE9771193CC6
:109E00003C0B783E9417893E1D73F03D9EECBF3E9F
:109E1000D422A6BE4DFFA33D7667253EFDADED3DA8
:109E2000CE970F3E6D40F93E903BA13B39FFBC3EC3
:109E30007ABC913E87DF3F3EDEA1B33D47B94C3F40
:109E4000F86E29BE337D9CBD5BD6823E61C5C7BC22
:109E500036DC1A3B5695173F4FAAB73DC35282BE18
:109E600041FCEE3D2EC4E43D3A5113BD1A71E83E6B
:109E70002E7C4F3EAB6C96BE8873DC3DCBC3AF3CB3
:109E80008A0F8FBD8F3EFA3EA3940F3E9C0487BE7F
:109E90006D6FCCBC2EF75E3D185548BDB2E0583E04
:109EA00043F5463E608614BE03BE7ABD0650003EB2
:109EB0006F33DABC4D8E3F3E5A61033E3D566EBE57
:109EC000088620BE9B29CF3D996603BDC3C3EABD6A
:109ED000CB1AD13D602EE33DEBB327BE2D438D3D24
:109EE00018A423BDC3E018BE654F4CBEE1F788BD82
:109EF000981154BEDDB13E3D14BE773D18F650BEFC
:109F0000498E01BEDA1216BDDF49B9BED3899EBDA6
:109F10002C0CAA3D5876C3BEF8BE033E1DFE5B3E28
:109F20000AA528BE4172B5BD5DFFDDBC9713FBBE1F
:109F3000366CF93D8EDB02BFD2392FBECCEBD4BCE0
:109F40004E4613BE33621DBFC1901DBE812F06BF9A
:109F5000DD713CBE121402BD0AF355BD561918BF7F
:109F6000F424EEBC850E3FBE7018313D3B8E9FBD84
:109F7000BA7E0BBEFA1053BF6CC9D3BE31A795BED3
:109F8000E26DBF3D96121FBEB01680BEB6D65CBF56
:109F9000795CC8BE519085BEEABC3E3EC76CCD3CE4
:109FA00074BDA2BED3BAAABFA90889BCCA0524BF82
:109FB0003E78543E9F84EA3DCB25A0BE2ABB05C017
:109FC0007F5790BED8F523BFD487793C9D2602BE2B
:109FD0000F26363E8506BCBEDE630A3F3C62483E25
:109FE0007E3E433E4310B23DB50C543E49A1AABE4D
:109FF00047B2EB3E9FB6CC3E8BBC4C3E836504BD66
:10A00000833D783D8043C7BEF236413EC8A6253F1A
:10A01000CFABA13EC1D89C3D9619C3BDEED7F4BECF
:10A02000CD11813D5156EC3EC04C673E63DBD43DC3
:10A03000F0D3043E73E604BF703A6C3B5B2DE23D07
:10A04000A721913E360100BD1FF18CBCC485C6BE60
:10A05000B5F3413ECDB761BD7939B93E6C28453E77
:10A060000E85473D05A3D7BEC77C523E6D5A4BBEF9
:10A07000CC2E813D813A473DFB911B3D999ABDBE57
:10A0800001A7873E31327BBE76B883BEC9070F3E3B
:10A090004A531F3EB448C4BE43C599BB92D775BD51
:10A0A00066939ABC3CAF15BB6BB9E93DAB3691BE2C
:10A0B000F7E45B3E7B641E3DB690E9BD4E149E3EC8
:10A0C0007FCA943E2C3B5BBE4B3489BD3B3E20BED9
:10A0D00069EF04BE0459AB3E37431F3EC12E91BE0B
:10A0E000C52150BD0A6B37BEDA5F99BE5813923E48
:10A0F0004B8CE13DC871ACBE091CBB3DE15F333EFA
:10A100004A982CBF063E7C3EEF19F9BDD6C0F93DFA
:10A110004DB5243E93CD4C3E85D690BEC863333EAC
:10A120001E8986BDD89DADBDCBA8CE3E3A3C253D0F
:10A130006C9C3DBD9BF2A33E90103B3CFFDE883EF5
:10A1400088395C3E7C27323E8FF1873C85AB313DC0
:10A150000ADA0BBD5AEF633E969A223E3B5A693E9D
:10A160004ECFE63EEDD0A93D67815E3E3AA6FB3D6F
:10A170002EEB903E3DE204BE6CD20F3E49A961BB7E
:10A18000C4314D3E6E49A03EBBCBAEBD8D0C1ABC5A
:10A190007138673E36FB933E09BABBBB8C58713EA3
:10A1A00087B0773D11F924BEE22366BDE3936B3C93
:10A1B00027DEE6BBF6660D3E2186D43E856747BDA9
:10A1C000E52D3CBD0B36DC3DFB5F13BDAE39363FA4
:10A1D000B073B13E0F074DBEA702B63DAA542A3E4A
:10A1E000D1B176BED31B303F556BD73E68850ABFD1
:10A1F000DB32253EFB71B43EACB788BE4B597F3F86
:10A200001B18D93E441F0DBF3F5E043F49FB6F3C06
:10A210002F8843BEC6A85A3F8291253F179C1CBF7A
:10A2200073812CBCC1B7A4BDE4209C3E1AC1233E5F
:10A23000E71E023FE82D383F1E360BBE4DAE973B62
:10A24000DCC6FF3DD3E4923EECB2E33EAFC6523FE4
:10A25000408CCA3CDAA2BA3B235F423E65B13D3E28
:10A260003128B2BC5222003F51AF343DF6FD50BB05
:10A27000CE78723E22EBDB3DBD4A113EBFF3833EFA
:10A28000AC687ABB4882FABDC063023E2199573D53
:10A2900006AFF1BD6D31DD3E1BFEF9BD98EBACBDE7
:10A2A00061DE4E3ECADCBABD8A28013C97B48B3DC4
:10A2B0005A650CBEF81AA9BD3987733E25E44D3E98
:10A2C0009081CBBD17DC65BE249717BEBBFAC4BD19
:10A2D000D508223E97EB3E3E67762F3CD5ED3B3EC0
:10A2E000C72963BECFEE31BD5CE80E3E931E943E9F
:10A2F000B7FCD4BD2280273EC0D498BED5805D3B3C
:10A30000902C293ECF6C783EDE569B3D2DF17C3D56
:10A3100072DB38BE6E8C5D3D77231C3E099EDA3EB3
:10A320001A288F3D5A2C21BEBD6C20BE7B69193E78
:10A33000172A873E9401B73E2CAEC8BE16BC043E19
:10A34000C655C8BEF2F44F3E8103E03CE6B5533F2C
:10A35000BE2CEFBEAB219CBDBDC434BE80EC4EBB59
:10A36000A2E486BDC1732E3F1EABF2BE30240ABEEE
:10A370008F1682BEB3EE893DABB6BBBD6B36153FC3
:10A380005942B5BE7EB819BE7A7EA3BD4AFF413D93
:10A390005C95CCBD81F0013FACD14ABDD1B6273D23
:10A3A0001E5DEC3C0BF5C03CC3B0EA3D5CA6B53E7F
:10A3B000B6A03DBE70B6983EBAE260BDA9C9413DA7
:10A3C0001CE7CD3CC3D1CF3E17BD103EE6743F3DE8
:10A3D000F635993ED7A9C53D7C728FBD67317A3E6F
:10A3E0007C8A3ABE03E928BDF49C973EECFCE2BCB3
:10A3F000C74A4CBEEB73C63EEC7236BED5F0D93DB3
:10A40000FB62EF3E3C0F4F3ED9F3F4BD694DF03E89
:10A41000A97907BB07B9C13D74EC123F4828593EE2
:10A4200009C087BEEE6E253F540481BE68131CBE72
:10A43000C37D7B3EEFDE983EFBD280BE4305853F69
:10A440004987F63C12D60FBE0A738B3EA277853E33
:10A450001CF653BE205D963F0209B63EA7B893BED8
:10A46000AB0F0CBE542A4E3E408E63BEF0F9B53F92
:10A47000E0795F3ED90E793CA9C71D3D63305A3E55
:10A480003B71A03DFF442FBE78095BBF5F3D623F3B
:10A490008C23D4BDE91CA73E0C28C03EB62A75BC4F
:10A4A0000F5D3CBFEDE63D3F23C8CBBDCC295E3EF2
:10A4B0003BC9E43DCB9CCE3D5BC129BF7E362B3FE3
:10A4C0004AC45F3E4D934D3EFC074D3E1B563FBE7A
:10A4D0001A70D0BE6EE2473FAE70BE3E11ACFB3D7F
:10A4E000D434F93D9BA1EEBDE5B6F9BE1ED18E3F39
:10A4F000EB7729BD0264F33DEEEE1D3EC74F9B3D59
:10A500008268B4BEF356943FE1F0143EA59C103E21
:10A510006D65253D04BCF7BD22B7B8BE681B5C3F26
:10A52000A7EF64BE5EC2E83D7FEA983C0DFF0BBE1C
:10A53000B7357DBE9D466C3F6ADE523E155492BDD6
:10A540004D7D853DC55216BEABEDAFBE05EE863FD7
:10A550005B83B23EF3BEC5BDFCE05F3D8C950CBE97
:10A56000111601BE4F87833FBFACE93EF6721D3E18
:10A57000664FA3BEDF0368BE55228B3D9DBC3A3FAC
:10A58000FDDD983E3EF5523DC20CDB3C1D5F04BE36
:10A590001189893D7F575E3FA49AD73E93F990BDBC
:10A5A000DDC2ADBD59624BBEC8E5CE3B2FC2903F68
:10A5B00013C5DF3E34D0273E538C913DA898C9BDCA
:10A5C000192F44BC3E5B823F1088513E500617BD98
:10A5D0000FEEB13C5BD220BE720BB33D1B73393F13
:10A5E0009A719B3E291D8C3E15647BBCFEFE1FBEEE
:10A5F0005196873EAC88143F47D5523E9C60743ECE
:10A6000039DCCABD2A0806BD13690A3E61B89D3E01
:10A610004FCFD63ED2B2AF3EBDA325BEC8E1283E45
:10A620005C99AC3E8812BF3EC326963E91A18E3CFB
:10A63000D8CAEDBDB404A63D6D2EE93EE4EBA03EC4
:10A64000AE42F03D1F16B7BD52E7DFBEFB2B9C3E6E
:10A650003EA6A13E1C96853E2E88173E1F65A33D53
:10A6600055D1CDBE8A76EA3E65EC293E91BCB0BD9F
:10A670003205B03EE11DD4BDEA7C7BBE7C7E4F3E00
:10A680000BFC073E876D243E8046AD3E093E99BDDA
:10A69000B57EF5BE441CF13E21DB813E6C7F903ED1
:10A6A000BEC0A7BC248DF43EF22C58BEE4872E3FDA
:10A6B0001BD5983E2901D43E5F2E843DC825AB3E74
:10A6C000413CE7BEB6812D3FF6DE873EC492C43ED4
:10A6D000E72C313FCA893B3E01C9B13EA9449C3EAB
:10A6E0003D2F903EC4140EBFA623C13EDB3C0A3D65
:10A6F0000E0CDF3E8B94CF3E8DE81B3EF4E47CBE17
:10A70000D3D1A83EB505F33D3B7B173FB574833EDF
:10A710003EC5D43E29CB81BE4AA9E33EE4959D3D8A
:10A7200025F0B53E3F95DF3ED578AA3DF8B178BE1D
:10A73000D9FE243FC9974F3EB092863E2B06583D26
:10A74000DAAA683DEF424DBE268B293F1F9B903E03
:10A75000DD11123F0B56C63E8DF52E3E4424143DAE
:10A760004571203F31E0573E5E6B1C3FB1F4DE3E49
:10A77000EA5BCB3EFD4AF0BD6B8AC33E7F06973E47
:10A78000AF10DB3E0BE5BC3E73D00F3FDC4A44BD4F
:10A790003EFF053F36CFE83E37BB053FC2F6AD3E34
:10A7A000371B063FDAF4E4BD96EFB83E772DA43EA2
:10A7B000CEF6D83E5FFE223E5F36D93EA0E955BEBA
:10A7C000E088CF3E32AB8F3E4299303FA6BD083D78
:10A7D0005A14123FACD0293EF018113E758E103E2F
:10A7E00071F6DD3E42AA913E4A840F3F089A0EBEA2
:10A7F000530B923E4F03573E2BAAE43E91B12FBE1E
:10A80000AF8D3A3F2385323E1AD8EE3E489806BDBA
:10A81000CA682D3ED7B99DBE67053F3F176A34BE53
:10A8200054355D3E5BE4F63D9CC3BE3E165AB2BE57
:10A8300073E7EE3E0E2C54BD9F6F923E97478F3DBF
:10A84000881E823E995473BEE9AE193F8FB8F8BD99
:10A850006ED2C73EF09E3D3ED4C1C63E2B57D8BDFA
:10A86000B5D81F3FEC198F3E8ACAC13EA9AC493EFC
:10A87000410B943E185E82BC3E1EEA3ED4431BBD93
:10A8800089F0623EAC4E4F3E7B970C3E0B7E9CBEE9
:10A89000264C123FF0DB323ED629693EA3FEE6BCD1
:10A8A000709F873C234AAABCB45F883EE9A4203E3F
:10A8B000D0FFA4BCD56C963D03F3953DECA09F3E24
:10A8C00000BD7D3E1DC2373E1A42963DBDD3973E28
:10A8D000CD1FCC3E0462D83D1C38083FF4DCF23E6C
:10A8E0004B2CE03CEECD003E90B1923E9231CA3D01
:10A8F0000C02CC3E32CADC3E8B528D390DB0373E55
:10A90000391EAB3E5753A4BDB107F83E70A0993E27
:10A91000AE75453D62E1F93C7D15AA3ED861B43D76
:10A92000E601503E0833023FDA768F3E277D703EC7
:10A93000B66AC53DE7731EBF01865D3C520F24BE5B
:10A940003B14CF3D69AA933E462D723D5D9046BEB5
:10A95000ABA286BE2DE055BDFDC2B5BB0DAF273EF7
:10A960004CD5C53C7FCBE4BCAB63C3BEC50E8DBE2E
:10A970003ABBA93CEC01B83E8F251C3EEE7FC5BC1E
:10A980004C0B76BE4CFA9ABB431DB7BB7AB2853EE0
:10A9900072C0AA3E4B6400BE2AD6CABC5314CFBEB6
:10A9A0009411963EE7D7123E0E9FC3BD68536EBE0C
:10A9B00033AC42BD5072CBBD0BD1123E1E818E3ADC
:10A9C000C8C5613E515CE0BE89C4973D03857F3EAA
:10A9D000C8548A3EB37EF1BB7225B53D387ACFBDEF
:10A9E000DEF70FBC2AA280BCC20AE13D943E5F3E66
:10A9F0009D0A75BDDB25A13E15431F3C7254B13D38
:10AA0000A03713BED2EFA73E954E603D7F80CE3E6D
:10AA1000E8C8A6BAD13A47BE0F48833E3E70633EAF
:10AA2000F9F04B3D0A72013FF762D8BD8F2F39BE56
:10AA30004538873C5E108F3EB02987BC7395A03E99
:10AA40007002E8BD4740403E375F183E10AD383DCC
:10AA5000731424BE0B778C3D48AEB7BE48199A3E9E
:10AA6000CA2591BD641EB03C88DDBE3D6BF8903EAA
:10AA70001A2F32BE154BAB3DAE5AF93C70561D3EF7
:10AA8000841D1C3D2548E13EA68844BE1579BBBC0B
:10AA900061CDA5BEC6F37B3E72B0333EA2B19A3EF5
:10AAA000250458BE78D2793E655E7EBE96E4173E98
:10AAB0001F2B4E3D94020D3FB5E4D43C26F8923D49
:10AAC000A25479BA0063BA3D770B20BD42F3E13E50
:10AAD00021012FBE28B7903EFA8482BE1862D43D71
:10AAE0006C3988BB9179E33E66BDBEBE3C1C1F3EFF
:10AAF0000C4C3DBEBE26A4BC7BEE123E4369043F17
:10AB0000BB40683CF9EDC93EAA159CBD703F033BB4
:10AB1000286DA93E6B7AAE3EB6E633BE37821F3F44
:10AB2000EC4A00BE4A2C5D3E6CF2873E1381383EF3
:10AB30007FFFBFBEC1E1373F1B6E9FBD0413973D32
:10AB4000639AE33DC7DCB33E503303BF1A65203F31
:10AB5000DFD3C5BEEF7A1E3E856E9A3EEEAEC53E91
:10AB6000F08CD3BE1635F33E7F920FBFE23F47BE57
:10AB70004394FD3ED9B0723FE8738ABE8708483FD0
:10AB80007FE6463EFEB819BD9CD5C83EE47D0EBFAB
:10AB9000B1740D3E664AB8BE7399773CF472D43DE9
:10ABA00078758D3E2C7BBBBEE2F407BE73AF23BD30
:10ABB000031C4B3EDC65D13C75A3303E896001BF70
:10ABC0003CC978BD45FD0BBEBC64603E7992B63D84
:10ABD000F6FB37BDDDFF4BBEE5011BBE410DACBD35
:10ABE000D59C623EF79FAA3DB214373E8F289BBD8D
:10ABF0000E67A3BE2086EA3DF983203E4C9318BC25
:10AC000094F3A5BDBC7F8ABD61C78ABE14714EBDD9
:10AC1000CF13633C69AFB5BD2D1D0EBDFE2AF4BD3B
:10AC20002888BDBEC0383CBD5FBC4F39DFFD6E3DDE
:10AC3000A2D4673D0AB019BEA3FA87BE9C75863EB2
:10AC4000B60490BC2D14A0BDC37A403C9772D3BD0E
:10AC5000BE10DEBE6A92DB3E299DF63C170586BE1D
:10AC60001D511FBDDA7F4ABE4EE5D0BE4B6AA33EE2
:10AC7000D4732F3D2D5EB9BD44FA06BEF3E2F63D16
:10AC8000F6A3BCBECEEEE73EC1C68BBEC3AE773CDC
:10AC9000D2C09DBE52FACF3D6699EEBDB2C6443ECB
:10ACA000F0C4C1BC77432F3D6B28DCBC963626BE72
:10ACB00026185ABE6AD8173F15833CBEA79B8DBA8B
:10ACC00002E481BEC0B3163D113333BD37BC6E3FC5
:10ACD000A0E711BEE7628FBD6B0564BE0139633E1C
:10ACE000C06A163DA173E43E579AD9BD41FE15BE18
:10ACF000F96F8BBEE360623E8632EFBC048D9F3DF0
:10AD0000085E69BEC07CF2BD2F3A36BE3C50DD3DC8
:10AD1000449D513EFD67013DD740D33D588E1ABC3E
:10AD2000172029BEF688443EDD0885BDCF3087BE9A
:10AD30003F3A05BD6C907AB74125BCBD9E9D2C3E27
:10AD4000B8A7453E8BE041BEE226573DC50ECE3D3D
:10AD5000A65E98BD48CBC73E77612E3E491900BE1E
:10AD6000AA9B163E3D206A3E423B59BEC5AD193FE7
:10AD70008260433D8B1C8B3D6043B83DE724323EEF
:10AD8000A3EEF7BDD98B0B3F895CD43D26D31A3C8B
:10AD9000C35B9F3C5D4C7C3E4113CFBEDC38533FD0
:10ADA000AA947FBEE4B3843E4D0EE9BD3C77E83EF5
:10ADB000F705DCBECD008C3F800557BD89B1203F33
:10ADC0007E59273E4804BC3E99E3D7BE457EE53F09
:10ADD0006F3763BECFED3F3FB1C34E3EDD5E94BEE5
:10ADE000F78FCDBEFAA405BF7D8E99BE100042BF7D
:10ADF000957D70BCFD9747BD07A803BEA76604BF3D
:10AE00003C600D3E4BC305BF2B35063EC3540EBE02
:10AE10005C4F80BD2233D9BE03353FBDCBE75FBE5B
:10AE20007B54403EA321983CD8F7D0BDF3320FBFEE
:10AE3000A93A573D8CDEC73C7F22353E83785EBD04
:10AE4000433D89BD620020BEBE9C1FBE1A6990BEF4
:10AE5000300F003EB5AEF7BD88AC5CBE4B0A83BC7C
:10AE6000AFCF80BE950BD1BD153ADA3EAA6FE73D54
:10AE7000C4B586BD050581BE2E2B953D31B740BEBC
:10AE8000C7B6693E13643BBE3738293DA90CF1BDF6
:10AE90007C30613ECAD108BFF329EC3E6DE1543DE0
:10AEA0003465C33D91B818BE9490EC3D412623BF54
:10AEB000E20E543E863A07BC3C4F253DBD0F08BE0E
:10AEC00061808DBC088B18BFD9269D3E544B333D05
:10AED0005930EEBC98E52EBE42CFF53C606A6EBE9E
:10AEE000ED7A693E17E9CE39CE9DC43C499FC6BE76
:10AEF000CFA09C3E7F2DE6BEDE9D8D3D26F68DBB10
:10AF0000D2208B3DAE59DFBD6994003FC25CC0BE0C
:10AF1000D31CB23D0535E23D1060453BAABAD3BE15
:10AF2000C310123F6FE1C6BE016253BEE43EB33DA3
:10AF300015BCCB3D688321BE6856A53EE085C0BEEA
:10AF400091F8B73BB303A2BC45CF9EBCA6D2A8BE26
:10AF500040D0263FF9A30DBE10EEB0BCCDEEE13DD2
:10AF6000DBEE39BC9D91A5BE9BEBDF3E2B9427BE4B
:10AF70001D8071BE1D47A63C092D8F3D3C79DEBE6C
:10AF8000C1C8003F699325BE16905DBEA764063E0A
:10AF90001182143E89C4A3BE5834903E9E3ABCBE72
:10AFA000D794CBBE946D00BDC1584BBC0DD3EDBE44
:10AFB000D734443DDC2FA0BE1DF908BE90716E3E13
:10AFC000D6A01C3EF195C8BEFA8E90BDD6B0B6BED6
:10AFD00045046FBE18D6083E4479503DDD4F8CBE07
:10AFE000275164BE24DA15BFFCCA2EBE1314ED3DF2
:10AFF000F681313E38D014BF552B05BD569014BF95
:10B00000942715BDDA04683E0F41143B6BCE3BBF5D
:10B0100027AA73BEF77C81BF2C7346BEB837033FA7
:10B0200005C9E43C437B3BBF76226A3DEEC40BC0BE
:10B03000C1870B3DC4CFA5BD10F1FE3C02C585BF45
:10B04000D9CE363F1A24C23E9B7FFDBD3A18A63C9E
:10B050008290893D003E0FBF9F54143F0E84AC3E4A
:10B06000EFCE12BDCEA7463E4CAC24BE76DBE1BE91
:10B07000279BC03E68FF903E6E555D3D2FB6D9BD03
:10B080002D14333E6C9018BF289C7F3EF9239E3EC2
:10B090007EEF08BE2F9C0D3E5921783E502B9BBE63
:10B0A0004EBBCA3E2E37433EFA13B2BE8B631A3EE6
:10B0B0009C30BABD3D8AA4BEEE837D3EE01718BE2B
:10B0C0004D32E6BE4459D23D763A243EE44002BDBC
:10B0D0008889B63E8CA086BE2E85AFBEEFE2343E98
:10B0E0003B8167BCF45EBA3D90D0B43E9F8DA1BE5B
:10B0F000A9019EBC02D8B83D2312943DE47D913D48
:10B100000851863CD687B0BD18F332BDC2CA5DBEB9
:10B11000D4D9343D2BB9E8BCDBF3B13DC5DD85BEE8
:10B1200081BAD7BDDAB888BE51C7053E55A3BF3E28
:10B1300073BA603EBFE024BD49D838BEEED2C4BD6C
:10B14000FA1900BD268A683EA465F5BDF9C92ABE74
:10B15000D51299BED10D94BE5918673D301BC1BDA3
:10B16000C03087BD484156BE1EB046BEE44F15BE36
:10B1700058F1013D8A969F3DA3A28ABD042666BC74
:10B1800063BD6ABE5399FABDA621E23D6CC1583E2B
:10B19000D9DF543B98D49BBDB75243BEBD3FDEBD03
:10B1A0001D24063EBD18443F18F8BFBD76CC0B3EAB
:10B1B000640A88BE4FF828BE7C3C393EEDED823EE5
:10B1C0008C4C11BEB1CD203E06CB0CBFFD6F5EBCDA
:10B1D000B141923E8907663EF4297ABE0C11023EC7
:10B1E00085FE67BE045C9ABD9DBF0A3E9756573EDA
:10B1F000D88DD5BD6813B13D429E4BBE88F4F43D59
:10B20000132DBBBC26F1843E491FAC3D817A043D21
:10B21000EC567BBEC203CB3E9384FFBCF9C48A3E8E
:10B2200089CF8D3D5582A63EC046DF3C677EEA3E13
:10B23000E40352BD21DBCC3ED53E6EBEAABFF13E3B
:10B2400088C1F7BC12BF323F0543823E1EAED33EDB
:10B250000004B4BEF963C23EA228A6BE2ED9913F17
:10B260002258123F82DABD3E35E17BBED419E33E5F
:10B27000C0DDD0BE13BF1B3F051D5B3E8AD8573EC5
:10B2800016A13DBEB517AE3E904E10BDDB0F3C3E45
:10B29000F8F9403FF88084BEB13B2ABEFC67DFBEB0
:10B2A00001DC85BD226381BD6E74DD3E8CAE2A3E1D
:10B2B0009EB6973C39CADBBEBADA063D0E4D1FBEBC
:10B2C0004E8BAA3E480F013EDF1ECDBEF5E0E2BE2A
:10B2D000E16DECBD48113D3DADC85C3E5725C93E12
:10B2E0009DB30BBD61D50FBF725114BE7E2E003EC3
:10B2F000CEAB033EBBBAEC3E79C8593EE4E004BF96
:10B3000022E8D1BDE7F27F3DF1E8163E9480B53EDC
:10B310003A368BBE6987A9BCB026E8BD0C77513E92
:10B32000AD39503D2EED053FC1953CBE0219B4BE6E
:10B330006E9245BE6711B13DC9E0883EDCC3D73E81
:10B3400081BDF6BD2D4A50BEC097FB3D4D3813BDA3
:10B350001064633DF2526C3E601F7CBEE25FCEBE65
:10B36000C81A893DB960C63D2266C6BDC5AE373F25
:10B370007AD39CBE033C21BE532D243E8F647A3E7B
:10B38000D5E8233EE749733F7C02363D1FB1D7BD68
:10B390005A19763E5B599ABDF45F3EBE3C6D153F2F
:10B3A000D7E2ADBDE5A0A33DBC6492BD83E1E93A1F
:10B3B000857533BE77025E3F924624BE5337173FF2
:10B3C000B834033E981CE73DBC5D09BEF68E013FD4
:10B3D00080DDB73D327C233FDE5CD13E98D289BD13
:10B3E0004D2E133E44069B3E9E996DBD1D6CD53E71
:10B3F0006AD0E13E29F28A3DE274353EA04CB13E6E
:10B40000A533DFBD8CE619BD7521573ED2CF913DE6
:10B410006E7D0E3DBDDEFB3D8876973DB53D89BE18
:10B4200085A1223E41EB8F3E8610B8BD68B63D3EF9
:10B43000B0D28D3E3533853D3456EC3D54E80A3E5E
:10B44000E346AABDEFC0883DDBD1603EE6870B3EF8
:10B4500050F6C23C74A0C53D7F5CAA3CF005A53EF9
:10B460003968E13EB9657E3E64B842BE9070AABDBF
:10B470005DD5B23D607FC83E55C8CA3EB464943DB8
:10B480005C3020BE131337BD0CDB68BD4FBD9C3E46
:10B490006B879E3E992ED13D6727A4BE611D0F3D4F
:10B4A000C84E47BEA7650D3FE37BD63DD10E553F45
:10B4B0002CCF54BEAFEA2DBD6D254FBE45B7573FCB
:10B4C0002789543D8FB2383FC1C3E1BEE6755ABDEE
:10B4D0007EB1D7BE896C893F146C4D3E29A6463E8D
:10B4E00059A4A1BE149280BD3814883EB51BAC3E51
:10B4F000BFD2F53EE92F66BE3BE3A1BE5BAED0BD39
:10B500009C8A7F3DB4649D3E8DB5073E8D19CBBEB0
:10B510009DD23ABE0C1B75BCA975233E9556883E3C
:10B52000880F04BB8A828EBEAAD197BEC44DD0BC00
:10B53000FC58823D6229B7BDD5460ABE5AD1DEBE4F
:10B54000A83F99BE65E3F5BD629B8C3E55C812BE0F
:10B55000C5BBB33D7F9ECEBE2CDC8CBEDFA1103EB2
:10B56000EFA2153E7197F93D8C8C553EB5F3F3BEB5
:10B57000C76964BDC16CC53D55CE703E2E6C1FBD04
:10B58000F0E0033E768F57BE762755BD6E4BF03DFB
:10B59000CEF67F3EB77C0CBDFDF3D43D3368ADBE27
:10B5A00029BFC8BD9343CB3D1718133E556AF13DE3
:10B5B000B72F003EA16539BF8A2DB3BB19D2053E16
:10B5C00020654DBAD9AE10BE186D15BE5E1807BF06
:10B5D000BCABC73D6AF6BB3D49DDD53D47D9593CBB
:10B5E0008EB26CBEADC483BECA0F223E93E9B23D9B
:10B5F000F292D8BC4C5C8DBE55A086BD906ACCBE84
:10B60000D0EAEEBD769EBA3BB09AD73B6D59A3BE49
:10B61000D6F693BE7BCAB6BEB11639BDF80A2F3E28
:10B6200062BF26BE856E5DBE648F61BDE513E0BE60
:10B630002A4164BDA78F36BEEDEAFABC2BF60CBFDB
:10B640003E8F6CBEEB631DBF90E20F3EB212373DE2
:10B65000EA02A7BD3822F0BEA074D2BD5DE3D5BE1C
:10B660001816F7BD70B8C2BD444C25BE9FBF44BF7D
:10B67000164938BE5189C5BE248B90BEF053F5BC27
:10B680006925AABD3E4321BF696092BEC00111BFBA
:10B69000E4100BBECF29843C422A85BD57D22ABF75
:10B6A0003DE918BE47C90BBF9D65D2BD660D1B3E67
:10B6B0006744BEBD91E576BF0767F7BE2BE327BEA3
:10B6C00071618E3D9BD6623ECD0545BE2B2075BF78
:10B6D00051F987BEAA9E1EBE1E817B3E6D59443E17
:10B6E000C7568DBEEDEA54BFF7F5CBBE72CD0D3D0A
:10B6F00069D3223EBF3B86BDCDAE80BEC2AF82BF06
:10B70000B9B4F4BE11CA973D68D2283EB2F4353DB3
:10B7100045669ABE3295D2BE07BADFBE61A755BE56
:10B720000C38CABD75EA3C3C77720CBFE9CA483E8A
:10B730006F26ABBE5D88C33A315314BD86CD34BC91
:10B7400065C62CBD699A37BF846AB7BD315CA63D1A
:10B75000558B0DBD758339BEA7847BBC9BC121BFB2
:10B760002DC2F13C25AF783E98A02ABE5CA5863E4E
:10B77000186438BE5E1A90BEA0683B3C68F8AE3DC7
:10B780001ECE42BDBC997F3E8D1405BAADBD13BE21
:10B79000398277BDF1CABD3DB90188BE6281063FDD
:10B7A0004C319D3D59CAFABCAF75A73D9FE9C33DD9
:10B7B000204F14BE6EF01E3F5C4FBEBDBEB16CBCD0
:10B7C000BCCFD03B88336A3D156079BE33FA9D3ECD
:10B7D000DD9EA1BD49F28E3DA85B623EC7206E3E54
:10B7E00028513ABEC0EC313EE657BEBD29F8203D97
:10B7F0005F2375BE9D9CB83EC98C04BE82A50A3DE0
:10B80000CCC78C3D9F462D3D83D159BD3BB0A53E55
:10B8100044885EBD2B29673DAE92BCBDE3D398BE84
:10B820003CF21ABEEE62023F33A2A53D918994BC60
:10B83000B8E3F13D1434043E7C456BBE7777BA3DE6
:10B840003962453DC65EABBD5EE038BC9D2331BD6F
:10B8500047A792BE926B4EBE30DDF4BD61D53ABEB5
:10B86000B0B3143EE5FC1DBDCF7A7EBE83FB36BD72
:10B87000362CC6BB18A8F8BDC1E72FBEFCCBA73D30
:10B88000B472113E278A61BD29412E3E23DB95BE4D
:10B89000DD0626BE1A5AC7BC6B3F0B3EE594F1BDD0
:10B8A000ED2E803E1DC95BBEEBE056BDF511873C19
:10B8B000CFFF9E3E42BF283E18612A3EB9A342BE3A
:10B8C0003A035EBDF9C1C33DA0333B3EE0962F3E37
:10B8D000207BB43B625B6EBE3295633CA0E10DBE43
:10B8E000B2941F3E73633F3E0BD9C93D4CBAF3BDC2
:10B8F000A764B23DFDE3643D5EF8333DF5595B3E20
:10B900003509173E696B063D24FA9D3DB29D95BDF4
:10B91000332E873DAB5C3F3ED087053C5A77CDBC8C
:10B9200001BE32BD9AE5B6BEF8EE8B3EB0333B3D6C
:10B9300008F6433EC4D9FF3C2E00E03D7526F1BE1B
:10B94000E607633ED9168F3E601D86BB82186F3EA8
:10B95000980B74BD12F8C3BE3A4E6A3EDF42983E61
:10B9600089A2873E1451C63E4D585D3EA8DE84BE76
:10B97000DD69983E7127DC3E40D4183E21B2DC3DA3
:10B980003A3670BC21E7F9BE573B00BD5809543F19
:10B990000B39EFBD1774003D8EB3923E225FDA3E45
:10B9A000C32D723E50F742BE65F4A83DE7A89A3E0B
:10B9B00044AC3E3E93A23C3E963B9E3E961C12BE3D
:10B9C000901A7D3C25890B3ECC94B93E0E992C3EB5
:10B9D00078236D3EE80A363EA48ACE3DD4DC333E61
:10B9E00081392D3CB3925D3EA94B3D3E90A6343E3D
:10B9F0006CE9883D93DD993D643C783B2CB7233D51
:10BA0000CE57BF3D63B9CB3EFD284E3E9E2EE13B57
:10BA1000BD07D63D0E4A6FBD99513B3D1DDDF73D3B
:10BA2000CC3A6E3E3E1D493D2C0563BD6374DA3E43
:10BA3000BCBD63BC22EDF03CC736953C51B51ABE87
:10BA4000912576BD944E043FB44EA83D4EEB64BDA7
:10BA50006C867A3EF6D229BE2881313E057C7C3E3A
:10BA60002169923DECD828BE6AB4B83DDF36E8BD06
:10BA700092D36DBCD40CEC3ED2B0CA3E4AF6333DF4
:10BA800056EF233E3A9022BCD6AC73BB45CD443E24
:10BA9000B7596F3E20F8C8BE5482573D35DE343D5D
:10BAA0001E5CECBD2B1CA43E8D75D83C9232E7BDCC
:10BAB00059C8A13D0636E03D1CCABCBDE16FA83E99
:10BAC000D4B0B53E8979B6BE9DD3E93D3940493EF3
:10BAD0009A4C27BEE7B7DA3DB4F1F33E9FE7C0BE0C
:10BAE0007F09353E354BE03DD2E011BE92A82CBE19
:10BAF000DBE6883EC92FF6BE5D056A3E21CF3FBD1D
:10BB0000D35583BD0FC88ABEE436C03EA51D3BBFDA
:10BB10001D406D3DD010EEBD914414BE191EA3BD55
:10BB20006D7A063F28E162BF2DE885BB79FF11BE23
:10BB3000902BC7BD72E2C5BDFCF5EF3ECEC740BF3E
:10BB4000ADD9E2BDA9C211BD0C849F3D33D59BBECA
:10BB500005BCBB3EADDD65BF31F4ABBB7714923D98
:10BB6000C281C0BDF75CBDBE8896883EFB6A56BFE9
:10BB70001517073E38A1023E280581BE961054BE17
:10BB8000B8BF013F7C8F23BF1AF25A3E90165B3E2E
:10BB900074B7733D318029BE78293A3FF8B834BF75
:10BBA0001F4915BD4A757A3D2A5A57BE1C204D3D86
:10BBB000DA8D0F3F7BF650BFCC4F12BD70EE873D44
:10BBC00043A9343DD87483BE77B0563F722611BF67
:10BBD0003D3915BEDFFB2D3E497D5B3EA749573EF3
:10BBE0007FFB863F4A0276BF915D1C3E4313643E55
:10BBF00033E546BE117D9E3E44DBD4BEA55CC0BE8F
:10BC00003F1340BD692F853E85D415BEDFE78C3ECE
:10BC1000235CEDBE15F7B63B38754D3E620B1CBE7E
:10BC2000543B37BE3B19913E53991ABFE163E9BDBE
:10BC30009609B23D5655C3BD1B2333BE7917373D18
:10BC4000804FC7BE2EF24EBD831F2B3ED03E1FBE7F
:10BC500004147E3D956FBA3CCBA3DEBE8257193EDD
:10BC6000CFBE863E169BF3BD02B9BC3D3827C63C0D
:10BC700097225ABE0D2A1BBEE7813F3EDB35B33CFF
:10BC80001436CC3E346F97BE3DACC7BEA753843D3F
:10BC90002F9B763E85614D3E038BCC3E6B9F9BBEBA
:10BCA000C6F4C6BCB3B1073E50F5873ECFE9043EAB
:10BCB000874FC83E431EF6BD3EDCC7BDC82275BDDA
:10BCC000AFE6983E655D963D12CB323E12F609BE58
:10BCD0005ED70F3E5CD7423DFEA5403DFFC8A43D68
:10BCE0008B3F8ABCDB4659BE36A1F8BD9DF0C6BD70
:10BCF000D3C9833E12EC0EBE50DEABBD1222CDBCCA
:10BD00007A8936BE99C9B6BDF95EA63D232C4FBED1
:10BD1000B62F8FBDD378113D413489BD1E8477BDC8
:10BD20005868073E8CD294BD609D323EDD66B53CBE
:10BD3000F3D6CBBC73F50EBF7414BDBC052FF9BD93
:10BD4000FE324C3E19AC1ABE94FBBB3E10500BBFEA
:10BD50001B1B9CBD522D2B3EC7A9173E4475B1BE7F
:10BD60000AFA133EE51A76BD254CB5BD4F84E73D72
:10BD7000425A6E3DBC8F8DBE8C6172BD552BD13D3C
:10BD8000CE08063DD136973EE21AEEBCB621C1BDC3
:10BD90007DB5B8BDD0087CBEB2A822BEEA42B93E8D
:10BDA0005D3DEABDF7D4B2BE73D1ECBE1513CCBE77
:10BDB000DBF425BD38F52E3E6C1853BCC03557BE9C
:10BDC0008C349CBED88AF0BDAAE2CBBEFBD0823DAB
:10BDD0000FBBE5BD68BECEBE415B0ABF2225853ED6
:10BDE000529981BEAD14453EED4F54BE130517BFA9
:10BDF000148D04BF689C9D3E5340CCBE7904DE3E4A
:10BE0000A02590BE832A5EBF33F8B7BEE2E3B23E00
:10BE1000B69AC3BE64E2263F536A71BE75924FBFA5
:10BE200012BC97BE72D36D3F10A4A8BEEB824C3FEC
:10BE30003C3E81BE751797BFF11A45BE87AE963F4F
:10BE40004AFFFFFF0400000008000000FFFFFFFFA3
:10BE5000960000005EFFFFFF04000000800000006D
:10BE6000F763B4BF5472A2BD2D36A93F10902F4086
:10BE70000ED5353EA119903E349F3F3FB4D1E8BE68
:10BE80008445753E0BC91ABED728433E005724BED1
:10BE90006330293E047C00BEA82650BFBB52AFBE13
:10BEA0007D99973E759C9EBF846B86BE282403C0F7
:10BEB0006872083E3F94573D6815A7BFC61640BE3E
:10BEC0007650A3BD4B2962BE1B9B17BEF8E662BF2E
:10BED0006C847BC0C01F2DBF59B537C0090D46BE4D
:10BEE000EAFFFFFF040000000800000086BBB2BFAD
:10BEF000A52D933F00000600080004000600000086
:10BF000004000000800000003DB7B33F03A2C1BDA4
:10BF1000702CAF3EA2D112BF2172AE3EA062993FFB
:10BF2000C9EF3DBFEB2C52BF07B413BF800E42BF19
:10BF30009AA65ABD1E6F47BF3B8F87BF7C62D0BF9A
:10BF40002038D3BEB5F032BF7B19973FC13AD53EFA
:10BF500084734BBCE1F99C3E1B75303FC1DC34BFA0
:10BF600004863CBEADD544BEBAB067BF8E805F3F8D
:10BF70004BDC5DBF29F1353F3894CCBEC40C89BF82
:10BF8000D57F78BEAC082FBCBCF9FFFFC0F9FFFF1E
:10BF90000F0000004D4C495220436F6E766572745D
:10BFA00065642E00010000001400000000000E0077
:10BFB0001800140010000C00080004000E0000001F
:10BFC000140000001C0000004401000048010000B3
:10BFD0004C010000040000006D61696E000000006B
:10BFE0000500000008010000B80000006C0000001F
:10BFF000340000001000000000000A0010000C00D7
:10C00000080004000A0000000C00000010000000FE
:10C0100002000000010000000C0000000100000010
:10C020000B00000092FFFFFF14000000000000085A
:10C0300010000000140000000100000070FAFFFF73
:10C04000010000000B000000030000000A000000D7
:10C050000700000002000000C6FFFFFF1400000000
:10C06000000000081400000018000000010000009B
:10C07000B6FFFFFF00000001010000000A00000001
:10C08000030000000900000006000000030000009B
:10C0900000000E001A00140010000C000B00040039
:10C0A0000E0000001C000000000000081C00000042
:10C0B000200000000100000000000600080007004A
:10C0C000060000000000000101000000090000005F
:10C0D000030000000800000005000000010000004F
:10C0E00000000A000C000000080004000A00000024
:10C0F000080000000C000000010000000800000023
:10C100000200000000000000040000000100000028
:10C110000C00000001000000000000000D00000005
:10C120008004000018040000AC0300005803000065
:10C1300014030000B8020000700200002802000092
:10C14000D001000050010000CC00000060000000A1
:10C1500004000000CAFBFFFF000000011400000003
:10C160001C0000001C0000000D0000003400000056
:10C1700002000000FFFFFFFF02000000B0FBFFFF16
:10C1800019000000537461746566756C50617274B7
:10C190006974696F6E656443616C6C3A30000000CD
:10C1A00002000000010000000200000022FCFFFF6E
:10C1B00000000001140000001C0000001C00000032
:10C1C0000C0000004400000002000000FFFFFFFF21
:10C1D0000200000008FCFFFF2A0000006D6F64658C
:10C1E0006C2F64656E73655F322F4D61744D756C95
:10C1F0003B6D6F64656C2F64656E73655F322F42B3
:10C2000069617341646400000200000001000000E5
:10C21000020000008AFCFFFF000000011400000083
:10C220001C0000001C0000000B0000005C0000006F
:10C2300002000000FFFFFFFF2000000070FCFFFF76
:10C24000420000006D6F64656C2F64656E73655FFE
:10C25000312F4D61744D756C3B6D6F64656C2F6152
:10C26000637469766174696F6E5F312F52656C75A6
:10C270003B6D6F64656C2F64656E73655F312F4233
:10C280006961734164640000020000000100000065
:10C29000200000000AFDFFFF000000011400000064
:10C2A0001C0000001C0000000A00000058000000F4
:10C2B00002000000FFFFFFFF20000000F0FCFFFF76
:10C2C0003C0000006D6F64656C2F64656E73652FB4
:10C2D0004D61744D756C3B6D6F64656C2F6163745B
:10C2E00069766174696F6E2F52656C753B6D6F6412
:10C2F000656C2F64656E73652F4269617341646478
:10C30000000000000200000001000000200000000A
:10C3100086FDFFFF00000001140000001C0000006B
:10C320001C000000090000003000000002000000B6
:10C33000FFFFFFFF960000006CFDFFFF15000000EF
:10C340006D6F64656C2F666C617474656E2F5265D9
:10C3500073686170650000000200000001000000C9
:10C36000960000003EFEFFFF0000000110000000EC
:10C37000100000000800000024000000B0FDFFFFD6
:10C38000140000006D6F64656C2F64656E73655FEB
:10C39000322F4D61744D756C0000000002000000EA
:10C3A000020000002000000082FEFFFF00000001EC
:10C3B0001000000010000000070000002400000032
:10C3C000F4FDFFFF140000006D6F64656C2F646561
:10C3D0006E73655F312F4D61744D756C0000000008
:10C3E000020000002000000020000000C6FEFFFF49
:10C3F0000000000110000000100000000600000016
:10C400002000000038FEFFFF120000006D6F646521
:10C410006C2F64656E73652F4D61744D756C0000F3
:10C42000020000002000000096000000000016003E
:10C430001C001800170010000C000800000000008D
:10C4400000000700160000000000000114000000BA
:10C4500014000000050000000000000220000000A1
:10C4600094FEFFFF130000006D6F64656C2F666C17
:10C47000617474656E2F436F6E7374000100000069
:10C48000020000005EFFFFFF00000001100000003E
:10C49000100000000400000034000000D0FEFFFF88
:10C4A000240000006D6F64656C2F64656E73655FBA
:10C4B000312F426961734164642F52656164566132
:10C4C000726961626C654F7000000000010000003D
:10C4D00020000000AEFFFFFF000000011000000080
:10C4E00010000000030000003400000020FFFFFFE8
:10C4F000240000006D6F64656C2F64656E73655F6A
:10C50000322F426961734164642F526561645661E0
:10C51000726961626C654F700000000001000000EC
:10C5200002000000000016001800140000001000B7
:10C530000C000800000000000000070016000000CA
:10C5400000000001100000001000000002000000C8
:10C550003000000088FFFFFF220000006D6F64655F
:10C560006C2F64656E73652F426961734164642F3B
:10C57000526561645661726961626C654F7000005A
:10C580000100000020000000000016001C00180040
:10C590000000140010000C0000000000080007005C
:10C5A000160000000000000114000000240000003C
:10C5B00024000000010000003C0000000300000017
:10C5C000FFFFFFFF19000000060000000400040048
:10C5D000040000001900000073657276696E675FE1
:10C5E00064656661756C745F696E7075745F313A0D
:10C5F00030000000030000000100000019000000EE
:10C6000006000000030000003000000014000000DD
:10C6100004000000E8FFFFFF0E0000000000000E15
:10C62000F4FFFFFF09000000000000090C000C00EF
:10C630000B000000000004000C00000016000000C9
:10C640000000001681B000F5E0700268914203D34B
:10C6500043681A44914202D380680028F5D101B0A2
:10C660007047DFF86817086890B94FF48050486049
:10C670004FF480324FF0FF308A60C86008610420B8
:10C68000DFF84C27DFF84C374861C2F8BC010B607B
:10C690000120704701F1080313F0070F0EBF0023BC
:10C6A000C3F1080303F007031944D21A8161C26081
:10C6B00042F001034B60091D28238B50DFF80C1753
:10C6C0000A69C26170472DE9FC4B074601F1080079
:10C6D00010F0070F0FBF8946C0F1080000F00700F7
:10C6E00001EB000902F1080111F0070F06D002F179
:10C6F0000800C0F1080000F0070002441546A5EB51
:10C70000090009EB0306A0EB030B43F00303C9F890
:10C710000430AE4228BF01F0FFF92879C10758BFA5
:10C7200001F0FAF9BBF1100F38BF01F0F5F9B86963
:10C73000854207D1F8685844F860BE6140F00100B6
:10C74000706050E1786985420AD1B8688344C7F8BF
:10C7500008B07E614BF00100706046F80BB042E11A
:10C76000686800F00301012940F0AB80C008C000F8
:10C770000190C0081F2839D8AC68D5F80C8000900B
:10C78000454508BF01F0C8F9A54208BF01F0C4F94A
:10C7900068680099C008C000B0EBC10F18BF01F075
:10C7A000BBF9009907F1280000EBC100844206D0D4
:10C7B0003A699442C0F08080E168A9427CD1A045EA
:10C7C00006D100983968012282409143396075E0B2
:10C7D000804506D0386980456ED3D8F80800A84255
:10C7E0006AD1C4F80C80C8F8084067E0EC68D5F856
:10C7F0001880AC420CD0A8683969884222D3C1683D
:10C80000A94204BFA168A9421CD1C460A0601BE07A
:10C8100005F11402146834B905F1100214689CB1D2
:10C8200001E01A46146804F114031968002902BFD4
:10C8300004F1100318680028F3D139698A4228BF2F
:10C84000106001D201F068F9B8F1000F36D0E96943
:10C8500007F5987000EB81000268954208D10460EA
:10C86000A4B9E8697968012282409143796025E0A2
:10C870003869804508D3D8F81000A84214BFC8F81A
:10C880001440C8F8104001E001F046F9B4B139692C
:10C890008C4211D3C4F81880286928B1884226BF79
:10C8A0002061846101F038F9686938B139698842DA
:10C8B00002D36061846101E001F02EF901982D1826
:10C8C000834468684008400068604BF00101716073
:10C8D0004FEADB0446F80BB01F2C23D807F12800E1
:10C8E00000EBC4084546BBF1100F38BF01F014F946
:10C8F000386820FA04F1C90705D4012101FA04F4CB
:10C9000004433C6007E0D8F80800396988422CBF2E
:10C91000054601F001F9C8F80860EE60B560C6F898
:10C920000C8060E05FEA1B2008BF002123D0B0F537
:10C93000803F28BF1F211ED2A0F58072120C02F08A
:10C9400008029040A0F58051090C01F004018840D4
:10C95000A0F580431B0CC2F10E0203F00203521A31
:10C96000D21A984002EBD032D01D2BFA00F101F020
:10C97000010101EB420107F5987202EB8100F161C0
:10C980000022726132617A6822FA01F3DB0707D470
:10C99000012303FA01F1114379600660B0611DE0E3
:10C9A00002681F291DBF4908C1F119010BFA01F1E5
:10C9B000594600E002465068C008C000584516D0ED
:10C9C00002F11003CC0F03EB840349001868002820
:10C9D000F0D13869834204D31E60B261F660B6605C
:10C9E00001E001F099F809F10800BDE8F68B39691A
:10C9F00090688A4228BF8842F3D3C6609660B060D0
:10CA0000F2600020B061EEE72DE9FE4F04468B4650
:10CA1000A5692E46904699463146FFF713FEA8F1C8
:10CA200028020168406801EB000AAAF1270111F011
:10CA300007000EBF0021C1F1080101F007010AEB58
:10CA40000100A0F12F0706F11000874238BF3746DA
:10CA500007F1180001905946002000902046FFF78A
:10CA600019FE07F1080010F0070F18BF01F054F885
:10CA70001B20786007F1080104F5E07090E80C5085
:10CA800081E80C50C0F800B0C0F80480C0F80C90E9
:10CA900081600198009900E0001D07224260491C56
:10CAA00000F108025245F7D30129D8BF01F034F84C
:10CAB000B74200F09580BF1B301D311DC0594008A2
:10CAC0004000C85147F0010171604FEAD70BF751A0
:10CAD000BBF11F0F21D804EBCB0000F12805A846BD
:10CAE000102F38BF01F018F8206820FA0BF1C907A1
:10CAF00005D4012101FA0BF10843206006E0A86883
:10CB0000216988422CBF804601F006F8AE60C8F863
:10CB10000C60C6F80880F5606FE0380A08BF002195
:10CB200023D0B0F5803F28BF1F211ED2A0F5807210
:10CB3000120C02F008029040A0F58051090C01F09F
:10CB400004018840A0F580431B0CC2F10E0203F0E3
:10CB50000203521AD21A984002EBD032D01D27FAA3
:10CB600000F101F0010101EB420104EB810200231D
:10CB700002F59870F16173613361626822FA01F322
:10CB8000DB0707D4012303FA01F11143616006605A
:10CB9000B0611DE002681F291DBF4908C1F11901DC
:10CBA00007FA01F1394600E002465068C008C000AB
:10CBB000B84216D002F11003C80F03EB80034900FE
:10CBC00018680028F0D12069834204D31E60B26146
:10CBD000F660B56011E003B0BDE8F04F00F09CBF17
:10CBE0000BE0216990688A4228BF8842F3D3C6606F
:10CBF0009560B060F2600020B06103B0BDE8F08FD6
:10CC00002DE9F041714F05463868884608B9FFF7AD
:10CC100028FDB96801EB08002F30491E20EA010108
:10CC200088457DD205F5D876B06828B13268891874
:10CC30008A4275D2884273D300F0AEFF01001CBF58
:10CC40000C6811F1010F6BD03068201805F5D8720F
:10CC500030605368984238BF18467060A86960BB5E
:10CC6000286908B1814200D22961316174610020D4
:10CC7000F06105F12802386868624FF0FF302862E1
:10CC80000020D260926002F1080353611361801C9E
:10CC900010322028F5D34E48854208BFA4F128025F
:10CCA00028D055F8040CC00805EBC002A2F108001A
:10CCB0000A19121A283A01461CE005F5E0700246EE
:10CCC00000E092687AB3136857683B449942F8D100
:10CCD000137B1F0727D4AB691768BB4223D3D2F855
:10CCE00004C06744BB421ED2A444C2F804C0E86832
:10CCF000A96922182846FFF7CDFC1FE08068C0B163
:10CD000003689342FAD1027B130712D402680160D0
:10CD10004368E418446043462846BDE8F041D2E445
:10CD20000020BDE8F0812A69914238BF29610A19C3
:10CD3000E5E7002322462846FFF766FEE8688045BF
:10CD4000EED2A0EB0800A969E86001EB0802AA6135
:10CD500040F00100506048F00300486001F1080015
:10CD6000BDE8F08138B4194B1A6882B94FF480528B
:10CD70005A604FF480344FF0FF329C60DA601A61E1
:10CD80000422134C134D5A61C4F8BC211D6011F1EB
:10CD9000400F17D28269AAB1C368283199420BD2D9
:10CDA00000F5E0710C68A24203D34D682C44A24206
:10CDB00002D389680029F5D1C16999423CBF4FF07F
:10CDC000FF31C16132BC002070470000684700207D
:10CDD000704400206859883C2DE9F84F00258946A9
:10CDE000090AC9F1000B08BF002323D0B1F5803F29
:10CDF00028BF1F231ED2A1F58072120C02F0080278
:10CE00009140A1F580531B0C03F004039940A1F558
:10CE10008044240CC2F10E0204F00204D21A121B48
:10CE2000A14002EBD132D11D29FA01F303F0010335
:10CE300003EB4203074607F5987858F8230030B310
:10CE40001F2B0FBF4C465C08C4F1190409FA04F407
:10CE5000AC46594600E064004268D208D200A2EB1A
:10CE600009028A4203D21100054600F06881426936
:10CE700010304FEAD47B50F82B00002A1CBF8242AE
:10CE800094460028E7D18B466046B0BBBDBB01206D
:10CE900000FA03F35B00584203437868034000F054
:10CEA0004D81584203405B1E180B00F01000C34038
:10CEB000590901F00801CB409A0802F00402D3405E
:10CEC0005C0804F002040818E3401018C3F340069D
:10CED00020183044F3401B1858F823000DE0084692
:10CEE0004168C908C900A1EB090159453CBF8B46FF
:10CEF000054601690029F2D140690028F0D1002DD2
:10CF000000F01C81B868A0EB0900834580F0168111
:10CF100038698542C0F010816868C008C00009EB1C
:10CF20000B01884218BF00F0F7FD05EB0906B5427A
:10CF300080F00281EC68D5F818A0AC420CD0A8684B
:10CF40003969884222D3C168A94204BFA168A942B5
:10CF50001CD1C460A0601BE005F11402146834B950
:10CF600005F1100214689CB101E01A46146804F13E
:10CF700014031968002902BF04F11003186800287F
:10CF8000F3D139698A4228BF106001D200F0C4FD94
:10CF9000BAF1000F36D0E96908EB810002689542CA
:10CFA00009D10460200014D1E86979680122824027
:10CFB0009143796026E03869824508D3DAF8100099
:10CFC000A84214BFCAF81440CAF8104001E000F0AB
:10CFD000A3FDBCB13869844212D3C4F818A02869F3
:10CFE00030B13969884226BF2061846100F094FD28
:10CFF000686938B13969884202D36061846101E0AF
:10D0000000F08AFDBBF1100F0CD2D94449F00300A7
:10D010006860291D281D50F8090040F0010041F802
:10D02000090088E049F0030068604BF0010070607F
:10D030004FEADB0046F80BB01F281DD807EBC001F4
:10D0400001F12804396821FA00F2D207A34605D479
:10D05000012202FA00F00843386006E0A06839694E
:10D0600088422CBF834600F057FDA660CBF80C60C9
:10D07000C6F808B0F4605EE05FEA1B2008BF00213C
:10D0800023D0B0F5803F28BF1F211ED2A0F58072AB
:10D09000120C02F008029040A0F58051090C01F03A
:10D0A00004018840A0F580431B0CC2F10E0203F07E
:10D0B0000203521AD21A984002EBD032D01D2BFA3A
:10D0C00000F101F0010101EB4201F1610022726106
:10D0D000326108EB81007A6822FA01F3DB0707D49A
:10D0E000012303FA01F1114379600660B0611DE08C
:10D0F00002681F291DBF4908C1F119010BFA01F18E
:10D10000594600E002465068C008C000584518D093
:10D1100002F11003CC0F03EB8403490018680028C8
:10D12000F0D13869834204D31E60B261F660B66004
:10D1300001E000F0F1FC13E100F0EEFC0DE18B46A4
:10D14000A3E6396990688A4228BF8842F1D3C66055
:10D150009660B060F2600020B061ECE72DE9F84F16
:10D1600006468846716848420140491E080B00F097
:10D170001000C1404A0902F00802D1408B0803F0B8
:10D180000403D9404D0805F002051018E9401818AD
:10D19000C1F34004281806F5987A2044E1400918A4
:10D1A0005AF821104868C008C0000D46A0EB0809D5
:10D1B00009E001464868C008C000A0EB08004845E7
:10D1C0003CBF81460D4608690028F2D14969002913
:10D1D000F0D130698542C0F0BE806868C00808EBB5
:10D1E000090BC000584518BF00F096FC05EB08007D
:10D1F0008542009080F0AF80EF68AC69AF420CD000
:10D20000A8683169884222D3C168A94204BFB968BD
:10D21000A9421CD1C760B8601BE005F11402176871
:10D2200037B905F1100217689FB101E01A46176877
:10D2300007F114031968002902BF07F110031868E9
:10D240000028F3D131698A4228BF106001D200F072
:10D2500063FC002C31D0E9690AEB81000268954239
:10D2600008D107608FB9E869716801228240914353
:10D27000716022E03069844205D32069A84214BF5E
:10D280006761276101E000F047FCB7B13069874270
:10D2900011D3BC61286930B13169884226BF386139
:10D2A000876100F039FC686938B13169884202D37E
:10D2B0007861876101E000F02FFCB9F1100F0BD20B
:10D2C0004BF003006860291D281D50F80B0040F04A
:10D2D000010041F80B003DE048F00301696049F0AE
:10D2E0000100291D41F80800009840F80990D6F87F
:10D2F00008804FEAD80BBBF1200F28BF00F00CFCD0
:10D30000B8F1000F22D006EBCB00776900F12804BA
:10D31000A246B8F1100F38BF00F0FEFB306820FACB
:10D320000BF1C90705D4012101FA0BF10843306064
:10D3300006E0A068316988422CBF824600F0ECFB11
:10D34000A760CAF80C70C7F808A0FC60C6F808907F
:10D350000098706104E000F0DFFB0020BDE8F28F70
:10D3600005F10800BDE8F28F2DE9FE4F0546AFF349
:10D370000080F52DDFF89C6780F004810B2D31BF14
:10D3800010250B35ED08ED003068EC08E04010F09A
:10D39000030F46D0C04300F00100041906F1280035
:10D3A00000EBC408E700D8F808506868C008C0005F
:10D3B000B84218BF00F0B0FBD5F80890454508BF4B
:10D3C00000F0AAFB4D4508BF00F0A6FB6868C00846
:10D3D000C000B84218BF00F09FFBC84507D13168B4
:10D3E000012000FA04F421EA040434600DE03069FD
:10D3F000814508D3D9F80C00A84204D1C8F8089098
:10D40000C9F80C8001E000F087FB47F0030068607A
:10D41000291D281D05F10804C05940F00100C8511C
:10D42000F8E0B168A94280F0BE80002800F0A18039
:10D430004FF0010808FA04F1490000FA04F44842E8
:10D4400001430C4060420440641E200B00F01000B9
:10D45000C440610901F00801CC40A20802F00402B6
:10D46000D440630803F002030818DC401018C4F32A
:10D47000400718183818FC40241806F1280000EB63
:10D48000C40AE700DAF80890D9F80400C008C00020
:10D49000B84218BF00F040FBD9F808B0D14508BF2A
:10D4A00000F03AFBD94508BF00F036FBD9F804007C
:10D4B000C008C000B84218BF00F02EFBDA4506D104
:10D4C000316808FA04F421EA040434600DE030699C
:10D4D000834508D3DBF80C00484504D1CAF808B0EE
:10D4E000CBF80CA001E000F017FB45F00300C9F8F1
:10D4F00004007F1B09F1040147F00100485109EBCA
:10D5000005000190C751B4684FEAD40ABAF1200F60
:10D5100028BF00F001FB34B3CDF800A006F12800CD
:10D52000756900EBCA0AD346102C38BF00F0F4FA34
:10D530003168009821FA00F2D30704D408FA00F009
:10D540000843306007E0DAF80800316988422CBFF0
:10D55000834600F0E1FACAF80850CBF80C50C5F841
:10D5600008B0C5F80CA0B76009F108040198706113
:10D5700050E07068C0B329463046FFF7EFFD040065
:10D5800011D047E015F1400F28BF4FF0FF350AD208
:10D590000B35ED087068ED0028B129463046FFF7DD
:10D5A0001BFC040036D1B068A8421DD3411B726930
:10D5B00010290AD350197061B16041F00103436032
:10D5C000415045F0030555600BE00021B1607161E9
:10D5D000131D40F003015160111D095841F0010174
:10D5E000195002F1080415E0F06885420DD2401B85
:10D5F000B169F0604A19B26140F00100506045F035
:10D6000003054D6001F1080404E029463046FFF7A8
:10D61000F7FA0446AFF300802046FFF7EEBA002881
:10D6200000D170472DE9FC47A0F10805AFF3008059
:10D63000DFF8E06432699542C0F05982686800F012
:10D640000301012900F05382C1084FEAC109C10753
:10D6500005EB090839D42C6810F0030F00F049825B
:10D66000604205449542A144C0F041827069854200
:10D6700000F0C780E408202C5ED2D5F80CA0AF687B
:10D68000554508BF00F048FABD4208BF00F044FA13
:10D690006868C008C000B0EBC40F18BF00F03CFAC7
:10D6A00006F1280000EBC400874205D031698F42A3
:10D6B0003FD3F968A9423CD1BA452CD13068012149
:10D6C00001FA04F420EA04043460454580F00F8236
:10D6D000D8F80440E00740F10A82A00700F1688111
:10D6E000B069804540F0A080F068B5618144C6F81B
:10D6F0000C9049F0010068607069854202D10020F9
:10D700007061B060F069484580F0F38100213046D7
:10D71000FFF728FBEDE1824506D03069824508D34A
:10D72000DAF80800A84204D1C7F80CA0CAF80870BB
:10D73000CBE700F0F1F9C8E7EC68AF69AC420BD079
:10D74000A868904223D3C168A94204BFA168A94236
:10D750001DD1C460A0601CE005F114031C6834B93D
:10D7600005F110031C68A4B101E063461C6804F1D4
:10D77000140CDCF80010002902BF04F1100CDCF8D6
:10D7800000000028F1D1934228BF196001D200F0B7
:10D79000C3F9002F99D0E96906F5987000EB810074
:10D7A0000268954209D10460200011D1E8697168CE
:10D7B000012282409143716087E73069874205D337
:10D7C0003869A84214BF7C613C6101E000F0A4F913
:10D7D000002C3FF47AAF31698C42AAD3A761286943
:10D7E00028B1884226BF2061846100F095F96869FC
:10D7F00000283FF46AAF316988429AD3606184613E
:10D8000063E798F8040000F0030003287FF45DAF9D
:10D81000C6F8089049F00101D8F80400400840001B
:10D82000C8F8040069600AE0706980450AD1B068F0
:10D8300075618144C6F8089049F00100686045F8B8
:10D84000099056E1E408E400A144E408202C3AD20F
:10D85000D8F80CA0D8F80870D04508BF00F05CF9E3
:10D86000B84508BF00F058F9D8F80400C008C00057
:10D87000B0EBC40F18BF00F04FF906F1280000EB21
:10D88000C400874207D031698F42C0F08480F968B4
:10D89000414540F08080BA4507D13068012101FA46
:10D8A00004F420EA0404346077E0824506D031694C
:10D8B0008A4570D3DAF8080040456CD1C7F80CA04F
:10D8C000CAF8087069E0D8F80C40D8F818704445D8
:10D8D0000DD0D8F808003169884222D3C16841458B
:10D8E00004BFA16841451CD1C460A0601BE008F1E1
:10D8F0001402146834B908F1100214689CB101E0F4
:10D900001A46146804F114031968002902BF04F1CF
:10D91000100318680028F3D131698A4228BF1060CB
:10D9200001D200F0F9F8002F37D0D8F81C1006F516
:10D93000987000EB8100026890450AD104602000D5
:10D9400012D1D8F81C0071680122824091437160A5
:10D9500023E03069874205D33869404514BF7C61B4
:10D960003C6101E000F0D8F8BCB131698C4212D3BF
:10D97000A761D8F8100028B1884226BF20618461D1
:10D9800000F0CAF8D8F8140038B13169884202D3DF
:10D990006061846101E000F0BFF849F00100686057
:10D9A00045F80990706985420BD1C6F80890A0E04F
:10D9B00064086400C8F8044049F00100686045F854
:10D9C00009904FEAD907202F22D206F1280000EB58
:10D9D000C704A046B9F1100F38BF00F09DF83068B9
:10D9E00020FA07F1C90705D4012101FA07F7074317
:10D9F000376006E0A068316988422CBF804600F09D
:10DA00008BF8A560C8F80C50C5F80880EC6070E091
:10DA10005FEA192008BF002123D0B0F5803F28BF5E
:10DA20001F211ED2A0F58072120C02F00802904055
:10DA3000A0F58051090C01F004018840A0F5804355
:10DA40001B0CC2F10E0203F00203521AD21A9840C4
:10DA500002EBD032D01D29FA00F101F0010101EBF7
:10DA6000420106F5987202EB810000226A612A6188
:10DA7000E961726822FA01F3DB0707D4012303FA94
:10DA800001F1114371600560A8611DE002681F2962
:10DA90001DBF4908C1F1190109FA01F1494600E029
:10DAA00002465068C008C000484526D002F1100365
:10DAB000CC0F03EB8403490018680028F0D13069CB
:10DAC000834204D31D60AA61ED60AD6001E000F007
:10DAD00023F8306A401E30620BD1D6F8C80100E04E
:10DAE00080680028FCD14FF0FF30306201E000F088
:10DAF00013F8AFF30080BDE8F387316990688A427C
:10DB000028BF8842E3D3C5609560A860EA60002022
:10DB1000A861DEE770440020012000F053B8F0B4A3
:10DB20000246106895681318506803EB5004C0074C
:10DB300021D54D441FE0F0BC02F10C00704713F8F2
:10DB4000017B05F8017B491EF9D1A0B1B60813F895
:10DB5000011B06F00306032E08BF13F8016B01EB4F
:10DB600006214942801C294405D011F8016B05F8B3
:10DB7000016B401EF9D1A342DDD013F8016B16F002
:10DB8000030104BF13F8011BC91C30090F28DAD1A7
:10DB900013F8010B0F30D6E70749086808B10020D9
:10DBA00070470648C008C00008600549C908C90098
:10DBB000091A0160704700BF90470020A767002046
:10DBC000A087002080B500F007F8024A1100182055
:10DBD000ABBEFBE72600020010B500F052F80200D1
:10DBE0000023DB4300241068984203D01100022078
:10DBF000ABBE14605068984203D0111D0220ABBE2A
:10DC0000546010BDF0B583B0040000F03AF8A100F4
:10DC100047183D680026F643B54216D100F01AF8C1
:10DC20003D68B5420FD100BF09A00090002C01D182
:10DC3000002000E0042001900320029069460120AA
:10DC4000ABBE05003D6000F014F8280003B0F0BD45
:10DC50003A7474000C480121BFF35F8FD0E84F3F46
:10DC6000C0E8421F002AF9D1BFF35F8F002BF3D128
:10DC700070470548BFF35F8F00210170BFF35F8FCE
:10DC8000704702487047000098470020202C002071
:10DC90002DE9F0439FB000BF66A6269CDFF8E48A1A
:10DCA00002918DF83B4000210B914FF0FF37044665
:10DCB00091461D460AE019F8011B0298A04700286A
:10DCC000029000F0A4800B98401C0B9099F8000083
:10DCD00050B12528EFD10020002105900691079032
:10DCE000089109900A9103E00B98A7E041F0010127
:10DCF00019F8010F2028F9D023280CD02B2804D0A4
:10DD00002D2805D0302809D083E041F00201EFE74B
:10DD100041F00401ECE741F00801E9E741F01001AE
:10DD2000E6E700200D900AE00D98404505DA00EB8B
:10DD3000800302EB4302303A0D9209F1010999F890
:10DD40000020A2F130000A28EED399F800002E2816
:10DD500018BF0C9726D119F8010F2A2808D1286876
:10DD6000286009F1010950F8042B28600C9219E091
:10DD70002D280CBF19F8010B002000220C920BE09B
:10DD800040B90C9A424505DA02EB820203EB4203EA
:10DD9000303B0C9309F1010999F80030A3F13002EE
:10DDA0000A2AEDD3ADF83810304699F8001000F08B
:10DDB00093FE08B119F8010B8DF83A009DF83A006E
:10DDC000682804BF99F80010682903D162208DF8F3
:10DDD0003A0008E06C2804BF99F800006C2804D1D0
:10DDE00071218DF83A1009F1010910A804902A4612
:10DDF00019F8013B6946204600F060F838B910AACE
:10DE00006946204600F08CF900287FF55FAF384660
:10DE100014E02A2885D12A682A6052F8040B2A6067
:10DE200000280D9003D540420D9041F0040109F106
:10DE300001098AE7686A6C747A4C00001FB0BDE87B
:10DE4000F083622820D0682811D06A2803D06C287B
:10DE500027D0712825D10868C01D20F00700086070
:10DE6000D0E9002308300860194610467047002AA0
:10DE70000A680A60106803D0121D0A6000B217E039
:10DE8000121D0A6080B217E0002A0A680A60106852
:10DE900003D0121D0A6040B20AE0121D0A60C0B22F
:10DEA0000AE0002A0A680A60106803D0121D0A609E
:10DEB000C1177047121D0A600021704770B51C46DB
:10DEC0000D46B4F125002E69114600F017811C386B
:10DED0006AD0001F022867D9133843D0093863D0AD
:10DEE000801E16D0401E1ED0401E02285CD9001F86
:10DEF00019D0401F00F08380401E33D0401E00F038
:10DF0000CD80C01E00F0D880801E2BD0C01E29D02E
:10DF1000FAE06869421C6A610A680A6052F8043BC8
:10DF20000A603354FAE095F83A000122FFF789FFBE
:10DF3000C5E900010023994204DA6869411C69615E
:10DF40002D210DE0288F810704D56869411C696186
:10DF50002B2105E0C00722D56869411C6961202199
:10DF600031541CE095F83A000022FFF76AFFC5E93A
:10DF7000000195F83800010711D5D5E900230020EC
:10DF8000834208BF82420AD044F02000782806D19C
:10DF9000686930213154401C411C69613454214668
:10DFA00068693044E86083E00868C01D20F007001D
:10DFB0000860D0E9002308300860C5E90023D5E9EE
:10DFC0000001C80F04D06869411C69612D210DE072
:10DFD000288F810704D56869411C69612B2105E000
:10DFE000C00704D56869411C696120213154686902
:10DFF0003044E8602146284600F0C4F98EE005F17F
:10E000003A02507820B14FF0FF340FF648205EE01E
:10E010001078622808D0682824D06A2812D06C288A
:10E020002ED071280ED02BE00A680A6052F8040B3B
:10E030000A6020B94FF0FF340FF6302047E0E96A5C
:10E0400001706BE00A680A6052F8040B0A6020B99C
:10E050004FF0FF340FF6142039E0EA6AD317C0E915
:10E0600000235BE00A680A6052F8040B0A6020B9DA
:10E070004FF0FF340FF6F41029E0E96A01804DE01B
:10E080000A680A6052F8040B0A6020B94FF0FF34A6
:10E090000FF6D8101BE0E96A01603FE00A680A60E9
:10E0A00052F8040B0A600021C5E90001EE607821F6
:10E0B000284600F0BBF831E00868086050F8044BCF
:10E0C0000860EC603CB94FF0FF340FF6B81000F078
:10E0D0000FFD201A70BD2E6B002E04D5204600F0D7
:10E0E00027FD044608E032460021204600F03CFDB2
:10E0F000002814BF041B3446AC610FE06869411C62
:10E1000069612521315409E06969481C686125224B
:10E110007254210002D0411C69613454002070BD4A
:10E120002DE9FC410F460646796B7869BC6A091AED
:10E13000386A091AB869091A786A091AF869091A4D
:10E1400097F838000C1B410790460FD42021002C73
:10E150008DF800100ADD254601236A46394630460F
:10E1600000F060FC00285DD16D1EF5D17B69424650
:10E170003946304600F056FC002853D130208DF847
:10E1800000003D6A002D09DD01236A46394630460C
:10E1900000F048FC002845D16D1EF5D1BB69FA6836
:10E1A0003946304600F03EFC00283BD130208DF847
:10E1B00000007D6A002D08DD01236A46394630469D
:10E1C00000F030FC70BB6D1EF6D1F868B969FB69D0
:10E1D00042183946304600F025FC18BB30208DF837
:10E1E0000000BD6A002D08DD01236A46394630462D
:10E1F00000F018FCB0B96D1EF6D197F83800410751
:10E200000DD52021002C8DF8001008DD01236A4671
:10E210003946304600F006FC20B9641EF6D10020D5
:10E22000BDE8F6814FF0FF30BDE8F6812DE9FC47EF
:10E2300007468A463E69BAF16F0F08BF082405D029
:10E240004AF02001782914BF0A2410243C25D7E97C
:10E250000023BAF1640F18BFBAF1690F90469946CE
:10E2600006D100218B4203DAD8F1000869EB490995
:10E270000020814508BF80451FD1386BE8B9082CC4
:10E280004CD197F83800010748D530203B2586F857
:10E290003B0043E000280ED597F8380000F014004A
:10E2A000102808D17A6B7869121A386A121A511A32
:10E2B0000029C8BF3962BDE8F3878DF800A0404649
:10E2C00049462246E31700F09DFC3032D0B26D1E65
:10E2D0003A28019504DB9DF80000A0F151018A184D
:10E2E0007255404649462246E31700F08BFC8046B3
:10E2F00089460020814508BF804503D0F868711920
:10E300008842DCD3082C09D197F83800010705D5DD
:10E31000715D302902D06D1E30207055C5F13C0171
:10E32000B9617019F860386B8142B3DA411A396209
:10E330004FF6EF70398F01403987BDE8F3872DE93B
:10E34000D04306460F4614464FF00008DFF83894D5
:10E3500012E0E00707D542464B463046394600F00A
:10E3600069FD06460F464046494642464B4600F088
:10E3700061FD641080468946002CEAD1304639465A
:10E38000BDE8D0832DE9F34F054641F020048DB060
:10E39000D5E90089612C02AE09D0286B002848BF5E
:10E3A000062003D408BF672C01D101202863D5E9DA
:10E3B000002358004015401C0ED119030CD0032037
:10E3C000A8619DF8380061381A2802D20FF2D06196
:10E3D00011E00FF2D0610EE058004015401C0FD143
:10E3E00019030DD10320A8619DF8380061381A285F
:10E3F00014D30FF2B861E868032200F0EDFDD3E119
:10E40000194621F00043B3F5801F10460DD20027B6
:10E41000BB4208BFBA42019703D111E00FF28861F5
:10E42000E9E701AA00F020FE0AE0DFF8607307EBDD
:10E430001352DFF85C3301921940DFF85833194367
:10E44000C5E90001612C0ED1E86830210170811C02
:10E45000E9609DF8381061290CBF7821582141707E
:10E460006869801C6861D5E900AB2BF0004300208F
:10E470002AF00002834204BF8242002300F05A8146
:10E48000612C40F0A980286B00284CBF2120401C43
:10E4900000904046009F7F1C49460022002300F068
:10E4A0001BFED94601988DF8082038BF89F0004935
:10E4B000001F0190002FD0460DF1090040F3498163
:10E4C00040F2FF71DFF8D0B20C9106464046494653
:10E4D0000022002300F018FE80F03A814800400D31
:10E4E00000F11C0210D0002A0EDD0C98824205DBE0
:10E4F00009F0004040EA0B01002013E0A448084066
:10E5000040EA025140460DE029F00043002028F087
:10E510000002834208BF82420FBF40461C22404691
:10E5200000F00AFE8046894600F0A4FEFF1F002F7F
:10E53000044609DD00F0BCFE02460B464046494653
:10E5400000F0C8FE80468946F01D072104E004F073
:10E550000F0200F8012D2411002C01DD491EF6D513
:10E56000491E5CBF002200F8012DF9D5ECE0002027
:10E57000194602AA0A4400E05B1E12F80149491E2E
:10E580008442F9D00F2804D10DF10900425C521CDD
:10E590004254002904D50198001D02AE5B1C019075
:10E5A000591E12D49DF838007218147804F13008FE
:10E5B0005FFA88F4392CC4BFA0F13A04A044491E84
:10E5C00002F80189F1D58DF83800286B002840F158
:10E5D000B080591E2963ACE0404649460022002322
:10E5E00000F07AFD019938BF89F0004947F2975051
:10E5F00041436A4A91FBF2F20192D2F1070204DD33
:10E6000040464946FFF79BFE0AE05242002064491B
:10E61000FFF795FE02460B464046494600F0CCFE09
:10E620008046662C286BDFF87CB106BF019F0A3755
:10E6300006273F18142FC8BF142730208DF8080074
:10E6400089460DF1090000E03046002F34DD064612
:10E650004046494600F0D4FF01460A4606F1080349
:10E6600004200A26B2FBF6F606EB860EA2EB4E025B
:10E67000303203F8012C0A22B6FBF2F202EB820ED2
:10E68000A6EB4E063036401E03F8026DE9D1083F76
:10E69000002F03F10806D7DD084600F0C5FF02464B
:10E6A0000B464046494600F015FE00225B4600F04E
:10E6B000C1FB80468946CBE70DF10901401A0DF1F7
:10E6C000090604E00199491E401E0191761C31782B
:10E6D0003029F7D0662C02D10199491C03E0652C42
:10E6E0000CBF012100212B6BCB189842B8BF431EF1
:10E6F000002B1ED4834204DAF05C3528A8BF3920F1
:10E7000000DA30201946721E02EB010800E05B1EA1
:10E7100018F80199491E8145F9D0392802D1705C59
:10E72000401C7054002904D50198401C16465B1CFF
:10E730000190019800B200901BB29DF8381032464B
:10E74000284600F035F82FE0C61D002F3FF7BEAE7B
:10E7500030460DF10901401A009903468842C8BFAE
:10E760000B46002B0DF109063FF52FAF8342BFF694
:10E77000FEAE0DF10900C05C07287FF7F8AE0F2050
:10E78000F6E60000CBCCCC0C0000244002FCFFFFDE
:10E79000FFFF0F800000E03F0000F07FA086010037
:10E7A0000000F03F84D797410FB0BDE8F08F000024
:10E7B0002DE9F84783B006468A461746984600F08A
:10E7C00041FFB8F1000F406A356B90F8009002DC11
:10E7D0004FF00108B6A7BDF930404AF02000662886
:10E7E00008BF641C15D0672840F0848014F1040F22
:10E7F000C0F28680AC4280F2838096F83800641CB8
:10E80000010702D4A845B8BF454620B22D1A48BF1B
:10E8100000250FFA84FAF068B169BAF1000F25DC1F
:10E820004A1C30234354002D03DC96F838000107BE
:10E8300003D5F06800F80290521C15EB0A0FB8BF20
:10E840006C4220B2441941424445B8BFA046B2616F
:10E8500071620FFA88F5F561F068B3692A463946A6
:10E86000184400F0B9FB641BB462C4E022B29045C6
:10E87000084417DA4246394600F0AEFBB06940441E
:10E88000B061AAEB0801002D716203DC96F8381024
:10E890000A0705D5F16801F80090F069401CF061A5
:10E8A000B562A8E0394600F097FBB069002D5044EE
:10E8B000A8EB040803DC96F838100A0703D5F168C2
:10E8C00001F80090401CB0610FFA88F08542F068B2
:10E8D000B369B8BFA8460FFA88F207EB0A011844DB
:10E8E00000F07AFBB0690FFA88F10844B061681A49
:10E8F000706280E0BAF1610F14D14FF0700A16E037
:10E90000A84504DA96F838100A0758BF45466D1E28
:10E9100048BF0025BAF1670F14BF4FF0450A4FF00A
:10E92000650A04E0BAF1410F08BF4FF0500AB1691F
:10E93000F368481CB061002D17F8012B5A5403DC12
:10E9400096F838100A071BD5F168431CB36101F82B
:10E950000090002D14DDA8F101080FFA88F085421F
:10E96000F068B8BFA8460FFA88F23946184400F09C
:10E9700033FBB0690FFA88F108446D1AB061756213
:10E98000F068B1690844002C80F800A003D42B2162
:10E990004170811C03E02D2141706442811C0020E4
:10E9A0006A460AE023460A2493FBF4F404EB840548
:10E9B000A3EB450302F8013B401C24B2002CF1DC20
:10E9C000012806DC4AF02002652A04BF302201F843
:10E9D000012B48B9302001F8010B07E0401E1DF85B
:10E9E0000020303201F8012B0028F7DCF068B26912
:10E9F0001044091AF16196F8380000F0140010284C
:10EA00000DD17169B0694118706A4118F0694118F7
:10EA1000B06A4118706B8142BCBF411A316204B0C8
:10EA2000BDE8F087F8B505460E4617461C4600209F
:10EA300074B117F8011BB068A847B06030B1F06A34
:10EA4000401CF0620020641EF3D1F2BD4FF0FF3095
:10EA5000F2BD00007072696E74665F733A20256EB5
:10EA600020646973616C6C6F776564007072696EA5
:10EA700074663A2062616420256E20617267756D4C
:10EA8000656E74007072696E74665F733A206261BD
:10EA90006420257320617267756D656E74000000D7
:10EAA0006E616E004E414E00696E6600494E460032
:10EAB0003000202902460DD00023101D01E05B1C10
:10EAC0001C30D2F874C0634504D2D0F814C08C4511
:10EAD000F5D17047002070470278C9B28A421AB156
:10EAE0001CBF10F8012FF9E718BF002070477047CE
:10EAF00080B500B906A005490B681BB12222002190
:10EB0000984701E0FFF708F8222002BD8C4700205B
:10EB1000636F6E73747261696E742068616E646C89
:10EB200065723A20626164206D6573736167650088
:10EB300000F10103810704D010F8011B89B181079E
:10EB4000FAD10268B2F10131914311F0803F04BF64
:10EB500050F8042FF6E710F8011B11B110F8011B53
:10EB6000FBE7C01A70477047C9B2830706D0521E30
:10EB700022D310F8013B9942F7D11FE0083A13D392
:10EB800002F1040241EA012141EA014150F8043B4B
:10EB9000121F21BF4B40A3F1013C2CEA030C1CF0D7
:10EBA000803FF3D0C9B2001F083210F8013B521E5B
:10EBB00028BF91EA030FF8D818BF0120401E704704
:10EBC00013F0004C03D55B42524263F100039CEA10
:10EBD000210C00F0178010B5644603D3494240422F
:10EBE00061F1000100F00EF8640004D34942404294
:10EBF00061F10001244203D55B42524263F10003FC
:10EC000010BD0000B3BBD9B1B2F5803F7DD2022A5E
:10EC10001ED98C46B1FBF2F102FB11C31B0443EA7F
:10EC20001043B3FBF2FC02FB1C3380B240EA034307
:10EC3000B3FBF2F002FB103240EA0C4000237047B5
:10EC4000022A05D98446B0FBF2F002FB10C27047DD
:10EC50004AB105D100F0010249085FEA300070476F
:10EC600000220023704700F0F1BC0B0002000021DD
:10EC700000207047904271EB030CF6D3B3F5803F50
:10EC80002FD2F0B5B3FA83F7B1FA81F4A7F10F0EE2
:10EC90003D1B5340CEF1200602FA0EF2F3415340E1
:10ECA000B5F10F0746D80F3C2C444140C4F1200673
:10ECB000A040F1414140B1FBF3F603FB1611A2FB6A
:10ECC0000645001BA94102D2761E8018594180EAF0
:10ECD000010221FA0EF362FA0EF200215A40304688
:10ECE000F0BD30B4B1FBF3FC03FB1C11A2FB0C45DF
:10ECF000001BA94103D2ACF1010C8018594130BC72
:10ED000002460B46604600217047B2F1807F65D312
:10ED1000F0B5B2FA82F7B1FA81F4C7F10F063D1BE4
:10ED200022FA06F307F1110EF24120355A40B5F1EF
:10ED30000F07B8D94140C4F12006A040F14141403D
:10ED4000B1FBF3FC03FB1C11A2FB0C45001BA9410A
:10ED500003D2BCF1010C801859410F2F12D30F3F81
:10ED6000C90341EA5041B1FBF3F603FB1611A2FBC4
:10ED70000645D4EBC030A94102D2761E8018594115
:10ED800046EACC3C07B34140C7F12006B840F14108
:10ED90004140B1FBF3F603FB1611A2FB0645001B35
:10EDA000A94102D2761E8018594180EA010221FA57
:10EDB0000EF3C7F1200462FA0EF20CFA07F05A4083
:10EDC0002CFA04F13043F0BD80EA010221FA0EF37F
:10EDD000002162FA0EF260465A40F0BD8C46B1FB4B
:10EDE000F2F102FB11C31B0243EA1063B3FBF2FC16
:10EDF00002FB1C331B024CEA002043EA1063B3FB06
:10EE0000F2FC02FB1C331B024CEA002043EA1063B5
:10EE1000B3FBF2FC02FB1C331B024CEA002043EA6A
:10EE20001063B3FBF2FC02FB1C324CEA002000230F
:10EE30007047FEE7B0B581EA030C0CF0004C40F2DD
:10EE4000FF7515EA11541DBF15EA1357AC42AF42C6
:10EE500039E0E41923EA455343F48013C90241F031
:10EE6000004141EA505EC7021100A7FB02020028E0
:10EE70004FF00000EEFB01204FF00001E3FB072103
:10EE800018BF42F00102401800214941E3FB0E0186
:10EE9000A4F580640F0302D252004041494154F16D
:10EEA00001046CDD470872F1004250F1000051EBA3
:10EEB0000451A1F580115CBF41EA0C01B0BD4CEAE0
:10EEC00005510020B0BD05EA1357AC4214BFAF4254
:10EED00041E050EA410E1CBF52EA430E02E0614697
:10EEE0000020B0BD24423C441BD15FEA070EF6D09F
:10EEF000090302BF01460020AEF1140EB1FA81F7FA
:10EF0000AEEB070401FA07FE0C37C7F1200100FA47
:10EF100007F7C8404EEA000E23EA455343F4801336
:10EF2000A2E733F00043B3FA83F704BFB2FA82FEDC
:10EF300077440B3FE41BB7F1200E2FBF02FA0EF30C
:10EF4000BB40C7F1200E22FA0EFE38BF43EA0E0383
:10EF5000BA40641C82E750EA410E14BF52EA430EE5
:10EF60006FF000014FF4001717EB430F8ABF1946EB
:10EF700017EB410FB5E74CEA05510020B0BDD4F1C5
:10EF80000104B4F120070FDAC4F12007520828BFAA
:10EF900042F0010210FA07F501FA07F7E1BF2A4330
:10EFA000E0403843E1400FE0352C98DCC7F1200405
:10EFB00052EA400220FA07F218BF42F0010231FA89
:10EFC00007F0A1400A43002172F1004250F1000015
:10EFD00051EB0C01B0BD000062B38B0708D0521E8C
:10EFE00011F8013B00F8013B00F024808B07F6D1BB
:10EFF000830740F0208000BF103A07D330B4B1E857
:10F000003810103AA0E83810F9D230BC530724BFAA
:10F01000B1E80810A0E8081044BF51F8043B40F8DC
:10F02000043BD20724BF31F8022B20F8022B44BF47
:10F030000B7803707047083A07D3B1E80810083A14
:10F0400040F8043B40F804CBF7D25307E4E7000054
:10F05000024651EC100B10B5144600F00BF841ECD1
:10F06000100B226010BD000010B5144600F002F82D
:10F07000226010BDC1F30A5343B14A0012F5001FCC
:10F0800028D2A3F2FE32A1EB0251704750EA410CA4
:10F0900020D001F0004C31EA0C01B1FA81F204BF3A
:10F0A000B0FA80F3D2180B3AB2F120032CBF00FA69
:10F0B00003F1914041EA0C013EBFC2F1200C20FA5D
:10F0C0000CF319439040524240F2FD33D21A01EB47
:10F0D00003517047002270474FF4001C1CEB410F96
:10F0E00094BF1CEB430F09E041EA030C50EA4C0CBF
:10F0F00052EA0C0C03D2994208BF9042704714BFE9
:10F100008B428242704700004FF4001C1CEB410F01
:10F1100094BF1CEB430F09E041EA030C50EA4C0C8E
:10F1200052EA0C0C03D28B4208BF8242704714BFD4
:10F130009942904270470000124254D440F2FF7C42
:10F140001CEA11530FD0634531D09B1863453CBF77
:10F1500001EB0251704701F0004141EA0C510020DF
:10F1600000F084BA704750EA410320D001F0004C0F
:10F1700091EA0C011CD0B1FA81F30B3B9A420DD9F4
:10F18000D21A994051EA0C01C3F1200C20FA0CFC70
:10F1900061449840531C40F2FF7CD7E7914041EA1C
:10F1A0000C01C2F1200C20FA0CF319439040704777
:10F1B000B0FA80F31533202BE0D3202AEED3203A87
:10F1C000203B9A4209D9D21A00FA03F141EA0C0114
:10F1D0000020531C40F2FF7CB8E700FA02F141EA3C
:10F1E0000C0100207047524240F2FF7C1CEA115390
:10F1F0000DD06345DBD0B2EB030C3CBFA1EB025159
:10F2000070470CF1010221EA035141F4801150EAE8
:10F21000410CCCD001F0004C352A27DC30B481EA17
:10F220000C01B2F1200309DAC2F12003044601FA0D
:10F2300003F5D0402843D1409C400CE0C3F12002AC
:10F24000450020FA03F418BF44F0010421FA03F04A
:10F2500091400C43002174F1004550F1000051EB46
:10F260000C01244230BC7FF47BAF70476146002024
:10F2700076E70000C1F30A5340F2FE329B1A14DD18
:10F28000D3F120034FEAE17208DDC90241EA50518F
:10F2900041F00040D84080185040704703F2E13000
:10F2A00010B1D24382F00040704700207047000048
:10F2B000C11768B14840401AB0FA80F29040D21CA1
:10F2C000C907C2F5846241EA025202EBD02140052F
:10F2D0007047000070B44FF0004591EA030F40F111
:10F2E000D9816B40841A71EB030603D2001BB14134
:10F2F000121973414FF4001C1CEB410F34BF7CEB1F
:10F30000430442E00C0DA4EB1356352E4FDC45EAC6
:10F31000C323DB0A45EAC121C912B6F120050DDD80
:10F3200063FA05F6EB4086EA0305124218BF45F082
:10F330000105C01851F100010CD213E062FA06F584
:10F34000F2405540F3415A40B340F3405A408018D0
:10F35000594107D349085FEA30005FEA350528BF05
:10F3600045F0010501F58011420875F1004250F1A8
:10F37000000041EB04514E0016F5001F70BC38BF71
:10F3800070470020090D090570471CEB410F10D292
:10F3900052EA43060BD0BCEB410F05D80C0DAB4332
:10F3A000661E342EB6DD02E0AB438018594170BCB6
:10F3B000704770BC70470000F0B540F2FF7581EAFD
:10F3C000030C0CF0004C15EA11541DBF15EA13573D
:10F3D000AC42AF42E5E0BC41C1F31301C3F31303F8
:10F3E000801A994143F4801304D2641E40004941BD
:10F3F00080185941C90241EA5051B1FBF3F603FBB1
:10F400001611A2FB0675D7EBC020A94102D2761EC9
:10F4100080185941C90241EA5051B1FBF3FE03FB88
:10F420001E11A2FB0E75D7EBC020A94103D2AEF18D
:10F43000010E80185941890241EA9051760546EA49
:10F440008E2EB1FBF3F603FB1611A2FB0675D7EB6C
:10F450008020A94102D2761E80185941C90241EA92
:10F4600050514EEA060EB1FBF3F603FB1611A2FB58
:10F470000675D7EBC020A94102D2761E80185941EB
:10F48000C90241EA5051B1FBF3F703FB1711A2FB8C
:10F490000735D3EBC020A94167F100070CBF00423C
:10F4A00047F0010766F3D5274FEA1E31B80814F577
:10F4B000806412DDBD0775F1004250EB0E5051EB38
:10F4C000045111F5801F5CBF41EA0C01F0BD4CF006
:10F4D0007F6141F0E0410020F0BDBD076D0840EACA
:10F4E0000E5041F48011D4F10104B4F120060ADA7F
:10F4F000C4F120060200E04001FA06F3E14018439F
:10F50000B24015430EE0342C13DCC6F1200445EA6A
:10F5100040056D0820FA06F2154321FA06F0A140D5
:10F520000D43002175F1004250F1000051EB0C0138
:10F53000F0BD00205FEA0C01F0BDCFB992185B412D
:10F54000B3FA83F704BFB2FA82F6BF190B3FB7F1E3
:10F5500020062FBF02FA06F3BB40C7F1200622FAAD
:10F5600006F638BF3343BA401CB1E419641E33E7D2
:10F570007F4231F00041B1FA81F404BFB0FA80F665
:10F58000A4190B3CB4F120062FBF00FA06F1A140EC
:10F59000C4F1200620FA06F638BF3143A0403C1BD8
:10F5A0001AE7AC421ABF05EA1357AF4212E050EA1D
:10F5B00041061CBF52EA4306BFE750EA4107304606
:10F5C00061461CBF41EA0551F0BD52EA430C08BF39
:10F5D000C143F0BD00204FF4001616EB410F98BF59
:10F5E00016EB430F08BF16EB410F24BFC14305E0E4
:10F5F00016EB430F0CBF61464CEA0551F0BD00000D
:10F60000400D491840EA81200CD2490DA1F58061D6
:10F61000491C40F0004005DBD1F11F0154BFC84038
:10F62000C017704700207047014648B1B0FA80F11A
:10F630008840C91CC1F58461090501EBD021400552
:10F640007047000000487047E82B0020704700001A
:10F650001FB5044600F0D2F8094944501FBD0FB54C
:10F6600081B000F0CBF80649212205E00FB581B04A
:10F6700000F0C4F802492222425001B00FBD000040
:10F680009447002070B44FF0004591EA030F7FF5D6
:10F6900029AE6B40841A71EB030604D26E40001B46
:10F6A000B141121973414FF4001C1CEB410F34BFE0
:10F6B0007CEB430682E00C0DA4EB1356362E7BDC6C
:10F6C000012E45EAC32341DC43EA525312BFD20262
:10F6D00092025B08240545EAC12141EA5051D2EB70
:10F6E000C020994125D407D1B0FA80F610FA06F16E
:10F6F00062D00020203608E0B1FA81F6B140C6F1B0
:10F70000200220FA02F21143B0404FEAF474B4EB45
:10F71000465434F001064FEA74040AD8D6F50016B0
:10F72000760D04F00044F04061FA06F25040F140DA
:10F730004840C00A40EA415021F0004128BF5FEA3A
:10F74000500550F1000044EBD12135E0DB0A45EAD9
:10F75000C121C90AB6F120050EDD42EA0242120CAF
:10F76000C5F1200603FA06F6EB4042EA06056D42B3
:10F77000984161F100010DE062FA06F5F240554052
:10F7800063FA06FC82EA0C02F3405A406D42904153
:10F7900061EB030111F4801F05D1641E620502D0E4
:10F7A0006D004041494121F48011430875F1004347
:10F7B00050F1000041EB045170BC70471CEB410F4D
:10F7C00015D223F0004352EA43060BD04FEA4C0C0B
:10F7D000BCEB410F04D80C0D661E342EB7DDEBE7F1
:10F7E000801A994150EA410608BF0021E4E708BFAA
:10F7F0001CEB430F28BF6FF00001DDE700207047CE
:10F8000080B50B0000210022002815D0012824D14A
:10F81000042241F20C0118001B689B689847010004
:10F8200041F20C0000F01BFE002803D000F01AFE8D
:10F83000010000E0002110E004222C2118001B68C8
:10F840009B68984701002C2000F009FE002803D097
:10F8500000F088FE010000E00021080002BD2DE953
:10F86000FC4104000D001600002700E07F1CB74299
:10F8700037D2182000FB07F005EB000898F81400B9
:10F880000028F3D01021D8F8000001F02FF8010073
:10F89000D8F8100010F1010F0FD1D8F80C30D8F8BB
:10F8A00008202000D4F800C0DCF808C0E0470100C0
:10F8B00049B20029DAD040B214E0D8F81000009024
:10F8C000D8F80C30D8F808202000D4F800C0DCF8B4
:10F8D0000CC0E047010049B2002900D1C6E740B2A0
:10F8E00000E00020BDE8F6812DE9FC4704000D0092
:10F8F00016001F005FF000085FF0000908E00098A4
:10F900002844DAF80410086018F1010819F1010917
:10F91000B94517D2182000FB09F006EB000A9AF847
:10F9200014000028F2D05FF0FF3000906A46414694
:10F93000200023689B699847010049B20029DED066
:10F9400040B200E00020BDE8F68738B50C00002585
:10F9500001F087F80100200001F089F800280DD09F
:10F9600001F089F80400002C08D0200001F088F88C
:10F97000002803D0200001F088F80500280032BDDF
:10F980002DE9FC478246884616001D000B9C002C82
:10F9900001D1FEF7C1F82000202101F07BF82800FA
:10F9A00001F07BF814F11C0140B201F07CF8010079
:10F9B00049B2002901D040B2DDE00A9F280001F0E1
:10F9C0008BF8A07739002800FFF7BFFF206120697E
:10F9D000002802D10220607701E0012060776A46AA
:10F9E00014F11801280000F0D9FF010049B20029E4
:10F9F00001D040B2BFE0280001F07AF8002803D11E
:10FA0000DFF8A407606105E0280001F071F801F05B
:10FA10008DF86061280001F08BF80500002D00F0E2
:10FA2000A980280001F089F8002800F0A3802800B0
:10FA300001F083F801F086F8002800F09B80280090
:10FA400001F085F8002800F09580280001F07FF88B
:10FA500001F082F8002800F08D80280001F06DF898
:10FA6000002101F07FF884ED020A280001F06FF810
:10FA7000002101F091F8E060280001F05EF801F04B
:10FA800061F881463000C0B2002808D004220C2161
:10FA90004046D8F800309B689847070007E00422EA
:10FAA0000C215046DAF800309B6898470700002F79
:10FAB00005D1DFF8F80601F099F801205BE0F6B215
:10FAC000002E0AD0484601F099F804220100404671
:10FAD000D8F800309B68984709E0484601F08EF856
:10FAE000042201005046DAF800309B68984778609D
:10FAF0007868002805D1DFF8B80601F077F8012012
:10FB000039E0280001F019F801F011F83860786840
:10FB1000C0F800907868061D5FF000081DE028001E
:10FB200001F015F8002101F037F812E0280001F08B
:10FB30000EF801F011F88246280000F0FEFF01F0F7
:10FB400001F88245EBD1280001F001F8414601F0AF
:10FB500023F846F8280018F10108C845E6DB28001C
:10FB600001F0C0F8B860DFF84C26D2E90001390096
:10FB7000C4E900010020BDE8F68770B505000E005D
:10FB8000140000200021002284E80700280000F073
:10FB900084FF14F1080140B200F085FF010049B272
:10FBA000002901D040B214E031002800FFF7CDFE5B
:10FBB0002060280000F09CFF002803D1DFF8E80552
:10FBC000606005E0280000F093FF00F0AFFF606088
:10FBD000002070BD10B4DFF8E04504604260816031
:10FBE000036100210175002181610021C1610021B3
:10FBF000016210BC704770B504000D0016001021A2
:10FC0000200000F065FE04EB0501091A01F087F8F9
:10FC10000400002C01D0211D00E000213000FFF77E
:10FC2000EFFD0100200000F001F870BD38B50400C0
:10FC30000D00002C01D1FDF76FFF002D01D1FDF764
:10FC40006BFF04222421200023685B6B984701008E
:10FC5000242000F004FC002809D0002C01D0211D34
:10FC600000E000212B002200FFF7B4FF00E000209D
:10FC700032BD70B506000C00002C01D1FDF74CFF21
:10FC8000307D002805D0DFF8340500F0AFFF0020FC
:10FC900043E00120307504220821B068B3681B6876
:10FCA0009B6898470100082000F0D9FB002803D08A
:10FCB000B16801F035F900E00020F060300000F09C
:10FCC000B3FB002801D0002027E0B568200001F038
:10FCD00035F901F038F90422C10028002B689B682F
:10FCE00098470500002D05D1DFF8D40400F07EFF11
:10FCF000002012E02A00210030003368DB6A9847B8
:10FD0000002807D12A002100300033689B6A9847F9
:10FD1000002801D0002000E0280070BDF8B50400E4
:10FD20000D0016001F00207D002805D1DFF8940487
:10FD300000F05CFF01201BE0A2693900200023686D
:10FD40001B6C9847010049B2002901D040B20FE076
:10FD50003B683200290020002568ED6BA8470100B0
:10FD600049B2002901D040B202E0002020750020F5
:10FD7000F2BD80B50300102298689B681B689B68E1
:10FD8000984702BDF8B504000D0016001F002000C2
:10FD900000F05DFB0021002209E00C2303FB02F3CD
:10FDA00003445B6813F1010F00D1491C521CA36985
:10FDB0009A42F2D30C2906D30C21DFF80C0400F090
:10FDC00015FF012013E0A2690C214A4310440021D1
:10FDD0000022002380E80E0005605FF0FF314160E3
:10FDE0008660A0693860A069401CA0610020F2BD57
:10FDF00038B504000D0020002168496988470100DA
:10FE000049B2002901D040B227E0200000F01FFBDA
:10FE100000210DE00C2202FB01F20244526812F1B3
:10FE2000010F04D10C2202FB01F202445560491C6F
:10FE3000A2699142EED30423A2690C320C20424302
:10FE4000E169606864682468E469A047010049B218
:10FE5000002901D040B200E0002032BD2DE9F04180
:10FE6000070088461500002D01D1FDF755FE00263C
:10FE700002E045F83600761C404601F05FF801F0DC
:10FE800062F886421BD2404601F058F8310001F07A
:10FE90005FF80400002C01D1FDF73EFE200000F0C9
:10FEA0002CFE04224101B868BB681B689B68984718
:10FEB0000028DED1C54800F099FE012000E00020B6
:10FEC000BDE8F0812DE9FE4381460F0014001E00BD
:10FED000DDF82880380001F031F8414601F038F8AB
:10FEE000002801D1FDF718FE4846D9F80010496BEB
:10FEF00088470500002D04D1B54800F077FE0020AA
:10FF000026E000200190CDF8008033002A0039005F
:10FF10004846D9F80070BF6BB847002804D0AD48F8
:10FF200000F064FE002013E0002C10D004EBC800A9
:10FF300040680C2101FB06F14058286104EBC80021
:10FF400041680C20464301EB0600406868612800C8
:10FF5000BDE8FE8370B505000C00002C01D1FDF753
:10FF6000DBFD94F90000012811D16068002801D15F
:10FF7000FDF7D2FD6668716868686A681268D268C1
:10FF80009047310068686A681268D268904700201C
:10FF9000207000206060002020610020606121004E
:10FFA00068686A681268D268904770BD2DE9FE43A0
:10FFB00080460E0014001D000A9F300000F0BEFFB6
:10FFC000390000F0C5FF002801D1FDF7A5FD04228E
:10FFD0002021D8F80400D8F804301B689B689847A3
:10FFE00081460120019000972B004A46310040468F
:10FFF000D8F80060B66BB047002804D0764800F00F
:020000040005F5
:10000000F5FD002015E0002C12D004EBC70040687D
:100010000C2101FB05F14058C9F8100004EBC700A2
:1000200041680C20454301EB05004068C9F8140005
:100030004846BDE8FE8380B5010048684968096804
:100040004969884702BD2DE9F84F04000F001600EA
:10005000002E01D1FDF760FD00945FF0000804E080
:1000600006EBC800446018F10108380000F066FF94
:1000700000F069FF804549D2380000F05FFF41463B
:1000800000F066FF0500002D01D1FDF745FD2800B9
:1000900000F078FF00F07BFF814604220C2101FB79
:1000A00009F100988068009B9B681B689B689847D3
:1000B0000400002C02D05FF0000A0AE00C2000FBD4
:1000C00009F94946454800F091FD01201FE01AF169
:1000D000010ACA45C4D2380000F05EFF83462800FA
:1000E00000F050FF514600F05DFF0C2101FB0AF1CA
:1000F00004EB01025946FFF740FD40B20028E6D06C
:100100005146374800F072FD012000E00020BDE8B4
:10011000F28F2DE9FC4105000E0017001C005FF076
:10012000000812E010220099A868AB681B689B6861
:1001300098470C2101FB08F178500C2000FB08F0D7
:100140003858002826D018F10108300000F01AFFB6
:1001500000F01DFF804523D2300000F013FF414620
:1001600000F020FF00F0B8FC0028ECD0002C04D0F8
:1001700054F8280010F1010FE5D169460C2000FB6E
:1001800008F0384400F046FC010049B20029C9D00B
:1001900040B206E00099134800F028FD012000E07D
:1001A0000020BDE8F6810000C4DA050058C2050051
:1001B00088C2050004D8050074B7050028B60500FC
:1001C000F8C10500B8B70500E8BE050020BF05006E
:1001D000B0BE050004B80500E8BA050014BA050071
:1001E000C0C7050028C2050080B5030004222021F5
:1001F00098689B681B689B68984702BD2DE9FC477F
:100200000500894616009846DDF828A00B9C484654
:1002100000F0C2FE0700484600F090FE514600F094
:1002200097FE00F0AFFE414600F0BCFE019600973D
:1002300003002200D2B26968A868FFF7A1FBBDE8FD
:10024000F6872DE9F0438BB005000E0091461F00A4
:1002500000206A68310002A800F0BEFEA96900F023
:1002600044FF010049B2002901D040B2C2E00020A1
:10027000019001A902A801F0B5F9010049B20029D5
:1002800001D040B2B6E05FF0000801E018F10108CB
:10029000300000F053FE00F056FE804519D23000C9
:1002A00000F04CFE414600F053FE0400002C01D14A
:1002B000FDF732FC019B09EBC800426821002800D1
:1002C0002C68246BA047010049B20029DED040B25F
:1002D00090E04A46019902A800F0B0FF010049B23F
:1002E000002901D040B285E0280000F0B0F8CDF838
:1002F00000903B000200002102A801F055F8010027
:1003000049B2002901D040B274E002A801F0D8F946
:10031000060002A801F0D6F90700102168686A6893
:100320001268126B904780461022414668686B68DD
:100330001B689B6898470400002C01D1012059E0FC
:100340004246210028692B691B68DB699847320007
:1003500039002869FFF783FA010049B2002901D06A
:1003600040B247E0686869680968496A88473300AD
:100370003A0001002869FFF7B7FA010049B20029E5
:1003800001D040B236E002A800F0FFFE210068680C
:100390006A681268D268904768686968096849693C
:1003A0008847010049B2002901D040B222E0E96942
:1003B00068686A681268126A9047010049B20029A9
:1003C00001D040B216E0286929690968096988479F
:1003D000296A814200D228621022296A68686B6803
:1003E0001B689B6A9847010049B2002901D040B2BE
:1003F00000E000200BB0BDE8F08370B505000C00F4
:100400001600002C01D1FDF787FBA869002801D157
:10041000002008E00422B100A868AB681B689B6854
:1004200098472060002070BD10B504000020A06136
:1004300004229021606863681B689B699847E061AB
:10044000E069002801D1012000E0002010BD80B546
:100450000421C06900F03CFA02BDC0687047080082
:100460007047000025490160002141F204028150DB
:10047000002141F208028150704780B541F2040228
:100480008258B2F5806F06DB4FF480611C4800F0A3
:10049000ADFB012017E041F20402825800EB82021A
:1004A00041F20803C358536041F208028258891888
:1004B00041F20802815041F204014158491C41F2C5
:1004C00004028150002002BD41F2080140587047EB
:1004D00080B5002904D441F20403C358994207DBD4
:1004E00041F204028258074800F080FB012004E03A
:1004F00000EB810040681060002002BD50C3050081
:10050000A0C8050084C4050070B4030000200124C5
:1005100021E003EB840555F8045C53F82460B542F0
:1005200018DA03EB840050F8040C53F8245003EB62
:10053000840646F8045C43F8240001EB840050F87C
:10054000040C51F8245001EB840646F8045C41F891
:1005500024000120641C9442DBDBC0B20028D5D10A
:1005600070BC7047DFF85C130160704770B5040021
:100570000D0016000020A060012084F8280001F082
:10058000A3F8B6FBF0F06060E56060680001284405
:100590002061616800EB81006061616800EB8101AE
:1005A000A16162680C20424301EB020060620020FE
:1005B00070BD38B584684568AC4206DB4168DFF839
:1005C000080300F013FB012010E0C46885682D01CA
:1005D0002C442160A260E3605FF0FF3161608168BC
:1005E000491C8160012180F82810002032BD38B5F7
:1005F000C46885682D012C440568AD68A8470028AB
:1006000001D0012002E004986060002032BDC06883
:1006100049680901084481688B4201DA002005E03D
:10062000C068904201DA002000E0012070472DE907
:10063000F041040015001E000027002906D1A16921
:10064000226A0C20424301EB020818E0886810F18E
:10065000010F01D100201DE0A26989680C204143EF
:1006600002EB01080BE0D8F8080010F1010F10D0E0
:10067000A169D8F808200C20424301EB020833009E
:100680002A0041462000FFF7C2FF0028EBD0474672
:10069000FFE73800BDE8F0812DE9F84F050095F837
:1006A0002800002802D0A868002800D1C4E000205B
:1006B00085F82800A9680020002228E0EB681401D2
:1006C0001B592C6944F820306B6943F82020EB68F3
:1006D000140123445B686C6A44F82230401C15E026
:1006E000EB68140123445B6813F1010FE6D1491E46
:1006F000EB6814011B592C6944F821306B6943F8ED
:1007000021205FF0FF336C6A44F82230521CAB6842
:100710009A42E5DBAA68121A696901EB80012B692C
:1007200003EB8000FFF7F0FE002028620120E86163
:10073000A9692A6A0C20424301EB02065FF0FF30F0
:10074000B060686900687060E96802011144496836
:1007500011F1010F03D100216A6A42F82010696A81
:1007600051F820003060012716E0A0688860A26080
:1007700011E0D5F818C00C2043430CEB03000368CC
:100780009B45F2DB0400A36813F1010FF1D1A260D5
:100790005FF0FF3088607F1CA86887424CDA686988
:1007A00050F82780E8685FEA08110844D0F8009004
:1007B00081680091D0F80CA05FF0000B416811F146
:1007C000010F1DD1002405E00168B1EB0B01494583
:1007D00015DA04005346009A21002800FFF727FF8E
:1007E000002C09D0E9686268120111442268096886
:1007F0008A18934500DA93460028E5D102E001E02B
:10080000D0F804B0686A40F828B0A969EA690C20F9
:1008100042431144C1F800B0C1F80480EA69E869B4
:10082000401CE8613068834504DA0E00286AB06035
:100830002A62B0E73400A6E7BDE8F18F10B50400E6
:100840002000FFF729FFA068002801D100201EE04A
:10085000A169226A0C20424301EB0200002105E05D
:10086000A26983680C20434302EB030000280DD0EB
:10087000E26843681B011A4403681268D31899425E
:1008800000D21900826812F1010FE9D1080010BDF1
:1008900070B504000D0016002000FFF7FDFE002DCE
:1008A00002D4A068854206DBA2682900074800F050
:1008B0009DF9012004E0606A50F8250030600020B6
:1008C00070BD000020C3050080C8050058C40500A5
:1008D0000818401EB0FBF1F001FB00F10800704762
:1008E000B0FBF1F001FB00F1080070470818401E52
:1008F000B0FBF1F001FB00F10800704740B20128A5
:1009000020D0022827D003282BD004282FD0062857
:1009100033D007281CD0082835D0092824D00A282D
:100920000CD00B2811D00C2830D00D2822D00E2846
:1009300026D0102812D012282BD02DE002200860DB
:100940000020704704200860FAE708200860F7E7F5
:1009500002200860F4E704200860F1E70420086042
:10096000EEE701200860EBE701200860E8E70820D7
:100970000860E5E708200860E2E701200860DFE79B
:1009800004200860DCE708200860D9E71020086030
:10099000D6E701200860D3E70120D2E72DE9FC412A
:1009A00007000C0016000125380000F0A1F800280F
:1009B00012D05FF0000808E0380000F099F84146D6
:1009C00000F086FE454318F10108380000F090F869
:1009D00000F098FE8045EFD3380000F05EF86946DD
:1009E00040B200F060F8010049B2002901D040B2E5
:1009F0000EE031009DF90000FFF780FF010049B2D1
:100A0000002901D040B203E0306845432560002052
:100A1000BDE8F6817CB506000C00002C01D1FDF785
:100A20007BF80125706800280BD0002105E0706874
:100A300000EB810040684543491C706800688142B2
:100A4000F5DB694696F90800FFF758FF010049B247
:100A5000002901D040B203E0009845432560002002
:100A600076BD80B50022082100F051FE02BD80B5A0
:100A700000F060FE02BD80B5042100F075FE02BDED
:100A800080B5006800F075FE02BD80B500F072FE12
:100A900002BD0000002200F06FBE80B500220621DA
:100AA00000F083FE02BD38B504000D0000F092FE98
:100AB00002002900200040B200F00EFF32BDF8B560
:100AC00004000D0016001F0000F084FE3B00320001
:100AD00001002800A047F2BD80B500220E2101F0E0
:100AE000BDF8002801D0012000E00020C0B202BD06
:100AF00080B5042101F0C6F802BD10B50400200045
:100B000001F0C5F8002805D0200001F0C0F801F080
:100B1000C3F800E0002010BD10B50C0000F00EFA84
:100B2000210000F015FAFFF7E8FF10BD704770478D
:100B300080B50C2101F0B5F802BD80B5082101F0A7
:100B4000B5F802BD80B5006800F013FE02BD80B5A7
:100B50000A2101F0B0F802BD80B5006800F009FE7E
:100B600002BD000038B504000D002000FFF7EAFFC9
:100B7000854206D3B0220649064801F0A1F8AFF33A
:100B80000080200001F0AEF8290001F0ADF831BD81
:100B900074AB0500FCD7050038B504000D0020003B
:100BA000FFF7DAFF854206D3B0220649064801F076
:100BB00087F8AFF30080200001F09EF8290001F0D3
:100BC0009DF834BD04AC05000CD805000EB400B58A
:100BD00001A901F09BF85DF810FB80B501F096F8D3
:100BE00001A0FFF7F3FF01BD0D0A00000EB400B530
:100BF00001A9FFF7F2FF5DF810FB000080B501F0DE
:100C00008FF802BD40B200281BD0022821D01AD391
:100C1000042826D021D3062827D02CD3082826D074
:100C200015D30A2829D01AD30C2822D027D30E286E
:100C300027D018D310280ED025D3122825D004D3BE
:100C400025E0144824E0144822E0144820E0144829
:100C50001EE014481CE014481AE0144818E0144838
:100C600016E0144814E0144812E0144810E0144848
:100C70000EE014480CE014480AE0144808E0144858
:100C800006E0144804E0144802E0144800E0144868
:100C900070470000DCD90500E4D90500ECD9050057
:100CA000F4D90500FCD9050004DA05000CDA0500CA
:100CB00014DA05001CDA050024DA05002CDA050038
:100CC00078D7050084D7050034DA05003CDA050042
:100CD00044DA050090D705004CDA050054DA050027
:100CE000E0D4050080B50022102101F01DF802BDFE
:100CF0007A4B03607A4B43608160C260016142615C
:100D0000816881610021C16100210162704710B5D5
:100D100004000A442000FFF7EBFF200010BD30B5AF
:100D200089B004000D00002C01D1FCF7F5FE2A006B
:100D300021006846FFF7EBFF0422242100F06AF847
:100D400001002420FFF78BFB002804D0694600F047
:100D5000FFFF040000E00024684600F003F82000D4
:100D600009B030BD7047F8B504000D001600310021
:100D7000A068FFF7ADFD070033002A00390020000E
:100D80002468E469A047002801D1380000E0002071
:100D9000F2BD10B5012300220468E469A04710BD2C
:100DA00070B504000D0016003100A068FFF790FD3B
:100DB00033002A00010020002468E469A04770BDC8
:100DC000F8B504000E0015001F003900A068FFF7F9
:100DD0007FFD2169A269914201D1864204D0414838
:100DE000FFF704FF012013E03900A068FFF770FD52
:100DF0006269121AAA4206D2AB1A29003A48FFF7D2
:100E0000F5FE012004E0284420612069A061002053
:100E1000F2BD001F38B504000D00110060696A4280
:100E20001044FFF75DFD216988420AD22169081A42
:100E30000300281A020029002C48FFF7D7FE0020E3
:100E400000E0606132BD38B504000D001100A069FA
:100E5000FFF73EFD6269121AAA4206D2AB1A2900B8
:100E60002348FFF7C3FE002008E000EB0501A16165
:100E7000E1694140E161216A491C216232BDC269D8
:100E80005140C161016A491E0162704780B5016A23
:100E9000002902D1C16900290CD0C169002901D102
:100EA000012200E00022D2B2016A1248FFF79EFE42
:100EB000002000E0012002BD10B5040020002168E0
:100EC00009698847002804D10B48FFF78FFE0120ED
:100ED00002E02069A061002010BD0000D4B505002B
:100EE00018B605001CB2050070BB05009CB80500D3
:100EF000E8B80500B4BB05005CBA0500806870471F
:100F000070B504000D002900A069FFF7E1FC0600A0
:100F100029006069FFF7E4FC861B300070BD00000B
:100F200038B504000D00200000F036FF02482060B4
:100F30006560200032BD00BFB0CB050080B5082140
:100F400000F02EFF02BD80B5006800F012FC02BD6B
:100F500038B504000D002000FFF7F5FF854206D3E9
:100F6000B0220649064800F0ABFEAFF30080200037
:100F700000F01BFF290000F01AFF32BD44AE05004F
:100F80008CDA050080B5042100F019FF02BD80B5A0
:100F9000006800F0EEFB02BD80B50C2100F014FFEC
:100FA00002BD000038B504000D002000FFF7EFFF80
:100FB000854206D3B0220649064800F081FEAFF311
:100FC0000080200000F005FF290000F004FF32BD82
:100FD00094AC050074DA05000160426000210162F2
:100FE0007047000038B50C001500A068854201DA92
:100FF000FCF792FDA06810F1010F00D1A56031BD92
:1010000038B50C001500E068854201DAFCF784FD74
:10101000E56031BD2DE9FC470400894615001E003E
:101020005FF0FF375FF0FF38484600F0DCFE824695
:10103000206800F0DEFE514600F0E0FE00F0F8FE11
:10104000762804D0772816D081280DD020E0484695
:1010500000F0F4FE00F0FFFE0700484600F0EEFE50
:1010600000F0FFFE804613E0484600F000FF00F06D
:101070000BFF07000CE0484600F00CFF00F017FFE4
:101080000700484600F006FF00F017FF8046FFE724
:10109000DDF8289017F1010F10D0206A401C206263
:1010A000CDF8009033002A003900200000F07CF9D0
:1010B000010049B2002901D040B214E018F1010F3B
:1010C00010D0206A401C2062CDF8009033002A0026
:1010D0004146200000F068F9010049B2002901D022
:1010E00040B200E00020BDE8F687F8B504000D002E
:1010F0002068FFF723FFFFF726FF86000422310058
:10110000606863681B689B689847206120690028B5
:1011100006D13100DFF89805FFF768FD012033E0C4
:10112000002600270EE0206940F827602068FFF7BE
:1011300005FF3900FFF70CFFFFF724FFFFF727FF3C
:1011400086197F1C2068FFF7F9FEFFF7FCFE874237
:10115000E9D3A6616661AE19E660E561E56818202D
:10116000454304222900606863681B689B689847B0
:10117000A060A068002806D12900DFF83405FFF739
:1011800035FD012000E00020F2BD10B50400A1688B
:10119000606862681268D268904721696068626816
:1011A0001268D2689047002010BD2DE9F8430C006A
:1011B00015002000FFF7A1FC0600002700E07F1CBF
:1011C000B74238D2200000F062FD390000F07CFE0A
:1011D00080465FF0000904E00098002824D119F14E
:1011E0000109404600F08AFE0028E8D0404600F0A1
:1011F00085FE00F087FA8145E1D2404600F07EFE90
:10120000494600F065FA5FF0FF31009169460C2213
:1012100050432844FFF7FEFB0100080040B20028BD
:10122000DAD0080040B207E00099DFF88804FFF741
:10123000DDFC012000E00020BDE8F2832DE9F74F3E
:101240000400A06800905FF0000B002500E06D1C1A
:101250002068FFF773FEFFF776FE854280F08680F8
:101260002068FFF76BFE2900FFF772FE0600029868
:1012700000EBC50047680099206950F82520182028
:10128000424301EB02083A0031002000FFF78DFFD6
:10129000010049B2002902D15FF0000943E040B2E9
:1012A00080E05FF0FF30CAF810003AE05FF0FF30F6
:1012B000CAF808005FF0FF30CAF80C000C2000FBF1
:1012C00009F0385800284FD13000FFF75BFE49463F
:1012D000FFF768FEFFF700FC002845D1DAF80000B0
:1012E000002841D001208AF8140001980028D8D0A5
:1012F000019850F82B00CAF810001BF1010B3000C8
:10130000FFF740FE4946FFF74DFEFFF7E5FB0028DB
:1013100007D0DAF8100010F1010F02D001208AF88E
:10132000140019F101093000FFF72CFEFFF72FFE22
:1013300081458CD2182000FB09F008EB000A0C2034
:1013400000FB09F03844CAF8040051460C2000FBA9
:1013500009F03844FFF75EFB0100080040B20028A6
:10136000A4D0080040B21DE00020BCE700996269EB
:101370001820424301EB020000210FE0182202FB7B
:1013800001F202445FF0FF3393605FF0FF33D360FC
:10139000012313755FF0FF331361491CE269914229
:1013A000ECD30020BDE8FE8F2DE9F84F88B0040093
:1013B0000D00904699462068FFF7C0FD2900FFF711
:1013C000C7FD0600A06801900199206950F825200A
:1013D0001820424301EB02073000FFF78EFB02901A
:1013E0005FF0000A15E0300000F08DFD514600F07E
:1013F0006FF91821484307EB000B226A5946200079
:10140000FFF7F0FD226A59462000FFF7F9FD1AF1B7
:10141000010A300000F077FD002806D0300000F00F
:1014200072FD00F06FF98245DDD3CDF80C90CDF858
:1014300010805FF000082EE005A804990C2202FB42
:1014400009F2114491E80C1080E80C100098182162
:1014500001FB09F100EB010B0698404514D10798F8
:10146000A84211D1039800EB8900CBF8040005983D
:10147000CBF80000524659462000FFF7B3FD226A20
:1014800059462000FFF7BCFD19F10109E0698145CB
:10149000D2D318F10108029880457CD2206A401C02
:1014A0002062300000F0F3FB414600F00DFD814664
:1014B0005FF0000A0FE0484600F02AFD514600F0B8
:1014C00007F91821484307EB0001226A2000FFF7C3
:1014D00089FD1AF1010A484600F01AFD002806D0DD
:1014E000484600F015FD00F00DF98245E3D3D4F82D
:1014F00020A012980090039B049A49462000FFF711
:1015000089FD5FF0000B11E0484600F006FD5946EA
:1015100000F0DEF8002807D41821484307EB00014B
:10152000226A2000FFF76CFD1BF1010B484600F01A
:10153000F4FC002806D0484600F0EFFC00F0E2F88A
:101540008345E1D35FF0000B0FE0484600F0E0FC7C
:10155000594600F0BDF81821484307EB0001226A04
:101560002000FFF74DFD1BF1010B484600F0D0FCB9
:10157000002806D0484600F0CBFC00F0C3F88345B5
:10158000E3D3019962691820424301EB0200009005
:101590005FF000097AE7002514E0300000F0C2FC9B
:1015A000290000F095F81821484307EB0008226A4B
:1015B00041462000FFF716FD226A41462000FFF752
:1015C0001FFD6D1C300000F0ADFC002806D030007F
:1015D00000F0A8FC00F096F88542DED3002009B0A8
:1015E000BDE8F08F2DE9FC4104000E00206800F0FA
:1015F0009EFC002858D0002500E06D1C206800F0FB
:1016000096FC00F099FC85424ED2206800F08FFCD9
:10161000290000F097FC0700380000F0ADFC00281E
:10162000EBD0380000F0A8FC00F0ABFC00902248A2
:10163000FDF77EFA019001A9684600F0A7FC8046FC
:10164000380000F099FC00F0A8FCD8F800201A49F6
:1016500000F0A7FC002808D1DDF800801648FDF74F
:1016600067FA804501D1012000E00020C0B20028C7
:10167000C3D02068FFF790FC8046380000F0A5FC3E
:1016800001004046FFF7F3F9FFF7F5F9FFF7FDF921
:1016900081680C303060A0698842AED0A2690748EA
:1016A000FFF7A4FA012000E00020BDE8F681000069
:1016B0002CBB0500FCBD050018CE050050B8050088
:1016C000C068704780687047282028207047000055
:1016D00038B504000D00200000F014F8854206D350
:1016E000B0220649064800F0EBFAAFF30080200074
:1016F00000F071FC290000F070FC32BDF4AF050071
:10170000A4DA050080B5006800F033F802BD38B5F2
:101710000400150089B2200000F065FC010089B2C8
:10172000002905D080B2204400F073FC0500FFE7DB
:10173000280032BD38B504000D00200000F06BFC1D
:10174000854206D3B0220649064800F0B9FAAFF345
:101750000080200000F064FC290000F063FC32BD32
:10176000D4AE050094DA050080B589B200F062FCC1
:1017700002BD7047001D704700B500BF13009646BC
:101780009446103928BFA0E80C50FAD85FEA417C93
:1017900028BF0CC048BF40F8042BC90728BF20F859
:1017A000022B48BF00F8012B00BD38B5040015001E
:1017B00089B2200000F017FC010089B2002905D091
:1017C00080B2204400F049FC0500FFE7280040B249
:1017D00032BD000080B50A48006800280CD10949D4
:1017E0000420FEF73CFE002803D007490968016089
:1017F00000E00020024908600148006802BD0000C6
:101800008447002080470020EC2A002080B5080093
:101810001100FFF7E2F9002002BD000070B50E00D4
:1018200015001C00002801D1FCF776F9002E01D12B
:10183000FCF772F9002D01D1FCF76EF9002C01D1F3
:10184000FCF76AF970BD2DE9F84305000C0016009D
:101850001F00DDF82080002C07D14246DFF874120B
:10186000380000F0FDFB01201AE02000FFF74AFFDE
:101870008146AD084D4507D24246DFF85C1238007C
:1018800000F0EEFB01200BE0002506E0290020001F
:10189000FFF71EFF46F825006D1C4D45F6D30020CE
:1018A000BDE8F28340B2002808D002280AD007D34E
:1018B00004280BD008D305280AD00BE000200AE04A
:1018C000012008E0022006E0032004E0042002E0FA
:1018D000052000E00020704780B51300020052B2DE
:1018E000002A1ED0022A2CD017D3042A39D030D394
:1018F000062A42D03DD3082A43D01AD30A2A14D04C
:101900002BD30C2A31D040D30E2A46D041D3102AF3
:1019100013D01AD3112A44D047E00A2008700020BF
:101920004DE001200870002049E00B2008700020E5
:1019300045E007200870002041E0112008700020D9
:101940003DE002200870002039E0102008700020DF
:1019500035E003200870002031E0092008700020E5
:101960002DE004200870002029E00D2008700020E0
:1019700025E005200870002021E0062008700020E6
:101980001DE008200870002019E00C2008700020DD
:1019900015E00E200870002011E00F2008700020D4
:1019A0000DE012200870002009E000220A7040B209
:1019B0000200DFF83411180000F052FB012002BDD4
:1019C000F0B585B004000D0017001E0033003A008A
:1019D00029002000FFF722FF390004A800F052FB85
:1019E000010002A800F050FB002102A800F05DFBFE
:1019F000002810D13948019040F2FC500090384B3B
:101A0000DFF8E8202900280000F033FB02A800F0EE
:101A100057FB01204CE0200000F065FB0400002C87
:101A20003ED002A800F06CFB0700200000F06EFB27
:101A300040B2FFF737FF387002A800F061FB0700E3
:101A4000200000F069FBB87002A800F059FB070005
:101A5000200000F06DFBF87002A800F051FB0700B9
:101A6000200000F071FB2A00391D40B2FFF734FF5F
:101A70000700380040B2002805D002A800F020FB83
:101A8000380040B214E0200000F064FB002802D0CF
:101A900001280FD014E002A800F032FB00214170B1
:101AA00002A800F05DFB306002A800F009FB0020F6
:101AB00005B0F0BD02A800F023FB01214170EFE763
:101AC000DFF8F010280000F0CBFA02A800F0F8FAD6
:101AD0000120EDE768C10500A4BA0500B8CE0500F5
:101AE000ACB10500002070479CC5050078CB05000F
:101AF000F0B585B004000E0017001D002B003A0061
:101B000031002000FFF78AFE390004A800F0BAFA7D
:101B1000010002A800F031FB002102A800F03EFB0A
:101B2000002812D1DFF8900001904FF4FD60009082
:101B3000DFF88830DFF878203100300000F099FAC3
:101B400002A800F036FB012030E0200000F044FB4A
:101B5000002823D000F04DFB0400002C1ED002A86A
:101B600000F04CFBDFF8E41000913300020021008C
:101B70002020FFF768FE0600300040B2002805D0A4
:101B800002A800F016FB300040B20FE002A800F0FF
:101B900035FB06002000FFF7B5FD306202A800F01B
:101BA00033FB286002A800F004FB002005B0F0BD64
:101BB00078CB0500A8C30500B8CE0500ACB1050080
:101BC000F0B585B004000D0016001F003B00320088
:101BD00029002000FFF722FE310004A800F052FA8D
:101BE000010002A800F01DFB002102A800F02AFB62
:101BF000002812D1DFF85C00019040F695100090AB
:101C0000DFF85430DFF848202900280000F031FACE
:101C100002A800F022FB012016E0200000F030FBBB
:101C20000400002C08D002A800F037FB05002000BB
:101C300000F03AFB85ED000A02A800F03FFB386097
:101C400002A800F00AFB002005B0F0BDECD70500AB
:101C500078CB0500B8CE0500ACB1050038B504005E
:101C6000150089B2200000F0BEF9010089B20029F8
:101C700005D080B2204400F02EFB0500FFE72800CD
:101C8000C0B232BD80B589B200F027FB02BD80B57D
:101C90000A2100F035FB02BD80B50068FFF769FD41
:101CA00002BD80B589B200F030FB02BD80B589B2BB
:101CB00000F03EFB02BD80B589B200F04CFB02BDD6
:101CC00000B583B00091019202906A460449182041
:101CD000ABBE002801D1FBF71FFF03B000BD00BF62
:101CE00010100200001D704780B500EB810090EDE0
:101CF000000A00F043FB01BD001D704780B500EBFA
:101D0000C100D0E9000100F03AFB04BD80B50A0033
:101D10000100024800F034FB01BD0000802B0020D0
:101D200004218000001D704738B50400150089B2F9
:101D3000200000F058F9010089B2002905D080B2D6
:101D4000204400F035FB0500FFE7280032BD00000D
:101D500038B504000D002900200000F02BFB291DE0
:101D6000201D00F02BFB0A4820600A486060A8682C
:101D7000A060E868E0602869206168696061A8691E
:101D8000A061E869E061286A2062200032BD00BFDE
:101D9000D4B5050018B6050080B500F013FB02BDF0
:101DA00080B589B200F00FFB02BD001D704710B571
:101DB00000EB8104200000F02CF9204410BD80B518
:101DC00089B200F013FB02BD80B589B200F021FB9F
:101DD00002BD001D704710B500EB8104200000F02B
:101DE00018F9204410BD80B500220421FFF78FFCB4
:101DF00002BD80B5062100F01FFB02BD38B504000E
:101E00000D00200000F01DFB854206D3B0220649DC
:101E10000648FFF755FFAFF30080200000F016FBE7
:101E2000290000F015FB32BDB4AD050084DA0500D1
:101E300080B500220A21FFF777FF02BD10B504002C
:101E4000200000F00DFB5C2803D1200000F00EFB09
:101E500000E0002010BD80B500220421FFF764FFE0
:101E600002BD80B500220621FFF75EFF02BD10B55E
:101E70000400200000F0F4FA672803D1200000F0ED
:101E8000F5FA00E0002010BD80B500220421FFF724
:101E90004BFF02BD10B50400200000F0E1FA5D2800
:101EA00003D1200000F0E2FA00E0002010BD80B570
:101EB00000220421FFF738FF02BD80B50022062171
:101EC000FFF732FF02BD000038B504000D0020000E
:101ED000FFF7E2FE854206D3B02206490648FFF727
:101EE000EFFEAFF30080200000F0C5FA290000F0FB
:101EF000C4FA32BD24AD05007CDA050080B514219A
:101F0000FFF7C0FE02BD80B50621FFF7BBFE02BD94
:101F100080B50821FFF7B6FE02BD80B50621FFF7A8
:101F2000B1FE02BD80B50821FFF7ACFE02BD80B551
:101F3000102100F0AAFA02BD80B50068FFF719FC75
:101F400002BD000038B504000D002000FFF7F4FFCB
:101F5000854206D3B02206490648FFF7B1FEAFF32B
:101F60000080200000F096FA290000F095FA32BDBA
:101F700064AF05009CDA050080B5042100F094FAF6
:101F800002BD80B50068FFF7F4FB02BD0A68036874
:101F90009A4201D20800FFE7704780B500F089FA45
:101FA00002BD04E010F8013B6BB1491C521E52B156
:101FB0000B7890F800C09C45F4D002D24FF0FF306F
:101FC0007047012070470020704780B5002206212D
:101FD000FFF79DFB02BD001D704780B550F8210042
:101FE00000F069FA02BD38B50C0000F065FA050092
:101FF000280000F069FA210089B280B2814205D23E
:10200000A4B205EB040000F05FFA00E0002080B20B
:1020100032BD0068704780B50068FFF7AAFB02BDBB
:10202000001D704710B500EB81042000FFF7F1FFA1
:10203000204410BD10B5040089B22000FFF7D3FF83
:10204000010089B20C4480B2002804D02000FFF7C0
:10205000E0FF204400E0002010BD90F90000704730
:102060000CB480B502AA03689B68984702BC5DF86F
:102070000CFB08B400B5110001AA03689B689847DF
:102080005DF808FB016070477CB504000D0029680D
:10209000684600F01BFA0600286800F019FA3200C2
:1020A0000100200000F02AFA73BD80B5002100F085
:1020B00032FA002801D1012000E00020C0B202BDA8
:1020C00038B50400200000F030FA002809D02000C4
:1020D00000F02BFA0500200000F02CFA290000F097
:1020E0002DFA200032BD10B50400200000F0B8F930
:1020F000082803D1200000F0B9F900E0002010BD4D
:1021000080B500F023FA00F025FA02BD80B5002268
:102110000421FFF74AFB02BD80B500220821FFF72A
:102120009DFD002801D0012000E00020C0B202BDCA
:1021300080B500220A21FFF791FD002801D001207F
:1021400000E00020C0B202BD80B500220C21FFF7E4
:102150002CFB02BD80B500220621FFF726FB02BD45
:1021600038B50400200000F0E0F90500200000F080
:10217000F5F900210160280032BD7CB504000D0096
:102180002968684600F0A2F90600286800F0EAF91C
:1021900032000100200000F0FBF973BD80B5002182
:1021A00000F003FA002801D1012000E00020C0B2B5
:1021B00002BD38B50400200000F001FA002809D063
:1021C000200000F0FCF90500200000F0FDF92900D6
:1021D00000F0B4F9200032BD10B50400200000F07A
:1021E0003FF9112803D1200000F040F900E0002061
:1021F00010BD80B50421FFF745FD02BD80B500F09C
:10220000E7F900F0E9F902BD38B50400200000F05C
:10221000D6F90500200000F0E3F900210160280054
:1022200032BD7CB504000D002968684600F04EF907
:102230000600286800F0D8F932000100200000F004
:10224000E9F973BD80B5002100F0F1F9002801D152
:10225000012000E00020C0B202BD38B5040020001B
:1022600000F0EFF9002809D0200000F0EAF905009D
:10227000200000F0EBF9290000F060F9200032BDE9
:1022800010B50400200000F0EBF8092803D120006D
:1022900000F0ECF800E0002010BD80B500F0DAF9A5
:1022A00000F0DCF902BD000080B59FED030A0421B7
:1022B00000F0D8F901BD00BF0000000038B50400EF
:1022C000200000F0BEF90500200000F0E5F9002133
:1022D0000160280032BD0078704710B5040089B253
:1022E0002000FFF780FE010089B20C4480B2002874
:1022F00004D02000FFF78DFE204400E0002010BD38
:1023000080B589B200F0CCF902BD10B5040089B2E5
:102310002000FFF768FE010089B20C4480B200285B
:1023200004D02000FFF775FE204400E0002010BD1F
:1023300010B5040089B22000FFF755FE010089B2F4
:102340000C4480B2002804D02000FFF762FE204435
:1023500000E0002010BD10B5040089B22000FFF796
:1023600042FE010089B20C4480B2002804D0200053
:10237000FFF74FFE204400E0002010BD704770477B
:1023800037B504460D46AFF300800020009002AB45
:102390002A462146054878441230FBF779FC054669
:1023A0002046AFF30080284603B030BDB5AA000038
:1023B0000068704780B500F086F902BD80B500F076
:1023C00083F902BD704710B5040089B22000FFF701
:1023D0000AFE010089B20C4480B2002804D020001B
:1023E000FFF717FE204400E0002010BD10B50400E8
:1023F00089B22000FFF7F7FD010089B20C4480B2DA
:10240000002804D02000FFF704FE204400E0002054
:1024100010BD10B5040089B22000FFF7E4FD0100F3
:1024200089B20C4480B2002804D02000FFF7F1FDEF
:10243000204400E0002010BD80B589B200F045F9CD
:1024400002BD80B50068FFF794F902BD001D70471A
:1024500010B500EB81042000FFF7DBFD204410BD28
:1024600080B500220A21FFF7F9FB02BD80B50C21DF
:1024700000F03EF902BD001D704710B500EB81046D
:102480002000FFF7C6FD204410BD80B589B200F0E2
:1024900034F902BD001D704710B500EB8104200027
:1024A000FFF7B7FD204410BD80B589B200F038F9C0
:1024B00002BD001D7047704710B504002000FFF7F3
:1024C00077FF4042204410BD00887047016070478C
:1024D00010B50122052103681B68984701000520FB
:1024E000FDF7BDFF0400002C05D0052100222000CF
:1024F00000F02AF900E00024200010BD38B50400E7
:102500000D00100000F053F902002900200000F037
:102510004FF9200032BD80B500F04EF9002801D1FE
:10252000012000E00020C0B202BD80B500F04EF9ED
:10253000006802BD80B500F04DF902BD80B5020013
:102540001068126812685268904701BD80B5FFF7A5
:10255000ECFF02BD80B500F03EF902BD80B500F091
:102560003EF902BD10B50422242103681B68984778
:1025700001002420FDF773FF0400002C05D0242166
:102580000022200000F0E0F800E00024200010BD50
:1025900038B504000D00100000F009F90200290010
:1025A000200000F01EF9200032BD80B500F01DF9BA
:1025B000002801D1012000E00020C0B202BD80B59A
:1025C00000F01DF9006802BD80B500F01CF902BDE5
:1025D00080B5FFF7F4FF02BD80B500F015F902BD2C
:1025E00080B500F015F902BD10B50422042103687E
:1025F0001B68984701000420FDF731FF0400002C00
:1026000005D004210022200000F09EF800E0002404
:10261000200010BD38B504000D00100000F0C7F810
:1026200002002900200000F0F5F8200032BD80B53E
:1026300000F0F4F8002801D1012000E00020C0B231
:1026400002BD80B500F0F4F8006802BD80B500F06E
:10265000F3F802BD80B5FFF7F4FF02BD80B500F0CE
:10266000ECF802BD10B52DED028B0400B0EE408AEF
:1026700089B22000FFF7B7FC010089B2002906D01B
:1026800080B2204400F0DDF8B0EE408AFFE7B0EE03
:10269000480ABDEC028B10BD80B500F0D5F802BD34
:1026A00010B5040089B22000FFF79DFC010089B23B
:1026B0000C4480B2002804D02000FFF7AAFC20447C
:1026C00000E0002010BD7047704710B5040089B2CB
:1026D0002000FFF788FC010089B20C4480B200287A
:1026E00004D02000FFF795FC204400E0002010BD3E
:1026F00080B589B200F0AAF802BD10B5040089B215
:102700002000FFF770FC010089B20C4480B2002861
:1027100004D02000FFF77DFC204400E0002010BD25
:1027200010B5040089B22000FFF75DFC010089B2FA
:102730000C4480B2002804D02000FFF76AFC20443B
:1027400000E0002010BD000062F30F2262F31F4280
:10275000401810F0030308D0C91A1FD3DB0748BF85
:1027600000F8012D28BF20F8022D130030B41446C4
:102770001546103928BF20E93C00FAD8490728BF80
:1027800020E90C0048BF40F8042D890028BF20F83C
:10279000022D48BF00F8012D30BC7047C91818BF82
:1027A00000F8012DCB0728BF00F8012D70477047B6
:1027B00080B500F05EF802BD80B5FFF7B6FE0028D8
:1027C00001D0012000E00020C0B202BD80B500F0C1
:1027D0005DF802BD704780B500F05AF802BD001DDB
:1027E000704780B500F055F802BD80B5FFF7E7FEF1
:1027F000002801D0012000E00020C0B202BD80B559
:1028000000F054F802BD704780B500F051F802BDE9
:10281000001D704780B500F04CF802BD80B5FFF791
:1028200010FF002801D0012000E00020C0B202BD4E
:1028300080B500F04BF802BD704780B500F048F855
:1028400002BD90ED000A7047001D704710B50400EE
:1028500089B22000FFF7C7FB010089B20C4480B2A7
:10286000002804D02000FFF7D4FB204400E0002023
:1028700010BD32B50400100000F02BF86B460200CA
:102880002900200000F026F8200032BD001D70470E
:10289000704732B50400100000F01BF86B460200D0
:1028A0002900200000F025F8200032BD001D7047EF
:1028B000704732B50400100000F00BF86B460200C0
:1028C0002900200000F024F8200032BD001D7047D0
:1028D0007047704738B5040010001D00FFF7F9FF7E
:1028E00000682060280000F022F800686060200086
:1028F00032BD38B5040010001D00FFF7EAFF006884
:102900002060280000F014F800686060200032BDEC
:1029100038B5040010001D00FFF7DBFF00682060E1
:10292000280000F006F800686060200032BD7047A3
:10293000704770471CB504460020DFF84017C4E913
:102940000001CDE900000322694604F1080000F00F
:10295000F1FB204616BD000070B52DED048B054639
:102960000E4688B0B0EE408AF0EE608A002105F194
:10297000080000F0EEFB7168032909D013220FF262
:1029800070710FF26470FFF79BF9AFF300804EE0B7
:1029900053EC182B0020DFF8D816FCF74BFA41EC6B
:1029A000190BB0EE490AF0EE690A00F0F3FB8DED69
:1029B000040B324604A902A800F0F2FB7468012C53
:1029C0009FED8B8B11DB366896ED000B51EC100BF5
:1029D00053EC102BFCF72EFA53EC182BFCF752FE9D
:1029E0000836641E41EC180BEED1B0EE480AF0EE4A
:1029F000680A00F0F3FB8DED060B06AA02A96846F3
:102A000000F06DFC694605F1080000F086FC01212C
:102A1000684600F09EFB012102A800F09AFBB0EE90
:102A2000490AF0EE690A00F0AFFB85ED000B08B033
:102A30002846BDEC048B70BD10B52DED068B044609
:102A400082B084ED000B0020CDE90000B0EE418A99
:102A5000F0EE618AB0EE429AF0EE629AB0EE43AACE
:102A6000F0EE63AA0322694604F1080000F062FB5D
:102A7000A06880ED008B80ED029B80ED04AB02B07E
:102A80002046BDEC068B10BD10B52DED0A8B04461B
:102A9000B0EE408AF0EE608A94B09FED550B84ED65
:102AA000000BB0EE41BAF0EE61BAB0EE429AF0EE31
:102AB000629A8DED000B0322694604F1080000F0D4
:102AC00039FB9FED99AB53EC182B51EC1A0BFCF72B
:102AD000B1F941EC1C0BB0EE4C0AF0EE6C0A00F0C0
:102AE00059FBB0EE408AF0EE608AB0EE4C0AF0EE90
:102AF0006C0A00F049FB9FED3E3B9FED3D2BB0EE95
:102B0000481AF0EE681A0CA8FFF796FF53EC1B2B3F
:102B100051EC1A0BFCF78EF941EC1B0BB0EE4B0A93
:102B2000F0EE6B0A00F036FBB0EE408AF0EE608A01
:102B3000B0EE4B0AF0EE6B0A00F026FB9FED2C3B4B
:102B4000B0EE482AF0EE682A9FED291B08A8FFF78F
:102B500073FF53EC192B51EC1A0BFCF76BF941EC9A
:102B6000190BB0EE490AF0EE690A00F013FBB0EE63
:102B7000408AF0EE608AB0EE490AF0EE690A00F091
:102B800003FBB0EE483AF0EE683A9FED192B9FED4B
:102B9000181B10A8FFF750FF014608AA04A800F070
:102BA0002BF80CAA04A9684600F026F89DED000B4E
:102BB00084ED000B02A904F1080000F0AEFB012136
:102BC00002A800F0C6FA012106A800F0C2FA01210D
:102BD00012A800F0BEFA01210AA800F0BAFA0121F9
:102BE0000EA800F0B6FA14B02046BDEC0A8B10BD5A
:102BF000000000000000000070B52DED028B8AB0CF
:102C000004460D461646FFF795FE06F1080105F14C
:102C1000080000F095FBD5E90023D6E90001B0EEED
:102C2000408AF0EE608AFCF705F953EC182BFCF7AC
:102C300051FBC4E9000106F10802294604A800F08E
:102C4000AFFA05F10802314606A800F0A9FA06AA73
:102C500004A902A800F0B0FB06F1080205F1080182
:102C600008A800F0CBFB08AA02A9684600F0A4FB64
:102C7000694604F1080000F050FB0121684600F0AD
:102C800068FA012108A800F064FA012102A800F006
:102C900060FA012106A800F05CFA012104A800F006
:102CA00058FA0AB0BDEC028B70BD38B584B004464A
:102CB0000D46FFF73FFE95ED000BDFF8C41384EDE2
:102CC000000B0020CDE9020105F1080202A96846C7
:102CD00000F066FA694604F1080000F01EFB0121CD
:102CE000684635E010B504462DED028B04F108016D
:102CF00004F1080000F024FBB0EE408AF0EE608A98
:102D000094ED000B53EC102B51EC100BFCF792F8E8
:102D100053EC182BFCF7B6FCBDEC028B41EC100B0E
:102D2000BDE8104000F05ABA000000000000E03F8B
:102D300038B584B004460D466846FFF7B6FF28460E
:102D4000FFF7D0FF6946204600F0A0F9012102A854
:102D500000F0FFF905B030BD80B54A68032A04D100
:102D6000BDE80440083000F0ABBB81220FF2803197
:102D70000FF27430FEF7A4FFAFF3008001BD000036
:102D80002DE9F84F2DED068B0D4684B00446032344
:102D90000322002100F09EFB074627609FEDB59BB4
:102DA000A86895ED000B90ED00AB53EC102B51ECA7
:102DB000100BFCF73FF80646884653EC1A2B51ECF3
:102DC0001A0BFCF737F832464346FCF75BFC53EC32
:102DD000192BFCF72FF89FEDAB8B53EC182BFCF75E
:102DE00051FC41EC1A0B38690228A4BF204600F0C0
:102DF000AFFB2168086880ED00ABAE68D6E9002320
:102E0000D6E90201FCF716F807468946D5E9002302
:102E1000D6E90401FCF70EF802460B46384649464F
:102E2000FCF758FA53EC192BFCF704F841EC1A0B99
:102E3000206801690229A4BF204600F089FB2068B0
:102E4000016881ED02ABAE68D6E90023D6E9040142
:102E5000FBF7F0FF07468946D5E90023D6E90201D2
:102E6000FBF7E8FF3A464B46FCF70CFC53EC192BFA
:102E7000FBF7E0FF41EC1A0B206801690229A4BFAF
:102E8000204600F065FB2068016881ED04ABD5F8B1
:102E900008802668D8E90023D8E90201F768FBF723
:102EA000C9FF82468B46D5E90001D8E90423FBF728
:102EB000C1FF52465B46FCF7E5FB53EC192BFBF7D1
:102EC000B9FF41EC1A0B30690228A4BF204600F07C
:102ED0003FFB2168086800EBC700012380ED00ABD1
:102EE00001222146684600F04EFBA86895ED000BD4
:102EF00090ED02AB53EC102B51EC100BFBF79AFF4B
:102F000006460F4653EC1A2B51EC1A0BFBF792FFB7
:102F100032463B46FCF7B6FB53EC192BFBF78AFF16
:102F200053EC182BFCF7AEFBCDE9020102A9684671
:102F300000F032FB022301222146684600F023FB09
:102F4000AE68D6E90223D6E90401FBF773FF074612
:102F50008946D5E90023D6E90001FBF76BFF02465D
:102F60000B4638464946FCF7B5F953EC192BFBF7ED
:102F700061FFCDE9020102A9684600F00DFB0023C4
:102F800002222146684600F0FEFAAE68D6E9002328
:102F9000D6E90401FBF74EFF07468946D5E9002331
:102FA000D6E90201FBF746FF02460B463846494682
:102FB000FCF790F953EC192BFBF73CFFCDE902012C
:102FC00002A9684600F0E8FA012302222146684679
:102FD00000F0D9FAAE68D6E90223D6E90401FBF77E
:102FE00029FF07468946D5E90023D6E90001FBF70A
:102FF00021FF3A464B46FCF745FB53EC192BFBF7F8
:1030000019FFCDE9020102A9684600F0C5FA0223C2
:1030100002222146684600F0B6FAA86895ED000B3A
:1030200090ED04AB53EC102B51EC100BFBF702FFAF
:1030300004460D4653EC1A2B51EC1A0BFBF7FAFE23
:1030400022462B46FCF71EFB53EC192BFBF7F2FE36
:1030500053EC182BFCF716FBCDE9020102A96846D8
:1030600000F09AFA04B0BDEC068BBDE8F18F0000C9
:103070000000E03F00000000000000400000F03FC2
:103080000000F0BF000000000000F0BF38B52DEDDB
:10309000020B84B004460D46FFF74CFCD5E9000155
:1030A000DDE90423FCF788F9C4E900010021684642
:1030B00000F04FF8AA68E9680123684600F081FA39
:1030C00004AA694602A800F00AF902A92046FFF7FF
:1030D00043FE012102A800F03CF80121684600F0FF
:1030E00038F807B030BD000074657374000000004C
:1030F000443A5C757365725C626163685C446576D2
:10310000656C6F706D656E745C6E52463532333827
:10311000325C64312D6E72662D312E302E305C6241
:103120006172735C5175617465726E696F6E2E6346
:103130007070000070B50D4604461646002100F080
:1031400008F800232A463146204600F03AFA204685
:1031500070BD10B5044600291EBF2068002800F08D
:103160004DFA00206060206010BD41EC100B01BDE5
:1031700080B551EC100B00F047FAF6E780B551EC42
:10318000100B00F0B9FAF0E780B551EC100B00F02D
:10319000FBFCEAE780B551EC100B00F0F7FCE4E72C
:1031A0002DE9F041154688466968044600F0F0FCB8
:1031B000002600270DE028683844D8E90023D0E92C
:1031C0000001FBF737FE22683A44761CC2E9000191
:1031D000083760688642EED3BDE8F08151EC100BF1
:1031E00000B500F003F841EC100B00BD40F2FF7C8D
:1031F0000B0D4DD0634566D230B421EA035141F442
:10320000801103F2FD3C5FEA5C0C01D300184941D8
:10321000890041EA907180004FF440140023E202DB
:10322000D50AB1F5100107D46D081DD2091B641928
:1032300000184941491BF7D56D080AD20919641BCA
:1032400000184941491BEFD56D08F7D301E052083A
:1032500017D0C01861419B1AAC4100184941801A2F
:10326000A941F4D452080AD0C01AA1419B186C415C
:1032700000184941801AA941E9D45208F4D15B1CD5
:103280006C4161084FEA330001EB0C5130BC7047D0
:1032900050EA0103FBD030B4B1FA81F311B9B0FAAE
:1032A00080F41B190B3BB3F120042FBF00FA04F18B
:1032B0009940C3F1200420FA04F438BF2143984018
:1032C000D3F101039DE7634514BF50EA410CDEE7EB
:1032D00011F5801FDBD8D943FCF7C1B970472DE940
:1032E000F0410D4606466968904600F051FC002406
:1032F00000270DE028683844D8E90023D0E9000110
:10330000FCF75AF832683A44641CC2E900010837F5
:1033100070688442EED3BDE8F08138B504460D46AE
:10332000AC420AD00121FFF714FF28682060002179
:10333000686860602846FFF70CFF204632BD000039
:103340002DE9F04106460C462DED028B7068616850
:10335000884206D0322216491648FEF7B1FCAFF378
:1033600000803768766800259FED0F8BA84611E036
:1033700020684044D7E90023D0E90001FBF75AFD5B
:1033800053EC182BFCF77EF941EC180B6D1C083739
:1033900008F10808B542EBD3B0EE480AF0EE680A2F
:1033A000BDEC028BBDE8F0810000000000000000D1
:1033B00034B90500ACDA05002DE9F0410F460446AA
:1033C0007968154600F0E4FB0026B04610E0386846
:1033D0004044761CD0E9002328684044D0E900012D
:1033E000FCF750F92268424408F10808C2E90001DC
:1033F00060688642EBD3BDE8F08100002DE97043A0
:103400000E46044670681546032804BF6B68032BFC
:1034100006D03F2228492948FEF752FCAFF300802E
:103420000321204600F0B4FB2D6836682468D6E9F5
:103430000223D5E90401FBF7FDFC80468946D6E965
:103440000423D5E90201FBF7F5FC02460B46404692
:103450004946FBF73FFFC4E90001D6E90423D5E95B
:103460000001FBF7E7FC80468946D6E90023D5E951
:103470000401FBF7DFFC02460B4640464946FBF7DA
:1034800029FFC4E90201D6E90023D5E90201FBF7CF
:10349000D1FC80468946D6E90223D5E90001FBF735
:1034A000C9FC02460B4640464946FBF713FFC4E9F8
:1034B0000401BDE8708300BF80B90500B4DA0500DF
:1034C00010B504468C4203D00A68496800F06CFBD2
:1034D000204610BD70B514461C4A054610781E469D
:1034E00010B100231370536039B1022901D017D3F2
:1034F0002AE09068401C906026E09068401C906034
:10350000D068401CD060D068401ED060142000F00D
:103510006BFBD0B132462146BDE8704000F076BB6F
:103520009068401E9060D068401CD060D068401EFB
:10353000D0602C6834B101212046FFF70AFE2046F6
:1035400000F05CF800202860002070BDD82A002020
:1035500038B5044620680169012913D0C368826820
:1035600000212046FFF7B6FF05462068854204D0BB
:1035700002684168284600F017FB20680169491E6F
:103580000161256031BD30B40C68E568016005FB60
:103590000232426030BC704738B505460C46286898
:1035A00001680A69022AA8BFFFF7D2FF286894EDD4
:1035B000000B016868680A6802EBC00080ED000B30
:1035C00032BDF8B50C00054616461F4615D0B4F1BD
:1035D000005F01D3FAF7A0FAE00000F005FB2860D5
:1035E000002118B196ED000B80ED000B491C08304E
:1035F000A14206EBC706F4D36C60F1BD002818BFEA
:1036000000F012BB70470000D0B52DED048B41ECEB
:10361000180B48004015401C01D1090319D151EC89
:10362000180B20F0000221F000430020834208BF65
:1036300082420ED0C80F1ABF43EC182B0824002476
:1036400051EC180B00224FF07953FBF745FD05D2E2
:1036500034BB51EC180BBDEC048BD0BD9FED229B0D
:1036600051EC190B53EC182BFBF734FE06460F46B2
:1036700053EC182B51EC190BFCF704F832463B467F
:10368000FBF7D8FBFFF7B2FD41EC190B51EC180B1F
:10369000174A184BFBF720FD07D253EC192B0FE00C
:1036A00081F0004141EC180BD3E701220D4BFBF7F1
:1036B00013FD0ED284F0020451EC190B53EC182BBD
:1036C000FBF77AFEBDEC048B2246BDE8D04000F04B
:1036D000E3BAFBF7C4FFBDEC048B4FF0FF306FF093
:1036E0000041D0BD0000F03F000000000000F03FAE
:1036F000CE3B7F669EA0E63F41EC100B480080B5B4
:103700004015401C0ED148004015401C01D1090352
:1037100005D151EC100BC80F18BF9FED080B51ECF1
:10372000100B04BD002100910022034B51EC100B43
:1037300000F0B6FB04BD00BF0000F03F0000000039
:1037400000000000F8B52DED068B41EC180B154676
:1037500053EC182BDFF8A003DFF8A013FBF76AFB8C
:1037600041EC190B21F00041DFF89423DFF894338A
:10377000FBF7B2FC6AD253EC192B9FEDB90B03F0A7
:10378000004251EC100B0C46144353EC102B51EC3F
:10379000190B2346FBF776FFFBF76CFD040051D0B5
:1037A000FBF786FD0022D84BFBF744FB41EC190BDD
:1037B00053EC192B4FF0A040D449FBF73BFB0246DA
:1037C0000B4651EC180BFBF785FD06460F4653ECF4
:1037D000192B4FF0C040CE49FBF72CFB02460B469D
:1037E00030463946FBF776FD06460F4653EC192B5B
:1037F0004FF00050C749FBF71DFB02460B46304611
:103800003946FBF767FD06460F4653EC192B00209F
:10381000C149FBF70FFB02460B4630463946FBF722
:1038200059FD06460F4653EC192B4FF00050BB498B
:10383000FBF700FB02460B4630463946FBF74AFDD4
:1038400041EC180B04F003046519BAE051EC180BB5
:1038500048004015401C51EC180B0DD14800401594
:10386000401C02D1090340F04181BDEC068B4FF0B2
:10387000FF306FF00041F4BD21F000410022914281
:1038800008BF904205D1002D00F030819FEDBC8B28
:103890002CE153EC192B9FED720B03F0004251EC1D
:1038A000100B0C46144353EC102B51EC190B234610
:1038B0000026FBF7E7FE4B0043EAD0734200B34219
:1038C00008BFB24241EC190B19D040F23344A4EBCB
:1038D0005352352A04DB00F0000001F000410CE0F7
:1038E000202A03DD203AD140914000E001D10020A0
:1038F00003E0012AA4BFD040904041EC190B51ECE9
:10390000190B20F0000231F0004308BFB24251D041
:1039100053EC192B00207C49FBF78CFA41EC1A0B75
:1039200053EC1A2B4FF0A0407849FBF783FA02467C
:103930000B4651EC180BFBF7CDFC06460F4653EC3B
:103940001A2B4FF0C0407249FBF774FA02460B463F
:1039500030463946FBF7BEFC06460F4653EC1A2BA1
:103960004FF000506B49FBF765FA02460B463046B4
:103970003946FBF7AFFC06460F4653EC1A2B0020E6
:103980006549FBF757FA02460B4630463946FBF7C6
:10399000A1FC06460F4653EC1A2B4FF000505F492E
:1039A000FBF748FA02460B4630463946FBF792FCD5
:1039B00041EC180B51EC190BFBF75CFC00F0030019
:1039C000451951EC180B21F0004100224FF07953BA
:1039D000FBF782FB05F0010405D2002C00F07E808D
:1039E0009FED678B7AE053EC182B51EC180BFBF72B
:1039F00021FA002C41EC190B36D053EC192B484816
:103A00004849FBF717FA484A484BFBF73BFE53EC93
:103A1000192BFBF70FFA464A464BFBF733FE53ECE4
:103A2000192BFBF707FA444A444BFBF72BFE53ECE8
:103A3000192BFBF7FFF9424A424BFBF723FE53ECED
:103A4000192BFBF7F7F96FF051023F4BFBF71AFE0A
:103A500053EC192BFBF7EEF900223C4B3AE000BF88
:103A6000000000000000E03F53EC182BFBF7E2F9E8
:103A700006460F4653EC192B35483649FBF7DAF961
:103A8000354A364BFBF7FEFD53EC192BFBF7D2F909
:103A9000334A344BFBF7F6FD53EC192BFBF7CAF90D
:103AA000314A324BFBF7EEFD53EC192BFBF7C2F911
:103AB0002F4A304BFBF7E6FD53EC192BFBF7BAF915
:103AC0002D4A2E4BFBF7DEFD32463B46FBF7B2F9A3
:103AD00053EC182BFBF7D6FD41EC180BA80705D5C6
:103AE00051EC180B81F0004141EC180B51EC180B14
:103AF000BDEC068BF4BD000083C8C96D305FE43FA8
:103B00000000A0FFFFFFDF410000303EFB21B94174
:103B1000B410114026A6513E5C14D33C9A833B3B23
:103B200009260A1039BA213E3BA861C6F97D92BE2A
:103B300063AC30909F01FA3EF6FB51166CC156BF44
:103B4000B10255555555A53FFFFFDFBF0000F03FBF
:103B5000B08F2FC310D8E53D8F0C73A1E1E55ABE9D
:103B60004DADE44FE31DC73E3EE3B519A0012ABFAA
:103B7000FAF010111111813F425555555555C5BFE9
:103B8000000000000000F03F0122DBE50022D9E543
:103B900038B50D4604460021FFF7DBFA29462046DA
:103BA00000F08AFB204632BD70B504460D466068C1
:103BB000A84216460BD122680021814213D296ED0D
:103BC000000B82ED000B491C08360832F5E7012195
:103BD0002046FFF7BEFA324629462046BDE870402F
:103BE0000123FFF7EEBC70BD10B5044601E000F004
:103BF0007CFB2046F9F7B8FB28B903480068002889
:103C0000F5D08047F5E710BD8847002070B50D4618
:103C10001646044606FB05F1FFF7BAFF01202061B6
:103C2000A560E660204670BDF9F7F9BC443A5C75C2
:103C30007365725C626163685C446576656C6F7025
:103C40006D656E745C6E524635323338325C4C6949
:103C5000625C74666C6974652D6D6963726F2D3278
:103C600034303232325C74656E736F72666C6F77AB
:103C70005C6C6974655C6D6963726F5C6B65726EB8
:103C8000656C735C66756C6C795F636F6E6E656393
:103C90007465642E63630000D0B52DED048B41EC98
:103CA000180B144653EC182B00206C4900F020FB35
:103CB00008BF9FED558B00F0838051EC180B544AE0
:103CC000544BFBF721FA1DD89FED539B53EC182B57
:103CD00051EC190BFBF7AEF80022514BFBF7D2FC6D
:103CE00006460F4653EC182B51EC190BFBF7CAFC98
:103CF00002460B4630463946FBF75EFB41EC180B9B
:103D000044F0010451EC180B21F0004101224FF066
:103D10007953FBF7F9F953D853EC182B51EC180BE6
:103D2000FBF788F841EC190B53EC182BFBF782F8E2
:103D300006460F4653EC192B3A483B49FBF77AF8F5
:103D40003A4A3B4BFBF79EFC53EC192BFBF772F8FE
:103D5000384A394BFBF796FC32463B46FBF76AF88C
:103D600053EC182BFBF78EFC06460F4653EC192B31
:103D700032483349FBF75EF8324A334BFBF782FC9B
:103D800053EC192BFBF756F8304A314BFBF77AFC12
:103D900053EC192BFBF74EF82E4A2F4BFBF772FC16
:103DA00053EC192BFBF746F800222C4BFBF76AFC6F
:103DB00002460B4630463946FBF7FEFA41EC180B3B
:103DC000A00705D551EC180B81F0004141EC180B10
:103DD00014F007020BD000BF21A303EBC20251EC89
:103DE000180B53681268FBF74DFC41EC180B2007C9
:103DF00005D551EC180B81F0004141EC180B51EC4A
:103E0000180BBDEC048BD0BD182D4454FB21E93FA9
:103E100057CD9E5E1426D13FAA4C58E87AB6FB3F98
:103E20000000F0BF845D57134B57B03FB2934C195D
:103E3000ED5EE43FBEDE02B90240F83FDE39028F9C
:103E4000C7C0743F8AAB1283000CC83F24D7E50873
:103E5000B6D8F03F0F34580E5895FD3F0000F03FA4
:103E6000000000000000000066732D3852C1E03FE2
:103E7000182D4454FB21F93F66732D3852C1F03F91
:103E8000182D4454FB21F93F66732D3852C1004070
:103E9000182D4454FB2109403FD038C6A6F10440F8
:103EA000F8B52DED0A8B41EC1A0B48004015109D1A
:103EB000401C43EC182B24D051EC1A0B21F000418C
:103EC0000022914208BF90421BD051EC180B4800D1
:103ED0004015401C15D051EC180B31F0004108BFC3
:103EE00090420ED051EC1A0BDFF87433FBF7F4F864
:103EF00080F0B18051EC180B9FED870B01F0004270
:103F0000BAE051EC1A0B48004015401C02D10903DD
:103F100040F0A08151EC180B48004015401C01D125
:103F200009035DD151EC180B20F0000221F0004391
:103F30000020834208BF824208D151EC1A0B48008E
:103F40004015401C4CD109034AD10DE048004015F2
:103F5000401C12D1090310D151EC1A0B4800401536
:103F6000401C3DD109033BD1FBF779FBBDEC0A8B2B
:103F70004FF0FF306FF00041F4BD51EC1A0B21F00F
:103F8000004100220023994208BF90422BD151ECFE
:103F9000180B4800400D05EB000237D151EC180B0F
:103FA00021F00041994208BF984206D02A4651ECC0
:103FB000180BFBF7C1F841EC180B51EC180B20F073
:103FC000000221F000430020834208BF824205D056
:103FD00048004015401C03D1090301D1FBF746FB03
:103FE00051EC180B38E151EC1A0B48004015401CFD
:103FF0002AD1090328D153EC1A2B51EC180BBDEC34
:104000000A8B01B0BDE8F040FAF714BF002AC5DD05
:1040100040F2FF7082420FDB9FEDA50B51EC100BBD
:10402000084653EC182B03F00041084353EC102BC7
:10403000034643EC182BC0E76FF31E5141EA0251CF
:1040400053EC182B0B46F4E751EC180B9FED320B99
:1040500001F0004210E00122824BFBF755F811D825
:104060009FED930B51EC100B0A4651EC180BFBF72C
:10407000FDFA01F00040024351EC100BBDEC0A8B3D
:104080001146F4BD53EC1A2B77487849FAF7D2FE63
:1040900041EC100B53EC102B9FED759B03F000428D
:1040A00051EC190B0C46144353EC192B51EC100B2B
:1040B0002346FBF7E7FAFBF7DDF80446FBF7F8F8D1
:1040C00041EC1B0B53EC1B2B4FF078406A49FAF77D
:1040D000B1FE02460B4651EC1A0BFBF7FBF8064605
:1040E0000F4653EC1B2B65486549FAF7A3FE0246C1
:1040F0000B4630463946FBF7EDF841EC1A0B21F040
:10410000004100225F4BFAF7E7FF09D2B0EE48AA60
:10411000F0EE68AA56E000BF0000000000000000BA
:1041200053EC1A2B51EC1A0BFAF784FE41EC1B0BE3
:1041300053EC1B2B54485549FAF77CFE544A554B17
:10414000FBF7A0FA53EC1B2BFAF774FE41EC1C0BA7
:1041500053EC1B2B50485149FAF76CFE504A514B17
:10416000FBF790FA53EC1B2BFAF764FE53EC192B78
:10417000FBF788FA53EC1A2BFAF75CFE41EC190BAB
:1041800053EC1C2BFBF77EFA9FED47AB53EC1A2B3D
:10419000FBF778FA06460F4651EC1C0B53EC192B33
:1041A000FBF798F853EC1A2BFBF76CFA02460B4618
:1041B00030463946FBF700F953EC182BFAF73AFE74
:1041C00041EC1A0B51EC1A0B2A194800400D02EB76
:1041D00000031DD0002B1BDD40F2FF7083420DDB7E
:1041E0009FED330B51EC100B084653EC1A2B03F0E8
:1041F0000041084353EC102B034606E06FF31E51B9
:1042000041EA035153EC1A2B0B4643EC1A2B0EE0F8
:1042100051EC1A0B21F000410024A14208BFA0423A
:1042200005D051EC1A0BFAF787FF41EC1A0B51EC51
:104230001A0B20F0000221F000430020834208BF47
:10424000824205D048004015401C03D1090301D12A
:10425000FBF70CFA51EC1A0BBDEC0A8BF4BD000015
:1042600000C89CC000C89C40FE822B654715F73FE4
:10427000000000000000E03F422EE63FF2E4D5BC23
:10428000E7E84B3E0000903C112E5781A03F503F85
:104290005843128C8F71BC3F4BE8A541B752013F88
:1042A0000BBDF3DAE8708C3F000000000000F03F27
:1042B000000000000000F07F38B50C00054613D068
:1042C000B4F1005F01D3F9F727FCE000FFF78CFCA5
:1042D000286000210022002308B1C0E90023491C06
:1042E0000830A142F8D36C6031BDF9F715BC00006D
:1042F00090420CD141EA030C50EA4C0C07D0994291
:1043000005D14FF4001C1CEB410F38BF89427047A8
:1043100080B500F085FB01BDF7EE000A30EE200A03
:10432000F7EE000A80EE800A70470000F8B584B00E
:1043300006000F0014001D0097F91C00072829D162
:1043400040F202413000B26B904700280CD1DFF8F8
:104350005C0600902723DFF85826DFF85816300057
:104360007469A047012089E0A86240F20241300050
:10437000B26B904700280CD1DFF83C0600902B234D
:10438000DFF82C26DFF82C1630007469A0470120D6
:1043900074E0E86294F91C00072815D197F91C0015
:1043A000092810D097F91C0007280CD0DFF80C065C
:1043B00000903223DFF8F825DFF8F8153000746933
:1043C000A04701205AE01BE097F91C0094F91C104B
:1043D000884215D094F91C00039097F91C000290B4
:1043E000DFF8DC050190DFF8DC0500903423DFF80E
:1043F000C025DFF8D41530007469A04701203DE0E6
:1044000097F91C00072838D1E068002812D0002056
:104410000390E06802901AA00190DFF8B0050090C8
:104420003923DFF88C25DFF8A01530007469A04728
:10443000012023E04FF6FF700DF1010000F01EFB9C
:10444000AB6A02000021DFED0F0A47F6FF709FED17
:104450000E0A00F017FB684600F01AFBEB6A020038
:104460000021DFED080ADFF868059FED080A00F07B
:1044700009FBE068E861A0682862002005B0F0BD93
:104480003000000080000038A00020398000803714
:1044900080B50020FFF73CFF01BD80B50020FFF78D
:1044A0003BFF01BD2DE9F8432DED028B86B00400E2
:1044B0000D0090461F00109E330042462900200048
:1044C000FFF734FF002801D00120B7E195F91C0067
:1044D000092804D095F91C00072840F0758195F94A
:1044E0001C00072866D1E868002812D0002003903D
:1044F000E86802909BA00190DFF8D80400905B234D
:10450000DFF8AC24DFF8C01420006469A047012064
:1045100094E1D8F80C00002813D000200390D8F8BC
:104520000C0002908FA00190DFF8A00400905C23A3
:10453000DFF87C24DFF8901420006469A047012094
:104540007CE198ED020ADFEDC00AB4EE600AF1EEFC
:1045500010FA06DB98ED020ADFEDBC0A30EE200A05
:1045600005E09FEDBB0AD8ED020A30EE600ADFEDF0
:10457000B90AB4EE600AF1EE10FA1ADB00205FF01F
:104580007C51CDE90401D8F8080000F085FACDE9A6
:104590000201DFF844040190DFF8400400905E233C
:1045A000DFF80C24DFF8381420006469A0470120EC
:1045B00044E1B8E095F91C00092819D00920FCF75E
:1045C00021FB060095F91C00FCF71CFB03960290EA
:1045D000DFF810040190DFF8EC0300906023DFF8AF
:1045E000D023DFF8041420006469A047012025E1EE
:1045F00098F91C00072852D1D8F80C0010F5004F8C
:1046000015D0DFF8CC030390D8F80C000290DFF847
:10461000DC030190DFF8B40300906223DFF89023FD
:10462000DFF8A41320006469A047012006E198ED9B
:10463000020ADFED890AB4EE600AF1EE10FA06DB39
:1046400098ED020ADFED850A30EE200A05E09FEDC5
:10465000840AD8ED020A30EE600ADFED820AB4EE79
:10466000600AF1EE10FA19DB0020DFF88413CDE9BF
:104670000401D8F8080000F00FFACDE90201DFF8D4
:1046800074030190DFF8540300906423C84ADFF8F4
:10469000501320006469A0470120CFE043E098F95F
:1046A0001C00092815D00920FCF7ACFA050098F980
:1046B0001C00FCF7A7FA03950290CA480190C04875
:1046C00000906623BA4AC84920006469A0470120C7
:1046D000B4E0D8F80C0010F1800F11D07FF07F000B
:1046E0000390D8F80C000290C3480190B74800909E
:1046F0006723AF4AB44920006469A04701209DE0C8
:1047000098ED020ADFED580AB4EE600AF1EE10FAF5
:1047100009D0BA4800906823A54AA64920006469D8
:10472000A04701208AE095F91C0007281CD1A86841
:1047300000F0B2F904000D00386800F0ADF9220075
:104740002B00FAF777FB5FF01412AD4BFAF734FE4B
:1047500041EC100B01A916F1080000F0C1F9019815
:10476000F0606AE0300000006A4616F1080105209A
:1047700080460C009146A86800F08EF941EC110BC0
:104780004A4621004046B0EE418AF0EE618A0500BB
:104790000C009046386800F07FF941EC100B42465F
:1047A00021002800B0EE481AF0EE681A00F01AFA5C
:1047B0000098F0601F22F168052000F03EFA5FF0DB
:1047C000FF314843B06138E095F91C00012815D04D
:1047D0000120FCF717FA060095F91C00FCF712FA05
:1047E0000396029087480190764800908B23704A88
:1047F0007D4920006469A04701201FE098F91C0052
:10480000012815D00120FCF7FDF9050098F91C00DE
:10481000FCF7F8F9039502907A48019068480090F7
:104820008C23634A704920006469A047012005E099
:10483000386800F031F9C6E90001002006B0BDEC8F
:10484000028BBDE8F283000001000038000000B8D0
:10485000000000387012033301008037000080B779
:1048600000008037701283320000803B10B50400D6
:10487000A06B002801D1F9F74FF938212000A26B75
:10488000904710BD2DE9FF4106008846300000F03A
:1048900043FA0700404600F041FA012811D0404693
:1048A00000F03CFA0121039102903FA0019056488C
:1048B00000909A233E4A444930007469A047012081
:1048C0006EE0404600F032FA012811D0404600F078
:1048D0002DFA01210391029033A001904B480090E2
:1048E0009B23334A384930007469A047012057E0C0
:1048F00000224146380000F02DFA0500002D09D1B4
:10490000434800909D232A4A2A4930007469A047F1
:10491000012045E0280000F04CFA012809DA3D4862
:1049200000909E23224A234930007469A047012049
:1049300036E000224146380000F01FFA0400002C47
:1049400009D135480090A023194A1A4930007469EA
:10495000A047012024E0D8F80C00002809D12F48F6
:104960000090A223124A134930007469A047012025
:1049700016E0D8F80C00D8F810300090220029007A
:104980003000FFF78FFD0600290038003A68926971
:104990009047210038003A6892699047300040B251
:1049A00004B0BDE8F081000031000000B8CD050082
:1049B000F8B20500A0CD0500BCC60500C0BD0500CD
:1049C000F0D405009CD7050010CA05002CCA0500CC
:1049D0000080FFFF48CA0500A8D70500D0CD05001C
:1049E00060C80500B4D7050064CA05005CDA05009C
:1049F0000000F03EC0D7050064DA0500E0C60500FF
:104A00001400243F00D5050010D50500B0D10500E5
:104A1000C4D1050080CA0500D8D105009CCA050094
:104A200010EE100A0949B5EE400AD1F83CC0BCEBC3
:104A3000400FD1EC0D0AC0F00B80F1EE10FA4FF0F0
:104A4000000140F0B981B0EE600A70473CBC05003F
:104A50004FF0807C1CEB400F08D2004254BFB0EEF8
:104A6000420A31EE410A7AF501AE704704D8C042DD
:104A700002D3002000EE100A704700000048704783
:104A80009144050080B50093002300F005FA01BDB4
:104A9000004870479B440500C0F3C75181B1FF290E
:104AA00006D0C110400721F0E04101F1605170478C
:104AB00041020CBF40F4E0016FF00041002070475C
:104AC00000F0004100020AD0B0FA80FC00FA0CF0BD
:104AD00001F16051A1EB0C5101EBD0214005704771
:104AE000F8B52DED028BB0EE408AF0EE608A06003C
:104AF0000F0053EC182B00200021FFF7F9FB04D125
:104B0000002030600020386046E03800B0EE480AEF
:104B1000F0EE680AFAF79CFA53EC102B0020DFF84D
:104B2000E411FAF787F941EC100B00F083FA51EC2D
:104B3000100B00F083FA04000D00DFF8CC01002117
:104B40008D4204DB01DC844201D3F8F7E5FF5FF01E
:104B5000004000218D420CD184420AD1200029005E
:104B600002220023FAF72CF804000D003868401CDC
:104B700038605FF0004000218D4204DB01DC84429C
:104B800001D3F8F7C9FF386810F11F0F03DA0020CE
:104B90003860002400253460BDEC028BF1BD38B5CF
:104BA0002DED028BB0EE408AF0EE608A04000D001D
:104BB00051EC180B0122DFF85431FAF7A5FA01D9AC
:104BC000F8F7AAFF29002000B0EE480AF0EE680AC4
:104BD000FFF786FF2868002801D5F8F79DFFBDEC98
:104BE000028B31BD2DE9FF4180460E001700484879
:104BF0004849CDE9020153EC102B51EC110BFAF7A7
:104C000019F904000D000120D8F11F0810FA08F866
:104C10004046FAF74DFB22002B00FAF70BF9CDE9DD
:104C2000000102A9684600F037FA90ED000B390048
:104C30003000FFF7B4FFBDE8FF812DE9F041070028
:104C40000E0090460120B840401EFAF731FB0022CA
:104C50002E4BFAF7EFF804000D0001200021B8EB0D
:104C600007073A0000F026FA00F036FA22002B007F
:104C7000FAF7E0F804000D0001200021320000F0F6
:104C800019FA00F029FA02000B0020002900FAF7B7
:104C900093FB41EC100B00F049FA51EC100BFAF7C2
:104CA000E9FABDE8F081000010B52DED028B04009B
:104CB00000F070FAB0EE408AB0EE000A00F06AFA36
:104CC000F7EE000A80EE800A20EE088AB0EE480A6D
:104CD00000F0C0FA78EE400ABDEEC00A84ED000A8A
:104CE000B0EEE00ADFED060AB4EE600AF1EE10FA6B
:104CF00001D5012000E00020C0B2BDEC028B10BD48
:104D00006F12833A0000E041010000800000F03F94
:104D10000000C0FFFFFFDF41C06870470168002945
:104D200001D1002001E00068006870474168002957
:104D300001D1002001E0406800687047002806D4D7
:104D4000884204DA52F8200010F1010F01D15FF01F
:104D5000FF30704710B5040010000A68121D096882
:104D60000968FFF7EBFF0100002901D5002003E0EF
:104D7000200022685269904710BD10B50400100051
:104D80004A68121D49680968FFF7D8FF0100002929
:104D900001D5002003E0200022685269904710BD31
:104DA0000CB480B5080002A9FBF717FF01BC5DF841
:104DB0000CFB406900687047004248BFB1EE411AE1
:104DC00000EE211ABDEEC11A11EE10CAB8EEC11ADA
:104DD00001EE620A01EE430AB0EEC01AB4EE631AA5
:104DE000F1EE10FA614401F17F0113D420EE001AB4
:104DF00061EE042AB0EE623A01EE245A40EE052A32
:104E000072EEA52A00EE453A33EE253AC2EE832A29
:104E100060EEA20A19B3FF294FEAC15C00EE10CA86
:104E20000FD220EE200AB5EE400AF1EE10FA10EE95
:104E3000100A4FF0807C18BF1CEB400F3AF416AC00
:104E4000704701290BDB7F39FF294FEAC15C36BF70
:104E500000EE10CAB0EE420A60EE860AE1E77E314B
:104E600001294FEAC15CAABF00EE10CA30EEE00A89
:104E700060EEA60AD5E710EE90CA1CEB0C0F0042BC
:104E800054BFB0EE420A31EE410A28BFB1EE400AEB
:104E90007AF5ECAB70470000F8B52DED0A8B84B0C5
:104EA00015001E00149C614A121A01EE102AB8EE79
:104EB000C11A21EE008A47F6FF72101A01EE100A9D
:104EC000B8EEC11A61EE008A5848401A00EE100A86
:104ED000B8EEC00A20EE200A47F6FF70411A01EE34
:104EE000101AB8EEC11A61EE200A4FF4007038EEC5
:104EF000C81ADFED4C1A81EE219AB0EE001AC9EE05
:104F0000019A30EEC00ADFED480A80EE80AA5FF019
:104F10004740019046480090002760E000EE107A7C
:104F2000F8EEC00AB0EE480A00EE890A3100280007
:104F300000F094F9B0EE40BA00EE107AB8EEC00A74
:104F4000F0EE480A40EE090A30EEA90A31002800C6
:104F500000F084F9F0EE40BA781C00EE100AF8EE8A
:104F6000C00AB0EE480A00EE890A3100280000F0BD
:104F700075F9B0EE40CA2BEE0A0A00F06BF9F0EEBC
:104F800040AA2BEE0A0A00F065F90CEE0A0AF0EED0
:104F9000000A80EE200A00F05DF9B0EE40BA2BEE78
:104FA0008A0A00F057F93BEE400AF0EE000A80EE64
:104FB000200A00F04FF93AEEC00A8DED030A01A96C
:104FC00003A800F04EF9694600F057F990ED000A89
:104FD000BDEEC00A10EE100A24F817007F1CB7F5CA
:104FE000007F9BDBB0EE680A3100280000F036F944
:104FF00020EE0A0A00F02EF98DED020A01A902A89E
:1050000000F02FF9694600F038F990ED000ABDEE86
:10501000C00A10EE100AA4F8000404B0BDEC0A8B1C
:10502000F1BD00BF00000044000080470080FFFF8A
:1050300000FEFF4680B500F02DF901BDC1F30A5313
:1050400040F2FE329B1A24DDCA17C902D3F12003B5
:1050500041EA505141F0004104DDD94088185040E8
:105060001146704720330CDDC002C3F1200C01FA59
:105070000CFCD940D8406044801851415040514008
:10508000704740F2C1301B1803D0D04380F000417C
:10509000704700200021704738B504000D00D5E9A5
:1050A0000001D4E90023FAF717F801D22C00FFE73A
:1050B000200032BDD2B2203A22BF00FA02F1002015
:1050C00070475242D041D2F1200291404140D0403D
:1050D0009040414070470000CB17C01859415840DC
:1050E0005940DB07A1B1B1FA81F241409040C2F1D1
:1050F0002002D141414002F21D4243EA025CC30A50
:10510000420572F1004253EB41504CEBD121704704
:1051100050B1B0FA80F29040C4F2D011A1EB02522B
:1051200002EBD021194340057047000051EC100BF1
:1051300000B500F003F841EC100B00BD40F2FF7C1D
:105140001CEA115240F2FE33D21A18DD352A20DA59
:10515000B2F1150309DA6FEA4C53D340094201D585
:10516000401E59410020994370476FF00002DA4019
:10517000094202D5801851F100019043704750EA6E
:1051800041031CBF4FEA0C5101F1804138BF00219F
:105190000020704710EE100AB5EE400A4FF0807CF8
:1051A0001CEB400F42D2F1EE10FADFF8A4C0DCECA9
:1051B000090A45DD5FEAD05C2BD0ACF17E0CA0EB98
:1051C000CC5000EE100AB4EE600AF1EE10FA44BFC3
:1051D000ACF1010C20EE210A00EE90CAF8EEE00AD4
:1051E00070EE415A30EE016A85EE866A66EE066A16
:1051F00002EEA63A43EE263AB0EE650A03EEE60A60
:1052000020EE066A04EEE06A35EEC60A04EE200AD5
:10521000704720EE020A10EE100A4FEAD05CACF1A3
:105220007E0CA0EBCC50ACF1170CCAE707D80042BB
:1052300044BF6FF0004000EE100A3AF510AA704724
:10524000F6DB6FF00000C00500EE100A70470000AA
:10525000F8BB050080B500F04FF801BD80B5804770
:1052600001BD90ED000AD1ED000AB4EE600AF1EE46
:1052700010FA01D50800FFE7704791ED000AD0ED64
:10528000000AB4EE600AF1EE10FA01D50800FFE75B
:105290007047000051EC100B00B500F003F841EC32
:1052A000100B00BD40F2FF7C0CEA115240F2FE33BD
:1052B000D21A17DD352A1DDAB2F1150308DA6FEAC2
:1052C0004C53D34031EA5301C91899430020704729
:1052D0006FF00002DA4030EA5200801841F100011C
:1052E0009043704701F0004104BF41F07C5141F40C
:1052F000700100207047000010EE100AF44600F024
:1053000003F800EE100A6047C0F3C7527E3A09DD89
:10531000182A0CDA6FF07F41D14020EA5100401882
:105320008843704700F0004008BF40F07E5070474F
:10533000C0B2002801D0012000E0002070472DE914
:10534000FC4704000D001E000A9FDDF82C80DDF8EC
:105350003090DDF834A02560626014F1080064210B
:10536000FBF798FB5046C0B2FFF7E2FF020039009E
:105370003000FAF740FCE066CDF80080E36E2A00CA
:1053800014F1080114F1700000F0DEFA002084F836
:105390009000012084F891000020C4F894000020BF
:1053A000C4F898000020C4F89C0014F1700322682F
:1053B000E16E14F1A00000F0AFFC4946200000F0BF
:1053C00019F82000BDE8F68710B5040014F170004C
:1053D00000F01EFD002803D014F1700000F08AFBDD
:1053E00014F1A00000F0ADFC14F1700000F0CBFA55
:1053F000200010BD38B504000D00002114F1A000FC
:1054000000F004FD14F1A0006061DFF8D804E06151
:10541000DFF8D404A065DFF8D404E065E563DFF8C5
:10542000D004A064DFF8CC042063DFF8CC0420644F
:10543000DFF8C804E064002084F8910031BD2DE954
:10544000F14F86B05FF0000B01E01BF1010B0698F5
:10545000703000F057FC834580F2F38006980068B6
:10546000FBF76CFD5946FBF773FD00900098002890
:1054700001D1F8F751FB06980068FCF7BAFC0190DF
:105480000698C06EFAF7E9FF04900098FBF735FB29
:105490000390002475E031000198FCF7AFFC070091
:1054A0000698703000F0B4FC50F83B0061010844ED
:1054B00010F11C0206984168380000F0ABFC8046F1
:1054C000404640B2002878D10698703000F0A0FC29
:1054D00050F83B0061010844C06900287AD0D0F838
:1054E00014800026002700200290B8F1200F78D108
:1054F000280000F0DDFC00280BD0280000F0D8FCCC
:10550000FBF7C3FA0600280000F0D2FCFBF7B8FA5C
:1055100007002800FCF701FDFBF708FB8246280086
:10552000FCF7F6FCFBF702FB80460698703000F0B3
:105530006FFC50F83B00610100EB010948461C215B
:10554000FBF7A8FAC9F800A0C9F804800298C9F8C6
:105550001000C9F81460C9F818702800FCF7CEFCD8
:1055600000280DD02800FCF7C9FCFCF7CBF8002878
:1055700006D02800FCF7C2FCFBF7D8FAC9F80800EF
:10558000641C03988442BFF460AF0098FCF77FFB73
:105590002100FCF799FC05002800FCF724FC06001C
:1055A0000198FCF74EFF8642FFF475AF3100DFF83B
:1055B0005003FBF71BFB012044E0380000F07DFCAA
:1055C00000F090FC0100DFF83C03FBF70FFB4046C6
:1055D00040B237E03100DFF83003FBF707FB012072
:1055E00030E0280000F064FC002815D14146069800
:1055F0004068069A52681268926890470100002934
:1056000013D002AB049A2900FBF759FA01000800F5
:1056100040B2002812D17CE7404600F063FC010054
:10562000BA48FBF7E3FA01200CE0404600F05AFCD0
:105630000100B748FBF7DAFA012003E0080040B2A6
:1056400000E0002007B0BDE8F08FF8B50400216845
:10565000E06EFAF70EFB0100002907D1AD48FBF719
:10566000C5FA012084F891000120E2E014F17000F5
:1056700000F04FFB2000FFF7E2FE010049B20029D5
:1056800001D040B2D5E0002114F1A00000F0BEFB33
:1056900014F1700000F078F9010049B2002901D03E
:1056A00040B2C6E0012114F1A00000F0AFFB14F1FC
:1056B000700000F0A7F9010049B2002901D040B202
:1056C000B7E0022114F1A00000F0A0FB14F170007B
:1056D00000F09EFB14F1940302002168E06EFAF7DB
:1056E0001DFB010049B2002901D040B2A1E0D4F86D
:1056F000941014F1A00000F085FBE56E200000F08E
:1057000009FC810028002A68D2699047C4F89800F3
:10571000D4F89800002808D1200000F0FBFB81009D
:105720007D48FBF763FA012083E0002500E06D1C53
:10573000200000F0EFFB854224D2E66E200000F04E
:10574000F5FB2900FBF7C4FF070014F1700000F01F
:105750005FFB002100913B000200216830003668A9
:105760003668B047D4F8981041F82500D4F898006E
:1057700050F825000028DAD129006848FBF736FAEE
:10578000012056E0E56E200000F0DAFB81002800E1
:105790002A68D2699047C4F89C00D4F89C0000287D
:1057A00008D1200000F0CCFB81005D48FBF71EFA19
:1057B00001203EE0002500E06D1C200000F0C0FB51
:1057C000854224D2E66E200000F0C6FB2900FBF7DC
:1057D0007FFF070014F1700000F01AFB02000020A8
:1057E00000903B002168300036683668B047D4F836
:1057F0009C1041F82500D4F89C0050F825000028A2
:10580000DAD129004748FBF7F1F9012011E0200027
:1058100000F056F8010049B2002901D040B208E07A
:10582000012084F89000032114F1A00000F0EEFAAA
:105830000020F2BD10B5040094F99100002804D0B6
:105840003948FBF7D3F9012011E094F890000028C3
:1058500008D12000FFF7F9FE010049B2002901D06C
:1058600040B204E0002114F1700000F072F910BDA4
:1058700038B504000D00200000F04CFB854206D333
:10588000020029002948FBF7B1F9002003E0D4F811
:10589000980050F8250032BD38B504000D002000F6
:1058A00000F04EFB854206D3020029002048FBF79A
:1058B0009DF9002003E0D4F89C0050F8250032BD8B
:1058C00010B5040014F1700000F0E5F8010049B2D1
:1058D000002901D040B203E014F1700000F0B2F9E9
:1058E00010BD0000A14D05004DD205005FD205009E
:1058F00079CE050041D5050029D205003BD205002F
:105900002CC40500C8C10500E4C50500CCB90500DC
:10591000A0C70500C0C50500D4B60500B0C4050089
:1059200020B70500D8C4050098C10500D4C3050000
:1059300000C4050080B54169202901D1806902E0D9
:10594000406900F0CFFA02BD2DE9F04105000E00DC
:1059500014001F00DDF81880280000F007FBB54890
:1059600028606E60AC60EF600020286100206861F4
:10597000C5F81880002C03D02000FBF7DFFAE8619F
:105980002800BDE8F08170472DE9F84304006569FF
:10599000002600E0761CE069FBF7D5FA86422DD29E
:1059A00066613100A068FBF7B7F807005FF00008F8
:1059B000B845EFD2206950F836005FEA481100EB95
:1059C0000109206950F836005FEA48110844C369AC
:1059D0005869202803D0D9F81010002203E0D9F824
:1059E0001410D9F818201868002804D060681B68C3
:1059F0009847C9F80C0018F10108D9E76561002043
:105A0000BDE8F2832DE9F04704006569002600E057
:105A1000761CE069FBF797FA864238D2666131005E
:105A2000A068FBF779F807005FF0000805E0414641
:105A3000E068FAF7DDF918F10108B845E8D2206905
:105A400050F836005FEA48110144206950F83600EA
:105A50005FEA48121044D0F81C90D9F808000028DA
:105A6000E5D06068D9F8082090478246504640B299
:105A70000028DCD04846FFF75DFF4FFA8AFA53460C
:105A8000424601006C48FBF7B1F8012001E0656176
:105A90000020BDE8F0872DE9F0410400656900268B
:105AA00017E0206950F8360079010144206950F868
:105AB00036007A011044C269002A06D01069002815
:105AC00003D0C9686068126990477F1C4745E8D3D6
:105AD000761CE069FBF737FA864207D2666131002F
:105AE000A068FBF719F880460027EFE76561002002
:105AF000BDE8F0812DE9F04104006569002617E05A
:105B0000206950F8360079010144206950F83600C8
:105B10007A011044C269002A06D05068002803D0D8
:105B2000C9686068526890477F1C4745E8D3761C77
:105B3000E069FBF708FA864207D266613100A06887
:105B4000FAF7EAFF80460027EFE765610020BDE82D
:105B5000F0812DE9FC4704000D0066696561E0698C
:105B6000FBF7F1F9854209D3E069FBF7ECF9020094
:105B700029003248FBF73AF8012057E02900A068D5
:105B8000FAF7CAFF07005FF0000808E0484640B295
:105B9000002843D1684600F0EDF918F10108B84536
:105BA00042D2206950F835005FEA481100EB010944
:105BB000206950F835005FEA48110844D0F81CA06D
:105BC0005046FFF7B7FE61684A6B0100684600F077
:105BD000DEF9DAF80C00002801D1F7F79DFF4946FD
:105BE0006068DAF80C2090478146E068E16809684F
:105BF00049698847484640B20128C7D15046FFF757
:105C000099FE4FFA89F94B46424601000C48FAF7D3
:105C1000EDFF684600F0AEF9012007E0684600F0AD
:105C2000A9F9484640B201E066610020BDE8F68768
:105C300000000000CCBC050058BF05009CC005005A
:105C4000D0C005002DE9F8430400002500E06D1CDC
:105C5000E069FBF778F985424BD22900E06900F052
:105C6000A6F9060000271EE05FF000084846FAF794
:105C700014FF092808D14846FAF75AFFFAF767FFD8
:105C80000021FAF789FF80460099206900EBC500E2
:105C900040680C2202FB07F250F802904246484648
:105CA000FCF752FD7F1C3000FBF76CF9FBF76FF936
:105CB0008742CCD23000FBF765F93900FBF772F967
:105CC00081464846FAF708FF0028EBD0694620696C
:105CD00000EBC50040680C2202FB07F21044FAF703
:105CE00099FE0100080040B20028BDD0080040B273
:105CF00006E0A069002802D0A06900F05DF900204C
:105D0000BDE8F28380B58068FBF718F9FBF71BF953
:105D100002BD016170470000F8B504000D001600D7
:105D20001F00200000F064F9374820606560A7601C
:105D3000E66000202061002060610020A06120005A
:105D4000F2BD704738B504000D002069012804D069
:105D50002069002801D0F7F7DFFE2900606862683B
:105D60001268D269904732BD70B504000D0016006C
:105D70002069012801D0F7F7CFFEA06800F03CF9B8
:105D80000200330029006068F9F7FCFF70BD38B5E8
:105D900004000D002069032801D0F7F7BDFE6069FB
:105DA00000EB8500006832BDF8B504000D006668A0
:105DB000A06800F021F90700A06800F029F80200AF
:105DC00000972B00E168300034686468A047F2BD9A
:105DD00080B502005068526812689268904701BD11
:105DE00070B504000D00A06800F012F80600A0686D
:105DF00000F002F906EBC00041680C20454301EBBE
:105E0000050070BD416170478CBD050001617047A0
:105E1000006970472DE9F04106000F0015000024CD
:105E200000202860300000F048F88046B8F1CE0F1E
:105E300005DB41461B48FAF7D9FE01242DE0B8F1F5
:105E4000200F11D0414638003A6812689047286008
:105E50002868002821D1404600F044F8010012488B
:105E6000FAF7C4FE012418E0300000F0C7F800285B
:105E700004D10E48FAF7BAFE01240EE0300000F01B
:105E8000BDF8FCF78AF8010038003A68526890477C
:105E900028602868002800D10124200040B2BDE815
:105EA000F08100BF98C6050000C5050090BF050041
:105EB00080B50E21FBF758FC02BD1CB50400002C78
:105EC00001D1F7F729FE2000FBF7B2FF0090200078
:105ED00000F099F8019001A9684600F09AF800686E
:105EE00016BD000011B583B000200190CD200090B8
:105EF0006A4601A903A800F093F8002805D1039C85
:105F000000F09CF850F8240000E0014804B010BDF7
:105F1000D6EF040080B50068FBF710F80021FBF70E
:105F200017F8FBF7F0FFFBF7EDFB02BD80B500684B
:105F3000FBF704F80021FBF70BF8FBF7E4FF02BDC9
:105F400080B50068FAF7FAFF0021FBF701F8FBF7CC
:105F5000E9FFFBF7D7FB02BD80B50068FAF7EEFF5B
:105F60000021FAF7F5FFFBF7DDFF02BD80B500F079
:105F700069F802BD10B504006068002805D02168EA
:105F8000606862681268D2689047200010BD10B542
:105F900004000020206062606068002805D060680E
:105FA00062681268926890472060200010BD80B53A
:105FB000FAF7CEFF02BD000078B585B004000025D9
:105FC00010E068462168142202FB05F211441422F5
:105FD000F9F712F803999DF91020029E3000FCF7A2
:105FE000B3FB6D1CA0688542EBDB002006B070BDE2
:105FF00080B500F028F802BD4069704780B50621E1
:10600000FCF752FA02BD80B500220421FBF7CDFB5C
:1060100002BD02680B689A4201DA0800FFE7704788
:10602000036809688B4203DB11680068814201DA6A
:10603000012000E00020C0B2704700000048704717
:106040004C9C05007047704710B50400A06B0028F9
:1060500001D1F7F761FD24212000A26B904710BD0C
:106060002DE9F04F87B081460F004846FEF754FEF9
:106070008046F868002801D1F7F74EFD38690028FE
:1060800001D1F7F749FDD7F80CA0D7F810B0DFF829
:106090008804026839004046FEF75CFE0400002CCC
:1060A0000DD1DFF8780400903023DFF87424DFF896
:1060B00074144846D9F81440A0470120C7E0DFF81F
:1060C0006804026839004046FEF744FE0500002DD2
:1060D0000DD1DFF8580400903323DFF84424DFF8B3
:1060E00044144846D9F81440A0470120AFE0DFF837
:1060F0004004026839004046FEF72CFE0600DFF837
:106100003404026839004046FEF737FE0700002FCE
:106110000DD1DFF8240400903823DFF80424DFF8E1
:1061200004144846D9F81440A04701208FE094F9A0
:106130001C0097F91C1088421BD097F91C00FAF735
:1061400061FD050094F91C00FAF75CFD03950290CF
:10615000DFF8E8030190DFF8E80300903923DFF867
:10616000C023DFF8E0134846D9F81440A0470120C7
:106170006DE094F91C00012803D195F91C00012859
:1061800013D194F91C00092807D195F91C0009289E
:1061900003D095F91C00122807D194F91C00072898
:1061A00013D195F91C0009280FD095F91C00FAF7B6
:1061B00029FD050094F91C00FAF724FD2A000100CE
:1061C000E148FAF713FD012041E095F91C0012287F
:1061D0000FD16869021D68690168684600F0C0F95E
:1061E00000F0C6F91AF1200201004846D9F8403003
:1061F0009847CDF80CA0029701960095230094F9DA
:106200001C209BF90010484600F0EBF9010049B250
:10621000002901D040B21AE021004046D8F8002001
:106220009269904729004046D8F80020926990472B
:10623000002E05D031004046D8F8002092699047E2
:1062400039004046D8F8002092699047002007B0F6
:10625000BDE8F08F2DE9F047ADF5247D81460D00B6
:106260002869002801D1F7F757FCD5F810A0AA48F3
:1062700002682900484600F042FA0400AA48026871
:106280002900484600F03BFA0600A94802682900A8
:10629000484600F034FA0700A6480268290048463C
:1062A00000F031FA8046E868002801D1F7F734FCA5
:1062B000ED6894F90800012805D0072800F0CE8089
:1062C00009283BD010E19AF90010684600F079F9EE
:1062D00023A869462822F8F78FFE210088A800F03D
:1062E00026FA31008FA800F022FA390096A800F0B3
:1062F0001EFA41469DA800F01AFA404600F07AFACC
:106300000500380000F07EFA0700300000F080FA47
:106310000600200000F07CFA020004959DA803907E
:10632000029796A8019000968FAB88A923A800F049
:1063300077FA00200DF5247DBDE8F08796F9080076
:10634000092849D012287DD1296A4846D9F8442025
:1063500090478146310081A800F0E9F981A800F05A
:1063600007F98246300000F0CDFA4A46514600F067
:10637000D1FA2900684600F00CF919A869462822CC
:10638000F8F73AFE210065A800F0D1F931006CA8B9
:1063900000F0CDF9390073A800F0C9F941467AA898
:1063A00000F0C5F9404600F0DCFA0500380000F0C6
:1063B000E0FA0600200000F0A5FA04957AA90391FE
:1063C000029673A90191CDF800906CAB020065A90B
:1063D00019A800F0D4FAACE72900684600F0D9F813
:1063E0000FA869462822F8F707FE210049A800F007
:1063F0009EF9310050A800F09AF9390057A800F032
:1064000096F941465EA800F092F9404600F0A9FADC
:106410000500380000F0ADFA0700300000F072FA15
:106420000600200000F06EFA04955EA90391029721
:1064300057A90191009650AB020049A90FA800F09E
:106440009EFAC8E796F90800FAF7DCFB94F90820F1
:1064500001003E48FAF7CAFB01206BE796F90800F5
:10646000092835D129000FA800F093F805A80FA935
:106470002822F8F7C1FD21002DA800F058F93100BD
:1064800034A800F054F939003BA800F050F9414617
:1064900042A800F04CF9404600F002FB050038002D
:1064A00000F006FB0700300000F02CFA0600200088
:1064B00000F004FB049542A9039102973BA90191C6
:1064C000009634AB02002DA905A800F0FFFA30E7D2
:1064D00096F90800FAF796FB94F9082001001B488A
:1064E000FAF784FB012025E794F90800FAF78AFB04
:1064F00094F9082001001648FAF778FB012019E703
:10650000E0B50021019100210091124B124A13497C
:1065100000F0B8F807BD000014DB0500CCCE050084
:106520002C3C050090CB050018DB0500E0CE0500F3
:106530001CDB050020DB0500F4CE050070D2050051
:1065400050D5050030C9050068C005002CC60500FF
:1065500050C60500556205006160050049600500F0
:1065600010B504002160200000F04DFB200010BD9C
:1065700038B504000125200000F058FB002203E09C
:1065800050F822104D43521C21688A42F8DB280043
:1065900032BD80B58AB04A69524200928A6952423D
:1065A0000192CA6902920A6803924A6804928A6850
:1065B0000592C968069169462822F8F71DFD0BB0BF
:1065C00000BD10B58AB00400080008AA07A940B2AF
:1065D00000F02EFB200069462822F8F70DFD0AB0D6
:1065E00010BD2DE9F84384B00C001D0052B2012A01
:1065F00038D00E9E0D9B0C9F804600200021CDE9D7
:10660000020102A8019000963A002900404600F0DD
:1066100037FB010049B2002901D040B223E0DDF888
:106620003C9019F1040148469DED020BFEF758FA23
:10663000F868002801D0F7F76FFAE868C9F8140085
:10664000F868C9F81800F068C9F81C0019F10C00C6
:10665000009019F108033200210049B2404600F0D1
:1066600028FC00E0002005B0BDE8F083002906D436
:10667000914204DA53F8210010F1010F01D15FF0CB
:10668000FF3070472DE9F04387B0060088461400BC
:106690001D00DDF838900F9F68461C21FAF7FAF9C3
:1066A000CDF80080CDF80490029403950497300053
:1066B00069461C22F8F7A0FC07B0BDE8F08370B56E
:1066C00005000C001600002D01D1F7F725FA002C6B
:1066D00001D1F7F721FA2068031D20680268310014
:1066E0002800FFF7C3FF002801D5002006E020683E
:1066F00000EB8600416828006A6D904770BD80B548
:10670000FFF7DDFF02BD70B505000C001600002D7F
:1067100001D1F7F701FA002C01D1F7F7FDF9606814
:1067200000EB8600416828006A6D904770BD80B517
:10673000002902D04A68002A02D100F0FBFB04E0E5
:106740004A681168121DFFF70BFF01BDF8B506007E
:106750000C001500002C0CD1DFF88400009083237E
:10676000DFF88020DFF8801030007469A047012036
:1067700034E0002D0CD1DFF8740000908423DFF8A2
:106780006420DFF8641030007469A047012025E020
:10679000B06B002809D1164800908523114A124990
:1067A00030007469A047012018E06069076838006C
:1067B000FAF724FA01003000B26B90476169076074
:1067C00060616860002206E001EB82035B6800EB19
:1067D00082046360521CBA42F6DB0020F2BD000066
:1067E0009CD10500D0B3050070CD050088CD050013
:1067F000E8C2050010B50400002C01D1F7F78CF9B0
:10680000206810BD002801D1002000E0006870471A
:1068100010B50400002C01D1F7F77EF9206810BDF7
:106820002DE9F84F2DED028B82B0150099460E9E92
:10683000109CDDF84480129F90ED078AD0ED088A05
:10684000404600F07AFB8346484600F076FB8246DD
:10685000BBF10101404600F072FB0190BBF1010B5E
:106860005B464246BAF10201484600F087FB80468B
:10687000BAF1010A5146484600F0A4FB81465FF098
:10688000000A01E01AF1010A0198824533DA5FF04B
:10689000000B2AE009FB0A0105EB8101D1ED000A9A
:1068A00009FB0B0106EB810191ED001A00EE810A54
:1068B000401C4845EEDBDFED121A002C03D004EB40
:1068C0008B00D0ED001A0AFB08B007EB80000090A7
:1068D000B0EE681AF0EE480A30EE210A00F082FBB2
:1068E000009880ED000A1BF1010BC345CADA9FED49
:1068F000040A0020DDE702B0BDEC028BBDE8F18F99
:106900000000000010B50400002C01D1F7F704F9D5
:10691000206810BD30B400230BE0C45625016DB2D1
:106920002D1164B2241102F8135002EB43056C7070
:106930005B1C022491FBF4F4A342EEDB022391FBE7
:10694000F3F403FB1413002B09D0022391FBF3F3A0
:10695000C05C000140B20011114401F8010C30BCD0
:10696000704710B50400002C01D1F7F7D5F8206866
:1069700010BD002801D1002000E0006870472DE91B
:10698000F84F88B091469A46056846688168079135
:10699000C168069101690591416902918069019080
:1069A000504600F0CAFA022801DAF7F7B5F8159C4C
:1069B000200000F0C2FA012801DAF7F7ADF80198DB
:1069C0000299884201DAF7F7A7F8504600F0B5FAC5
:1069D0008346200000F0B1FA0700791E200000F085
:1069E000AEFA04907F1E3900200000F0EBFA070099
:1069F000BBF10201504600F0E5FAB84201DAF7F7C0
:106A00008BF8149CDDF84880CDF80C90BBF1010B9D
:106A10005946504600F0D6FA81465FF0000A01E080
:106A20001AF1010A0498824537DA5FF0000B2FE073
:106A3000039A09FB0A13D25609FB0B1318F903300A
:106A4000F318AA1802FB0300491C4945F0DB002C8F
:106A500002D054F82B100818059A069900F0D0FAC5
:106A60000090009907984118009102A9684600F02B
:106A700033FB0068009001A9684600F034FB006811
:106A8000009016980AFB07B1009A42541BF1010BC3
:106A9000BB45C5DA00200021D7E709B0BDE8F08F7B
:106AA00010B50400002C01D1F7F736F8206810BDAE
:106AB000002801D1002000E00068704710B50400F4
:106AC000002C01D1F7F728F8206810BD2DE9F84F08
:106AD00088B015001E00D0F80080D0F804B081689E
:106AE0000791C16806910169059141690291806928
:106AF0000190300000F021FA022801DAF7F70CF8D3
:106B0000159C200000F019FA012801DAF7F704F8C3
:106B100001980299884201DAF6F7FEFF300000F092
:106B20000CFA0700200000F008FA8146B9F10101D3
:106B3000200000F004FA0490B9F101094946200050
:106B400000F040FA0400B91E300000F03BFAA04209
:106B500001DAF6F7E1FFDDF85090DDF848A0039583
:106B60007F1E3900300000F02DFA0500002600E0FD
:106B7000761C0498864243DA00273AE0039A05FB24
:106B800006C332F9132005FB07C31AF903301BEBC8
:106B9000030318EB020202FB03F2D31780185941DA
:106BA0001CF1010CAC45E9DBB9F1000F05D009EB94
:106BB000C702D2E9002380185941059B069A00F0CC
:106BC00035FA0090009907984118009102A968468B
:106BD00000F082FA0068009001A9684600F083FA8C
:106BE00000680090169806FB0471009A20F81120A6
:106BF0007F1CA742BCDA002000215FF0000CD1E727
:106C000009B0BDE8F08F70B504000D001600072D27
:106C100001DBF6F781FF2560200000F06BFA04002D
:106C2000AA0031002000F8F7D7F970BD001D7047A9
:106C300003005BB2012B04D1002008600D481060F6
:106C400016E003005BB2032B04D1002008600A4861
:106C500010600DE040B2022805D1084808605FF0DE
:106C60007E50106004E07FF400000860014810606E
:106C7000704700BFFFFF7F7F0000C040000080BF63
:106C80002DE9F04D2DED028B82B0050088461600EF
:106C90001C000C9FD8F80800FDF7FEFE82468B46CC
:106CA000B068FDF7F9FE52465B46F8F7C3F841ECD1
:106CB000180B002C2DD0A068FDF7EEFE41EC100B58
:106CC00051EC180B53EC102BF8F704FB41EC100BB4
:106CD00051EC100B31F0004141EC180BB868FDF796
:106CE000DBFE41EC100B51EC180B53EC102BF8F7BA
:106CF00063FB8A4A8A4BF8F7EFF90AD38948009078
:106D000040F24313834A844928006C69A04701205C
:106D100007E00D9800903B0032004146280000F04B
:106D200005F802B0BDEC028BBDE8F08D38B52DED55
:106D3000028B82B004001D0091ED020AD2ED020A1E
:106D400020EE200A10EE100AFDF7A6FE41EC180B0B
:106D500051EC180B00220023F8F7D6F90AD9724833
:106D600000904FF4A8736B4A6B4920006469A047F8
:106D700001200CE0089CA868FDF78EFE02000B00C5
:106D800051EC180BF8F718FBC4E90001002002B021
:106D9000BDEC028B32BD0000FEB52DED028B82B042
:106DA00006000C980D9D0E9C90ED028AC7680800A5
:106DB00040B2012817D16A46DFED550A3900B0EE1E
:106DC000480A300000F098F9010049B2002901D0CA
:106DD00040B26AE0694605A800F07EF900682860C4
:106DE0000698206060E0080040B203282AD16A4675
:106DF000DFED470A3900B0EE480A300000F07CF9B8
:106E0000010049B2002901D040B24EE0694605A810
:106E100000F062F9006828606A46F1EE080A39005D
:106E2000B0EE480A300000F067F9010049B20029CD
:106E300001D040B239E0694606A800F054F9006874
:106E4000206031E049B202292AD16A46FFEE000AE9
:106E50003900B0EE480A300000F04EF9010049B2A6
:106E6000002901D040B220E0694605A800F034F9BD
:106E7000006828606A46F7EE000A3900B0EE480A5A
:106E8000300000F039F9010049B2002901D040B2C8
:106E90000BE0694606A800F026F90068206003E0D0
:106EA0000598286006982060002002B0BDEC028B97
:106EB000FEBD7FB50024002492F91C40032C0CD1A8
:106EC0000024FF25089E0296019300922B002200C9
:106ED00049B2FFF761FF04B070BD92F91C40092C64
:106EE00003D17FF07F047F25ECE792F91C40072C4B
:106EF00003D10E4C47F6FF75E4E70D4900914FF4BE
:106F0000CB73044A04494469A0470120E3E7000029
:106F10000000000068B5050048CE05007C14AE47AF
:106F2000E17A943F28C7050044CB05000080FFFFAD
:106F3000BCDA05000021016070470068704770B539
:106F400004000D002000FFF7F8FF0600002D01D41B
:106F5000B54201DBF6F7E0FD2000FFF767FE010018
:106F60000120002207E051F8223002E0AA42FAD1C3
:106F700001235843521CB242F8DB70BD2DE9FC419D
:106F800004000D0016001F002900200000F01AF870
:106F900080463900300000F015F8804501D0F6F742
:106FA000BBFD2900200000F00DF8009039003000F2
:106FB00000F008F8019001A9684600F094F8006814
:106FC000BDE8F68138B504000D00002D01D5F6F7B7
:106FD000A3FD2068854201DBF6F79EFD04EB8500EA
:106FE000406832BD00B52DED030A01A96846FEF7E1
:106FF00038F902A9FEF741F990ED000A07BD00003B
:1070000010B51400012C01DB220000E00022012C4D
:1070100001DB002400E06442012313FA02F2504332
:1070200000F0A4F8210000F0BFF810BD2DE9704376
:1070300004000D0090461E00B8F1000F06D558223E
:1070400022492348FAF73CFEAFF3008016F11F00F7
:10705000272806D359221D491D48FAF731FEAFF300
:107060000080201C55F50041B1F5803F09D301D8BF
:10707000002806D35B2215491548FAF721FEAFF325
:1070800000801448804504DA18F500485FEA284873
:1070900001E047F6FF78D6F10F0640465FEAE87157
:1070A000A0FB048900FB059901FB04990120002144
:1070B0003200521EFDF7FEFF18EB000059EB0101F4
:1070C000320000F09FF8BDE87083000038B405007E
:1070D0006CDA05000000FF7F02680B689A4201DA53
:1070E0000800FFE770470A6803689A4201DA08005F
:1070F000FFE77047001D70477CB504000D001600C7
:1071000080EE800AFEF7A6F8DFED130AB4EE600AFF
:10711000F1EE10FA08DBDFED110AB4EE600AF1EED1
:1071200010FA01D5012000E00020C0B200280AD1E9
:107130000B4800904FF4AF730A4A0B492000646972
:10714000A047012006E0BDEEC00A10EE100A451966
:107150003560002076BD00BF000000CF0100004F69
:1071600028C5050004B5050030CE050010B58842DD
:1071700006BFB0F1004F0124002481FB0023002151
:107180008B42ACBF4FF080400648C11710185941E0
:107190004FF000420023F7F713FD0CB16FF00040F1
:1071A00010BD00BF010000C0F8B50E00054648BF85
:1071B0004FF4B37203D4202E07DB40F267120F495D
:1071C0000F48FAF77DFDAFF3008001200021324621
:1071D000FDF770FF441E0021284600F024F800F05F
:1071E000010000EB640104EA050000F023F845FA11
:1071F00006F700F00100C019F2BD00BFD4AA0500D7
:10720000E4D70500D2B2203A22BF41FA02F0C917F2
:1072100070472032D141D04048409140D140484051
:10722000914011417047884202DA4FF0FF307047B9
:1072300000207047814202DA4FF0FF307047002093
:107240007047000010B504461020FCF7CDFC08B1D3
:10725000FBF770FB20600022DFF84C34C0E900230C
:1072600081689FED0C0B81ED000B816881ED020BB5
:10727000806880ED040B84ED020B84ED040B84ED3B
:10728000060B84ED080B84ED0A0B84ED0C0BA26356
:1072900010BD000000000000000000002DE9F041DA
:1072A0002DED108B0D46174682B00646984695ED9B
:1072B000009B97ED00ABB0EE408AF0EE608A51EC97
:1072C0001A0B53EC192BF8F705F8CDE9000195EDF1
:1072D00002BBD7E9020153EC1B2BF7F7FBFF41EC94
:1072E0001D0BD7E9040195ED04CB53EC1C2BF7F7EC
:1072F000F1FFB46B41EC1E0B6CB3DDE9002351ECE4
:10730000180B81F00041F7F7E7FE41EC1F0B5AD252
:10731000DDE9000153EC182BF7F7DEFE53D251ECF8
:107320001F0B53EC1D2BF7F7D7FE4CD251EC1D0B66
:1073300053EC182BF7F7D0FE45D251EC1F0B53EC52
:107340001E2BF7F7C9FE3ED251EC1E0B53EC182B47
:10735000F7F7C2FE37D2601CF7F7AAFF41EC180B13
:107360002046F7F7A5FF53EC192BF7F763FD53EC15
:107370001A2BF8F787F953EC182BF8F71DF8C5E925
:1073800000012046F7F794FF53EC1B2BF7F752FD53
:10739000D7E90223F8F776F953EC182BF8F70CF835
:1073A000C5E902012046F7F783FF53EC1C2BF7F7E2
:1073B00041FDD7E90423F8F765F953EC182BF7F7EB
:1073C000FBFFC5E904014445BCBF641CB46302B0C3
:1073D000BDEC108BBDE8F0812DE9FC412DED088B53
:1073E00004460D469846B0EE40AAF0EE60AA9AB068
:1073F00016469FEDAE0B42F2107305F108012846C8
:10740000FFF74CFFD6E90401D5E90623F7F762FF41
:107410009FEDA8BB53EC1B2BF7F70CFD53EC1A2B7D
:10742000F7F708FDD5E9042341EC120BD6E9020178
:10743000B0EE428AF0EE628AF7F74CFF53EC1B2B5A
:10744000F7F7F8FC53EC1A2BF7F7F4FCD5E9022315
:1074500041EC110BD6E90001B0EE482AF0EE682AA3
:10746000B0EE418AF0EE618AB0EE429AF0EE629A96
:10747000F7F730FF53EC1B2BF7F7DCFC53EC1A2B20
:10748000F7F7D8FC41EC100BB0EE492AF0EE692A70
:10749000B0EE481AF0EE681A0EA8FBF7F5FA0246AD
:1074A00029686846FBF7A8FB2868694600F016F9CA
:1074B000012102A8FBF74DFE00216846FBF749FEBB
:1074C00003216846FCF7F8FE00989FED7E9B80ED57
:1074D000009B9FED7A8B009880ED029B9FED790BCE
:1074E000009880ED048B0AA898ED043B98ED022BE0
:1074F00098ED001BFBF7A0FA0246296802A8FBF7EB
:107500007BFB296812A8FBF713FC12AA02A906A8A4
:10751000FBF772FB012114A8FBF71BFE012104A855
:10752000FBF717FE08A902A800F0F3F86A4602A9C3
:1075300004A8FBF763FF012102A8FBF70AFE08A9D4
:1075400002A800F0E6F804A800F0F2F8039E012E6D
:10755000B0EE40AAF0EE60AA11DB029F97ED000B9F
:1075600051EC100B53EC102BF7F764FC53EC192B78
:10757000F8F788F80837761E41EC190BEED1B0EE1B
:10758000490AF0EE690AFBF729FE51EC1A0B53EC9D
:10759000102BF7F711FF41EC100BFBF7E9FDB0EEF4
:1075A000409AF0EE609A012102A8FBF7D2FD98ED17
:1075B000000B98ED04AB98ED02BB53EC102B51EC93
:1075C000100BF7F737FC264607460C4653EC1B2BEF
:1075D00051EC1B0BF7F72EFC3A462346F8F752F80E
:1075E00007460C4653EC1A2B51EC1A0BF7F722FC0A
:1075F0003A462346F8F746F841EC100BFBF7EEFD50
:1076000053EC102B51EC180BF8F73CF841EC100B35
:1076100053EC102BF7F70EFC2C4A2D4BF7F7CCFE52
:1076200041EC100BFBF7AAFD53EC102B29482A491B
:10763000F7F700FC53EC192BF7F7FCFB04AC41EC1B
:10764000100B214616A8FBF787F92A68014612A8F5
:10765000FBF7D2FA286812A900F040F8012114A81B
:10766000FBF777FD012118A8FBF773FD2968304669
:10767000FBF786FB012104A8FBF76BFD012108A89D
:10768000FBF767FD01210CA8FBF763FD01216846AC
:10769000FBF75FFD012110A8FBF75BFD1AB0BDEC05
:1076A000088BBDE8F38100000000F03F00000000FF
:1076B00000002440399D52A246DF913F00000000A7
:1076C0000000F0BF00000000000000007C14AE4786
:1076D000E17A84BF9A9999999999B93F38B50D463D
:1076E000044604F1080005F1080195ED000B84ED56
:1076F000000B88420BD00121FBF72BFDA968A1608C
:107700000021E868E06005F10800FBF722FD204653
:1077100032BD38B50D4604460021FBF71AFD2A6834
:10772000696801232046FBF74CFF204632BD00006C
:1077300070B52DED028B056846689FED108B002417
:107740000FE095ED000B53EC102B51EC100BF7F7FD
:1077500071FB53EC182BF7F795FF41EC180B641CE9
:107760000835B442EDDBB0EE480AF0EE680ABDEC35
:10777000028BBDE87040FBF731BD00BF0000000088
:10778000000000000020704738B50D460446C821AF
:1077900000F0BEF92868206005223221201D00F08B
:1077A000BBF90522322104F1280000F0B5F904F1FB
:1077B0005000FFF747FD04F1900000F009FA204661
:1077C00032BD0000F8B52DED108B0E469AB096ED47
:1077D000009A96ED018AD6ED028A29EE090A08EE92
:1077E000080A054608EEA80A00F062FA86ED060AC5
:1077F000DFEDBB9A05F1A80420EE290ABDEEC00A10
:1078000084ED010AB0EE681AF0EE480AB0EE490ABB
:10781000281D00F0ABF995ED078A95ED081AD5ED16
:10782000090A28EE080A01EE010A00EEA00A00F09B
:107830003FFA20EE290ABDEEC00A84ED000A8DED64
:107840000E8A0EA9286A0F909FEDA6DB686A109039
:107850009FEDA6CB05F1900000F0CAF984ED070A70
:1078600096ED039A96ED048AD6ED058A29EE090A6B
:1078700008EE080A08EEA80A00F01AFA86ED070AD0
:10788000BDEEC00A84ED030AB0EE681AF0EE480AB5
:10789000B0EE490A05F1280000F068F995ED109A5C
:1078A000D5ED118A95ED128A29EE090A08EEA80A8B
:1078B00008EE080A00F0FCF9BDEEC00A84ED020AE9
:1078C00019EE100AFDF7E8F8CDE9080108AE18EE48
:1078D000900AFDF7E1F8C6E9020118EE100AFDF77B
:1078E000DBF8C6E9040102AEE869FDF7D5F8CDE999
:1078F0000201286AFDF7D0F8C6E90201686AFDF7BF
:10790000CBF8C6E90401002214A8002100230EC010
:107910000EC014A900919FED770B02AB08AA05F1E8
:10792000500101A8FFF758FD01A800F0D0F9286D1B
:1079300090ED008B806890ED009B90ED02AB90ED98
:1079400004BB53EC182B51EC1A0BF7F773FA0646ED
:107950000F4653EC192B51EC1B0BF7F76BFA024651
:107960000B4630463946F7F7B5FC53EC1D2BF7F7BD
:1079700061FA00F0BDF900EE100A00F0EDF910EE2A
:10798000100AFDF789F853EC1C2BF7F753FA5D4A00
:107990005D4BF7F711FDF7F76DFC206153EC182BE9
:1079A00051EC180BF7F746FA41EC1F0B53EC1B2B6D
:1079B00051EC1B0BF7F73EFA53EC1F2BF7F762FE67
:1079C00053EC1D2BF7F736FA9FED4CEB53EC1E2BC7
:1079D000F7F758FE00F08CF900EE900ACDED000AA2
:1079E00053EC1A2B51EC1B0BF7F724FA06460F4603
:1079F00053EC182B51EC190BF7F71CFA32463B46A7
:107A0000F7F740FE53EC1D2BF7F714FA00F070F96E
:107A100000EE100ADDED000A00F0CCF910EE100ABD
:107A2000FDF73AF853EC1C2BF7F704FA354A364BBE
:107A3000F7F7C2FCF7F71EFC5A38A06153EC192B7C
:107A400051EC190BF7F7F6F953EC1F2BF7F71AFE69
:107A500053EC1D2BF7F7EEF953EC1E2BF7F712FE44
:107A600000F046F900EE900AB0EE60EA53EC192BF4
:107A700051EC1A0BF7F7DEF906460F4653EC182BBC
:107A800051EC1B0BF7F7D6F932463B46F7F7FAFDF8
:107A900053EC1D2BF7F7CEF900F02AF900EE100A8F
:107AA000F0EE4E0A00F086F910EE100AFCF7F4FF33
:107AB00053EC1C2BF7F7BEF9124A134BF7F77CFC7B
:107AC000F7F7D8FB6061A06910F1B40FBCBF00F5F7
:107AD000B470A0611AB00020BDEC108BF2BD0000A4
:107AE0000000C8420000000000000040000000004C
:107AF000008066407B14AE47E17A943F00000000AE
:107B00000000F0BF182D4454FB21094070470000CD
:107B10000022FAF71DBE000000EE902AF8EEE00AFF
:107B20009FED111A00EE101A60EE810AB8EEC00A3D
:107B3000B0EE001A20EE010A30EE201A30EEC00A34
:107B400080EE010A80ED000A80EE810A002180EDBE
:107B5000010A80ED020AC160016141618161C16178
:107B60000162002070470000C3F5C84090ED012A73
:107B7000D0ED021AD0ED033AD0ED002A80ED030AD1
:107B800022EE003A01EEA33AD0ED063A02EEE33AD5
:107B900080ED063A22EE200A90ED043AC0ED040A88
:107BA00001EE830A90ED073AD0ED050A80ED051A43
:107BB00002EEC30A80ED070A22EE010A01EEA00AD6
:107BC000D0ED080A02EEE00A80ED080A00207047B6
:107BD00080B518B91820F5F7C7FB40B10021016046
:107BE0003249416000218160C1600161416102BD93
:107BF00010B504462DED028B2068401C20609FEDDF
